:020000040800F2
:10000000D0C50020E1010008496100088D5A0008B0
:1000100045610008510C000821C8000800000000DC
:10002000000000000000000000000000490100087E
:10003000D1150008000000008D01000835BF000840
:10004000FB010008FB010008FB010008FB010008A0
:10005000FB010008FB010008FB010008FB01000890
:10006000FB010008FB010008FB010008FB01000880
:10007000FB010008551500086515000875150008F6
:1000800085150008FB010008FB010008FB010008C2
:10009000FB010008FB010008FB010008FB01000850
:1000A000FB010008D1BF0008FB010008FB010008AC
:1000B000FB010008FB010008E1BF0008FB0100088C
:1000C000FB010008FB010008FB010008FB01000820
:1000D000FB010008ADC6000829C70008A5C7000835
:1000E000FB010008FB010008FB010008FB01000800
:1000F000F1BF0008FB010008FB010008FB0100083C
:10010000FB010008FB010008FB010008FB010008DF
:10011000FB010008FB010008FB010008FB010008CF
:10012000FB010008FB010008FB0100089515000811
:10013000DFF810D000F0FCF900480047EDD00008CF
:10014000AFF30080D0C50020224B19680868B0E8E2
:10015000F00F80F30988BFF36F8F4FF0000080F33A
:1001600011884EF00D0E7047000000000648006830
:10017000006880F3088862B661B6BFF34F8FBFF3A3
:100180006F8F00DF00BF00BF08ED00E0EFF30980D4
:10019000BFF36F8F0F4B1A6820E9F00F106008B59E
:1001A0004FF0500080F31188BFF34F8FBFF36F8F74
:1001B0000EF0F0FD4FF0000080F31188BDE808401C
:1001C00019680868B0E8F00F80F30988BFF36F8FF3
:1001D000704700BF100A0020EFF305807047000051
:1001E0000648804706480047FEE7FEE7FEE7FEE7D1
:1001F000FEE7FEE7FEE7FEE7FEE7FEE7CFBF00080B
:1002000031010008202A04DB203A21FA02F0002103
:10021000704721FA02F3D040C2F120029140084316
:1002200019467047A0F16101192900D8203870479C
:1002300040EA01039B0703D009E008C9121F08C068
:10024000042AFAD203E011F8013B00F8013B521EE8
:10025000F9D27047D2B201E000F8012B491EFBD25F
:1002600070470022F6E710B513460A4604461946C1
:10027000FFF7F0FF204610BDF0B480EA0102D40F72
:100280004200B2EB410F02D20246084611464A0034
:1002900042D0C30DDDB2C1F3C752AD1A202D35DAFD
:1002A000C1F3160141F4000204B15242C5F1200627
:1002B00002FA06F12A411044B3EBD05F23D0C4B157
:1002C000012DA0EBC35009DCF0BC4FF0004202EA64
:1002D000C352DBB200F5000000F0FBB8400000F1B3
:1002E000807000EBC350A0F1807040EAD1704900EB
:1002F00009E0490841EAC071A0EBC35000F50000D5
:10030000400800EBC350F0BC00F0DAB861420122B3
:1003100002EB4101001BF6E7F0BC704781F00041A1
:10032000AAE780F00040A7E780EA010210B502F0DA
:100330000043400022D04A001FD0010E01EB1261A1
:10034000C0F35600C2F3560240F4000042F400022B
:10035000A0FB022000047F39140400D0401C50EAA6
:10036000124001D44000491EC2B20C0604EBD0106A
:10037000401C4008802A02D003E0002010BD20F07D
:100380000100002900DA0020184310BD30B480EAD3
:10039000010202F0004530F0004221F0004013D08D
:1003A00090B1C30DD40DC2F31601C0F31600E41AC8
:1003B00041F4000140F400027D34914201D3641CF9
:1003C00000E04900002C02DA30BC002070474FF4F6
:1003D00000000023914201D3891A034340084FEAE9
:1003E0004101F7D151B1914202D14FF0004105E0F6
:1003F00002D24FF0010101E06FF0010103EBC450A4
:10040000284430BC00F05CB8C10F80EAE0700844BA
:10041000CA079623002100F05CB8962300221146FB
:1004200000F057B800F0004220F00040C10DC0F3CA
:10043000160040F400007F2901DA00207047962959
:1004400003DCC1F19601C84001E096398840002ADA
:10045000F4D04042704720F00040C10DC0F31600B8
:1004600040F400007F2901DA00207047962903DC60
:10047000C1F19601C8407047963988407047000026
:10048000002801DBC0F10040002901DBC1F100417F
:100490008142704730B50B460146002020220124DE
:1004A00009E021FA02F59D4205D303FA02F5491B42
:1004B00004FA02F52844151EA2F10102F1DC30BD58
:1004C0000029A8BF7047401C490008BF20F0010068
:1004D000704710B4B0FA80FC00FA0CF050EA010446
:1004E00004BF10BC704749B1CCF1200421FA04F4D8
:1004F00011FA0CF118BF012121430843A3EB0C01B1
:10050000CB1D4FEA00614FEA102042BF002010BC13
:10051000704700EBC35010440029A4BF10BC7047C3
:10052000401C490008BF20F0010010BC70470000CB
:10053000064C074D06E0E06840F0010394E8070030
:1005400098471034AC42F6D3FFF7F6FDEC0D0108E6
:100550000C0E010870B58D1810F8014B14F0030251
:1005600001D110F8012B231106D110F8013B03E053
:1005700010F8016B01F8016B521EF9D1ABB110F804
:10058000012B04F00C048A1A0C2C03D0A2EB841269
:100590009B1C08E010F8014BA2EB0422F8E712F8CC
:1005A000014B01F8014B5B1EF9D5A942D4D30020C1
:1005B00070BD000010B5124A302907D1A1F13003F7
:1005C00003EBC30302EBC303588018E0312901DABF
:1005D0003F2908DC04B2A1F1300303EBC30302EBB3
:1005E000C303DC800BE0412901DA4F2907DC04B2A8
:1005F000A1F1300303EBC30302EBC3039C8010BDE6
:10060000802E00202DE9F04104461746DFF850C146
:100610004FF6FF70844201D0814203D14FF6FF7044
:10062000BDE8F0810026002244F25060844201DAE5
:10063000264602E048F6A040061B40F6E44086420B
:1006400000DD064647480088301AB0F5FA7F04DD21
:100650004448008800F5FA7609E042480088801B8B
:10066000B0F5FA7F03DD3F480088A0F5FA76DFF8A1
:10067000F480A8F80060344644F25060814201DA08
:100680000A4602E048F6A040421A012F1FDD364814
:1006900030F81300101AB0F5FA7F05DD324830F853
:1006A000130000F5FA720BE02F4830F81300801A9F
:1006B000B0F5FA7F04DD2C4830F81300A0F5FA728B
:1006C000DFF8A48028F813201146BF1E30E0274829
:1006D00030F81300101AB0F5FA7F05DD234830F822
:1006E000130000F5FA720BE0204830F81300801A6E
:1006F000B0F5FA7F04DD1D4830F81300A0F5FA725A
:10070000DFF8688028F813201146A14208DB091B96
:1007100008B203EBC3080CEBC808A8F8060007E012
:10072000641A20B203EBC3080CEBC808A8F8060053
:100730003FB90D1B0E48854209DA48F6A040054432
:1007400005E00D1948F6A040854200DB2D1A46F65B
:100750007810854202DDA5F50C45A03D28465FE7EF
:10076000802E002052030020602E0020402E00200A
:10077000B0B9FFFF2DE9F041064688462C4C002514
:100780003F2E03DDA6F14000054402E0A6F1300053
:10079000054405EBC50004EBC000083005EBC501BE
:1007A00034F8311000EBC107224878603860608867
:1007B0004FF6FF71884228D0B4F90400401C68B19C
:1007C00008F040039A1C05EBC50304EBC303B3F91F
:1007D000041060882B46FFF715FF3860A6F1300043
:1007E00000EBC00004EBC000B0F90600401C60B193
:1007F00008F0200205EBC50304EBC303B3F90610B0
:1008000060882B46FFF7FEFE786005EBC50034F8E4
:100810003000401C80B205EBC50124F831000828E7
:1008200004DB002005EBC50124F83100BDE8F081B0
:10083000802E0020786FFFFF70B5544C544B012080
:100840000022544900BF9AE00025C0EBC00606EB29
:10085000860601EB4606F586C0EBC00606EB86066B
:1008600001EB46067586012253E09D89012D48D192
:100870001D89EDBB00EBC00504EBC505083505EB94
:10088000C2056D68444EB5420EDCC0EBC00505EBF9
:10089000850501EB45052D8F6D1CC0EBC00606EBF1
:1008A000860601EB4606358700EBC00504EBC5055F
:1008B000083505EBC2056D686D42B1F84260B5427E
:1008C0000BDC00EBC00504EBC505083505EBC205E4
:1008D0006D68B1F84260B54211DDC0EBC00505EBB3
:1008E000850501EB45052D8E6D1CC0EBC00600E0B3
:1008F00007E006EB860601EB4606358608E000BFFA
:1009000006E09D89012D03D11D89012D00D100BF75
:10091000521C022AA9DBC0EBC00505EB850501EBE3
:100920004505AD8FC0EBC00606EB860601EB46061B
:10093000B6F84060B54208DB0125C0EBC00606EB07
:10094000860601EB4606F58718E0C0EBC00505EB0F
:10095000850501EB45056D8EC0EBC00606EB8606EE
:1009600001EB4606B6F84060B54207DB0025C0EB58
:10097000C00606EB860601EB4606F586401C074DD1
:100980002D78A8427FF760AF70BD0000802E002058
:100990006037002000330020786FFFFF50030020F5
:1009A00070B58AB005461D4E1D4C28216846FFF7DC
:1009B00058FCA17F607F41EA0020ADF80000207D57
:1009C000062804D101221749684600F0CDFE012215
:1009D0001449684600F0B2FEBDF800000012287409
:1009E000BDF800006874BDF800004FF6FF71884242
:1009F00003D0BDF80000A6F86C00297C607F81421E
:100A000009D1697CA07F814205D1207D062802D1D1
:100A100001200AB070BD0020FBE700006037002015
:100A2000A238002050F0070810B50146324B334A77
:100A3000588800285DD1187D062812D101205880E1
:100A4000987F2F4C2070062060700020A07001203D
:100A5000E07000202071082060710620294C208061
:100A600045E0B2F87A00C0B1472088747F20C8748E
:100A7000FF20087500204875472088757F20C875BD
:100A8000FF20087600204876472088767F20C876A9
:100A9000FF2008770020487729E0B2F90000000E17
:100AA0008874B2F90000000CC8741088000A087538
:100AB00010784875B2F92800000E8875B2F9280040
:100AC000000CC875108D000A087692F82800487648
:100AD000B2F95000000E8876B2F95000000CC876CA
:100AE000B2F85000000A087792F8500048770020CA
:100AF00010BD0120FCE70000A2380020D8410020F2
:100B000016380020FA09002030B58BB0244D28217A
:100B100001A8FFF7A6FB00240122224901A800F04A
:100B20000DFEBDF804004FF6FF71884203D0BDF8FA
:100B30000400688001E00120688008221A4901A8A9
:100B400000F0FCFD002415E001A830F814004FF679
:100B5000FF71884207D001A830F8141005F1440055
:100B600020F8141004E0012105F1440020F81410CD
:100B7000601CC4B22888A042E6DC00240AE005F12B
:100B8000440030F8140009490988084407490880DE
:100B9000601CC4B22888A042F1DC0BB030BD00005C
:100BA0006037002024F0070860E00708FC090020F7
:100BB0002DE9F0410746244D00240026287D062813
:100BC00040D101206880AA7F2046611CCCB21F4919
:100BD0000A5406222046611CCCB21C490A54122237
:100BE0002046611CCCB219490A54EA7F2046611C98
:100BF000CCB216490A542020425D2046611CCCB27A
:100C000012490A54EA7F2046611CCCB20F490A54AB
:100C10002020425D2046611CCCB20C490A540821B8
:100C20000A4804F035FF064632122046611CCCB259
:100C300006490A542046611CCCB204490E540120D6
:100C4000BDE8F0810020FBE7A23800205C380020DE
:100C500000BFFEE770B58AB00546194E28216846E8
:100C6000FFF7FFFA002400BF08E004F1100006F1CE
:100C70000D01085C2DF81400601CC4B2307EA04247
:100C8000F3DC307D062806D1EA7A0E49684600F08A
:100C90006BFD00F031F9EA7A0A49684600F04EFD32
:100CA000002406E01DF8141004F110002954601C03
:100CB000C4B2307EA042F5DC01200AB070BD000055
:100CC000A238002000F007082DE9F04F85B08046DB
:100CD0000E4615461F4600200490784C012F06D082
:100CE000022F18D0032F2AD0042F54D13CE04046C5
:100CF000E16CFFF713FB7249086008460168E16286
:100D00004FF03F410068FFF7BBFB03D24FF03F407D
:100D10006B49086040E04046616FFFF7FFFA6849A1
:100D200008600846016861654FF03F410068FFF7C1
:100D3000A7FB03D24FF03F40614908602CE09C20A4
:100D400001594046FFF7EAFA5D4908600846016824
:100D5000E1674FF03F410068FFF792FB03D24FF08D
:100D60003F405749086017E0C42001594046FFF74B
:100D7000D5FA5349086008460168A42001514FF094
:100D80003F414F480068FFF77BFB03D24FF03F40E5
:100D90004B49086000E000BF00BF4A49484800686E
:100DA000FFF7C2FA8146FFF756FB4749088000204B
:100DB0004649088039E04548008835F81000424926
:100DC000098888422CDA41480088401C35F8100018
:100DD0003D490988884223DB3C49098836F81100DF
:100DE000FFF71BFB3A49086038490988491C36F867
:100DF0001100FFF712FB374908603449098835F8BC
:100E00001100FFF70AFB3449086030490988491C82
:100E100035F81100FFF701FB3049086000BF08E01A
:100E20002A480088401C2949088028480088C8288A
:100E3000C1DD00BF2448008800280DDC00202449C3
:100E400008602449086024490860244908601E4954
:100E50000880234908802AE01D4801681D48006871
:100E6000FFF75CFA03901C4801681C480068FFF714
:100E700055FA029014480088FFF7CFFA0090164800
:100E800001680098FFF74AFA01900299FFF77EFA8D
:100E900083460399FFF748FA82460D480168504699
:100EA000FFF7EAF98146FFF7D6FA0D4908800C48AA
:100EB0000088FFF7B2FA05B0BDE8F08F583F002078
:100EC000D409002000007A44E4090020E009002051
:100ED000E8090020EC090020F0090020F4090020B6
:100EE000E2090020704770477047704770477047AD
:100EF00070477047704770472DE9F04FA1B0FD4D26
:100F0000DFF8F483FD4FDFF8F893DFF8F8A3FE4E27
:100F1000DFF8F8B3802101A8FFF7A3F90024062227
:100F2000FB4901A800F00AFCBDF804004FF6FF7170
:100F3000884216D1C822F749F74800F015FCC822AC
:100F4000F649F74800F010FCC822F649F64800F0D0
:100F50000BFCC822F549F64800F006FC0320288067
:100F600002E0BDF804002880BDF806004FF6FF71CE
:100F700088420ED1002408E0012105F1340020F858
:100F800014100120A881601C84B22888A042F3DCE0
:100F90000FE000240AE0BDF8061005F1340020F847
:100FA0001410BDF80600A881601C84B22888A042F5
:100FB000F1DCBDF808004FF6FF71884202D1002035
:100FC000688102E0BDF808006881BDF80A004FF6AC
:100FD000FF7188420ED1002408E0012028820121FF
:100FE00005F1140020F81410601C84B22888A04277
:100FF000F3DC0EE0002409E001202882BDF80A108D
:1010000005F1140020F81410601C84B22888A04256
:10101000F2DCBDF80C004FF6FF7188420ED10024BF
:1010200008E001206882012105F1240020F8141055
:10103000601C84B22888A042F3DC0EE0002409E0A2
:1010400001206882BDF80C1005F1240020F814106E
:10105000601C84B22888A042F2DC0122AC49203115
:1010600001A800F06BFBBDF804004FF6FF71884249
:1010700002D10120288102E0BDF80400288101226C
:10108000A349283101A800F059FBBDF804004FF630
:10109000FF71884202D10020A88002E0BDF8040060
:1010A000A88001229A49303101A800F047FBBDF821
:1010B00004004FF6FF71884202D10120E88002E06F
:1010C000BDF80400E88008229A4901A800F036FB28
:1010D000002413E001A830F81400082807DA01A85A
:1010E00030F8141005F1340020F8141004E0012148
:1010F00005F1340020F81410601C84B2082CE9DBE0
:1011000008228C49203901A800F018FB002413E0C4
:1011100001A830F81400082807DA01A830F81410E4
:1011200005F1140020F8141004E0012105F1140069
:1011300020F81410601C84B2082CE9DB08227D49D9
:10114000203101A800F0FAFA002413E001A830F8D9
:101150001400082807DA01A830F8141005F124005B
:1011600020F8141004E0012105F1240020F81410E7
:10117000601C84B2082CE9DB01226549383101A8E2
:1011800000F0DCFABDF804004FF6FF71884203D18D
:101190000020A5F86E0003E0BDF80400A5F86E007D
:1011A00001225B49403101A800F0C8FABDF80400F3
:1011B0004FF6FF71884203D10220A5F8640003E0D6
:1011C000BDF80400A5F8640008225B4901A800F0FE
:1011D000B5FABDF804004FF6FF7188420ED1002425
:1011E00008E00021601C00EB800006EBC0004162BB
:1011F000601C84B22888A042F3DC2AE0002425E0A9
:10120000600001A931F8100000124C49C87060005C
:1012100001A911F81000494988706000401C01A91B
:1012200031F810000012454948706000401C01A9C7
:1012300011F810004149087008460168601C00EB75
:10124000800006EBC0004162601C84B22888A04286
:10125000D6DC01222E49483101A800F06FFABDF812
:1012600004004FF6FF71884203D10120A5F8660003
:1012700003E0BDF80400A5F86600012224495031BE
:1012800001A800F05BFABDF804004FF6FF71884238
:1012900003D10120A5F86C0003E0BDF80400A5F817
:1012A0006C0001221A49643101A800F047FABDF828
:1012B00004004FF6FF71884246D1002412E0052059
:1012C000C4EBC40101EB810108EB4101A1F840002E
:1012D00004EB041101EB410107EB4101A1F86000AF
:1012E000601C84B2082CEADB0520A9F84E00AAF89D
:1012F0007C0025E06037002000330020F638002015
:101300005C4A0020D8410020583F00205C42002069
:1013100000F0070800D007088003002000D4070869
:101320001005002000D80708A006002000DC0708F0
:101330003008002020E0070800C00708F402002061
:101340003084ABF87C002DE0002415E0BDF80400EB
:10135000C4EBC40101EB810108EB4101A1F840009D
:10136000BDF8040004EB041101EB410107EB41015E
:10137000A1F86000601C84B2082CE7DBBDF8040013
:10138000A7F86000BDF80400A9F84E0000BFBDF842
:101390000400AAF87C00BDF804003084BDF8040005
:1013A000ABF87C0021B0BDE8F08F00002DE9F05FC4
:1013B000614DDFF888A1DFF888B1624E4FF0000878
:1013C00000240327E88800287CD1B8F1100F72DAD6
:1013D0008146A888022822D100BF002707E005F136
:1013E000140010F814003844C7B2601CC4B2288836
:1013F000A042F4DC002410E04846421C02F0FF0941
:1014000001F07EFE611C01EB011101EB41010AEBD1
:101410004101A1F85800601CC4B2BC42ECDB288931
:10142000022821D10024002707E005F1340010F83C
:1014300014003844C7B2601CC4B22888A042F4DC4F
:1014400000240FE04846421C02F0FF0901F058FE5C
:10145000611CC1EBC10101EB81010BEB41018886ED
:10146000601CC4B2BC42EDDB0024002707E005F19C
:10147000240010F814003844C7B2601CC4B2288895
:10148000A042F4DC002410E04846421C02F0FF09B0
:1014900001F036FE611C01EBC10202EB411106EBCB
:1014A000410121F81800601CC4B2BC42ECDB08F119
:1014B000010000F0FF08B8F1100F3BDB4FF000080F
:1014C00038E0FFE7E888012834D181031E4802F0A4
:1014D0000FFEA6F852004FF400411B4802F008FE30
:1014E000A6F8A4004021194802F002FEA6F8F60072
:1014F0008021164802F0FCFDA6F848014FF48071E7
:10150000124802F0F5FDA6F89A014FF400710F4859
:1015100002F0EEFDA6F8EC014FF480710C4802F0E9
:10152000E7FDA6F83E024FF40061094802F0E0FD35
:10153000A6F89002BDE8F09F60370020F638002042
:10154000003300205C4A0020000C014000100140E4
:101550000008014010B5024802F0E4F810BD000098
:101560003C0D002010B5024802F0DCF810BD000070
:10157000B40C002010B5024802F0D4F810BD0000F1
:10158000700C002010B5024802F0CCF810BD00002D
:10159000F80C002010B5024802F0C4F810BD00009D
:1015A0009C0A002030B590F840500124AC40C56B37
:1015B0006C60046863604468102C04D10468A26005
:1015C0000468E16003E00468A1600468E26030BD83
:1015D000704772B600BFFEE70021074AD161074994
:1015E000096941F00401054A11611146096941F098
:1015F0004001116170470000A80F00200020024048
:101600000021074AD1610749096941F00201054AF1
:10161000116111464861096941F04001116170474B
:10162000A80F0020002002400022054BDA61054A85
:10163000126942F00102034B1A61018070470000F9
:10164000A80F00200020024000201E49C96801F0B8
:10165000100139B11C49C96941F002011A4AD1612E
:1016600040F010001749C96801F0040139B116496A
:10167000C96941F00101144AD16140F004001149E7
:10168000C96901F0010169B10F49C96941F004015B
:101690000D4AD16100BF0B49C96921F00101094A16
:1016A000D16100BF00BF40F20111884206D1054957
:1016B000C96921F00101034AD16101E00149C86013
:1016C00000BF704700200240A80F002070B50446FC
:1016D00002F026FD054609E0601C38B124B102F095
:1016E0001FFD401BA04201D9032070BD1248C068F5
:1016F00000F001000028EFD10F48C06800F0200082
:1017000020B100BF20200C49C86000BF0A48C06853
:1017100000F0100048B90848C06900F0010020B985
:101720000548C06800F0040018B1FFF78DFF0120E4
:10173000DBE70020D9E7000000200240F0B50346B7
:101740001C4600250026084607E010F8015B10F84B
:10175000016B45EA062724F8027B171EA2F1010C53
:101760001FFA8CF2F1D1F0BD2DE9F04786B080462A
:101770000E4691464FF0000A00270025C6F30A0ADC
:10178000A6EB0A0700200590019000BF03970120F7
:101790000490820239461648FFF7D0FF002507E083
:1017A00038F8150005EB5A01114A22F811006D1C9A
:1017B0004D45F5D302F0E4FA00BF05A901A802F0F7
:1017C00025FA00BF00240BE0094830F814C007EBED
:1017D000440162460023012002F07AFA601C84B2C0
:1017E000B4F5806FF0DB02F069FA06B0BDE8F0876F
:1017F000001000202DE9F04794B00446DFF870A4F3
:101800004FF00008002700260025A94628210AA835
:10181000FEF727FD28216846FEF723FD00BF24E0E0
:10182000152000EB48010AF10D00415C142000EB8B
:1018300048020AF10D00805C41EA00200AA921F863
:101840001800152000EB48010AF10D00415C14203E
:1018500000EB48020AF10D00805C41EA00202DF8FF
:10186000180008F1010000F0FF08B8F1140FD7DBF1
:101870009AF81400062841F0D683FE4890F810909C
:101880004FF6FF7000EA0929FA48407C40EA09094E
:10189000F848877CB9F1010F7ED1012F47D114227E
:1018A000F5490AA8FFF760FF1422F3490AA8FFF7D9
:1018B00045FF00250AE03DF815000AA931F815108A
:1018C000884201D1701CC6B2681C85B2142DF2DBAF
:1018D000142E1DD1E9480088401CE8490880E548DD
:1018E000007C2074E348407C6074E248807CA074F3
:1018F000E048C07CE074084600880A2802D1022033
:10190000207501E001202075012014B0BDE8F087AA
:10191000D848007C2074D748407C6074D548807CCF
:10192000A074D448C07CE07400202075EDE7022F3D
:1019300049D11422D04928310AA8FFF715FF1422F3
:10194000CD4928310AA8FFF7F9FE00250AE03DF845
:1019500015000AA931F81510884201D1701CC6B2D1
:10196000681C85B2142DF2DB142E1DD1C3480088EB
:10197000401CC2490880BF48007C2074BD48407CA0
:101980006074BC48807CA074BA48C07CE07408468F
:101990000088282804D100E070E20220207501E0D0
:1019A000012020750120B0E7B248007C2074B148C6
:1019B000407C6074AF48807CA074AE48C07CE0740A
:1019C00000202075A1E7032F47D11422AA495031E6
:1019D0000AA8FFF7C9FE1422A74950310AA8FFF749
:1019E000ADFE00250AE03DF815000AA931F81510F2
:1019F000884201D1701CC6B2681C85B2142DF2DB7E
:101A0000142E1BD19D480088401C9C490880994891
:101A1000007C20749748407C60749648807CA07459
:101A20009448C07CE074084600880A2802D102204D
:101A3000207501E001202075012066E78D48007CBB
:101A400020748C48407C60748A48807CA0748948EB
:101A5000C07CE0740020207557E7042F47D1142282
:101A6000854978310AA8FFF77FFE14228249783130
:101A70000AA8FFF763FE00250AE03DF815000AA951
:101A800031F81510884201D1701CC6B2681C85B2AD
:101A9000142DF2DB142E1BD178480088401C7749A6
:101AA00008807448007C20747248407C60747148DF
:101AB000807CA0746F48C07CE074084600880A28C7
:101AC00002D10220207501E00120207501201CE7D1
:101AD0006848007C20746748407C60746548807C5E
:101AE000A0746448C07CE074002020750DE7052FC9
:101AF00047D114226049A0310AA8FFF735FE14220D
:101B00005D49A0310AA8FFF719FE00250AE03DF85B
:101B100015000AA931F81510884201D1701CC6B20F
:101B2000681C85B2142DF2DB142E1BD1534800889B
:101B3000401C524908804F48007C20744D48407C2E
:101B400060744C48807CA0744A48C07CE0740846AD
:101B500000880A2802D10220207501E001202075AA
:101B60000120D2E64348007C20744248407C6074E7
:101B70004048807CA0743F48C07CE0740020207501
:101B8000C3E6062F47D114223B49C8310AA8FFF704
:101B9000EBFD14223849C8310AA8FFF7CFFD002514
:101BA0000AE03DF815000AA931F81510884201D164
:101BB000701CC6B2681C85B2142DF2DB142E1BD12A
:101BC0002E480088401C2D4908802A48007C20743B
:101BD0002848407C60742748807CA0742548C07CDD
:101BE000E074084600880A2802D10220207501E02E
:101BF00001202075012088E61E48007C20741D48C5
:101C0000407C60741B48807CA0741A48C07CE074DF
:101C10000020207579E6072F50D114221649F031A3
:101C20000AA8FFF7A1FD14221349F0310AA8FFF713
:101C300085FD00250AE03DF815000AA931F81510C8
:101C4000884201D1701CC6B2681C85B2142DF2DB2B
:101C5000142E24D109480088401C084908800548F2
:101C6000007C20740348407C60740248807C07E05C
:101C7000A23800200029002000D00708F809002021
:101C8000A074FE48C07CE074084600880A2802D18F
:101C90000220207501E001202075012035E6F7487B
:101CA000007C2074F548407C6074F448807CA0740B
:101CB000F248C07CE0740020207526E6082F45D14C
:101CC0001422EF490AA8FFF74FFD1422EC490AA895
:101CD000FFF734FD00250AE03DF815000AA931F8A8
:101CE0001510884201D1701CC6B2681C85B2142D33
:101CF000F2DB142E1BD1E3480088401CE149088028
:101D0000DE48007C2074DD48407C6074DB48807CC9
:101D1000A074DA48C07CE074084600880A2802D122
:101D20000220207501E0012020750120EDE5D34857
:101D3000007C2074D148407C6074D048807CA074C2
:101D4000CE48C07CE07400202075DEE5092F47D125
:101D50001422CB4928310AA8FFF706FD1422C849EE
:101D600028310AA8FFF7EAFC00250AE03DF8150033
:101D70000AA931F81510884201D1701CC6B2681C3E
:101D800085B2142DF2DB142E1BD1BE480088401CF6
:101D9000BC490880B948007C2074B848407C607415
:101DA000B648807CA074B548C07CE07408460088C2
:101DB0000A2802D10220207501E0012020750120AF
:101DC000A3E5AE48007C2074AC48407C6074AB480E
:101DD000807CA074A948C07CE0740020207594E544
:101DE0000A2F41F020811422A54950310AA8FFF79B
:101DF000BBFC1422A24950310AA8FFF79FFC002522
:101E00000AE03DF815000AA931F81510884201D101
:101E1000701CC6B2681C85B2142DF2DB142E1ED1C4
:101E200098480088401C974908809448007C20749A
:101E30009248407C60749148807CA0748F48C07C3C
:101E4000E074084600880A2802D10220207501E0CB
:101E50000120207500208B490880012055E5874826
:101E6000007C20748548407C60748448807CA07429
:101E70008248C07CE0740020207546E5B9F1020F6D
:101E80007ED1012F45D114227F490AA8FFF76CFCAF
:101E900014227D490AA8FFF751FC00250AE03DF80D
:101EA00015000AA931F81510884201D1701CC6B27C
:101EB000681C85B2142DF2DB142E1BD171480088EA
:101EC000401C704908806D48007C20746B48407C41
:101ED00060746A48807CA0746848C07CE0740846DE
:101EE00000880A2802D10220207501E00120207517
:101EF00001200AE56148007C20746048407C6074E1
:101F00005E48807CA0745D48C07CE0740020207531
:101F1000FBE4022F48D114225B4928310AA8FFF7BD
:101F200023FC1422584928310AA8FFF707FC002592
:101F30000AE03DF815000AA931F81510884201D1D0
:101F4000701CC6B2681C85B2142DF2DB142E1CD195
:101F50004C480088401C4B4908804848007C20744D
:101F60004648407C60744548807CA0744348C07CEF
:101F7000E07408460088282803D10220207502E07A
:101F80006CE2012020750120BFE43C48007C2074F5
:101F90003A48407C60743948807CA0743748C07CE3
:101FA000E07400202075B0E4032F47D11422364995
:101FB00050310AA8FFF7D8FB1422334950310AA840
:101FC000FFF7BCFB00250AE03DF815000AA931F82F
:101FD0001510884201D1701CC6B2681C85B2142D40
:101FE000F2DB142E1BD127480088401C25490880AD
:101FF0002248007C20742148407C60741F48807C0B
:10200000A0741E48C07CE074084600880A2802D1EB
:102010000220207501E001202075012075E4174899
:10202000007C20741548407C60741448807CA07447
:102030001248C07CE0740020207566E4042F50D163
:102040001422114978310AA8FFF78EFB14220E4999
:1020500078310AA8FFF772FB00250AE03DF8150069
:102060000AA931F81510884201D1701CC6B2681C4B
:1020700085B2142DF2DB142E24D107E000290020B4
:1020800018D10708F809002000D40708FC48008888
:10209000401CFB490880FB48007C2074F948407CC8
:1020A0006074F848807CA074F648C07CE0740846F0
:1020B00000880A2802D10220207501E00120207545
:1020C000012022E4EF48007C2074EE48407C6074DC
:1020D000EC48807CA074EB48C07CE0740020207544
:1020E00013E4052F45D11422E7490AA8FFF73CFB6A
:1020F0001422E5490AA8FFF721FB00250AE03DF874
:1021000015000AA931F81510884201D1701CC6B219
:10211000681C85B2142DF2DB142E1BD1D848008820
:10212000401CD7490880D748007C2074D548407CA3
:102130006074D448807CA074D248C07CE0740846A7
:1021400000880A2802D10220207501E001202075B4
:10215000012028E4CB48007C2074CA48407C60748D
:10216000C848807CA074C748C07CE07400202075FB
:1021700019E4062F47D11422C34928310AA8FFF7D2
:10218000F3FA1422C04928310AA8FFF7D7FA00252C
:102190000AE03DF815000AA931F81510884201D16E
:1021A000701CC6B2681C85B2142DF2DB142E1BD134
:1021B000B3480088401CB2490880B248007C2074B3
:1021C000B048407C6074AF48807CA074AD48C07C4F
:1021D000E074084600880A2802D10220207501E038
:1021E00001202075012028E4A648007C2074A54821
:1021F000407C6074A348807CA074A248C07CE074DA
:102200000020207519E4072F47D114229E49503130
:102210000AA8FFF7A9FA14229B4950310AA8FFF730
:102220008DFA00250AE03DF815000AA931F81510CD
:10223000884201D1701CC6B2681C85B2142DF2DB35
:10224000142E1BD18E480088401C8D4908808D4873
:10225000007C20748B48407C60748A48807CA07429
:102260008848C07CE074084600880A2802D1022011
:10227000207501E001202075012028E48148007CC0
:1022800020748048407C60747E48807CA0747D48C7
:10229000C07CE0740020207519E4082F47D1142277
:1022A000794978310AA8FFF75FFA14227649783124
:1022B0000AA8FFF743FA00250AE03DF815000AA92D
:1022C00031F81510884201D1701CC6B2681C85B265
:1022D000142DF2DB142E1BD169480088401C68497C
:1022E00008806848007C20746648407C60746548BB
:1022F000807CA0746348C07CE074084600880A288B
:1023000002D10220207501E001202075012028E47F
:102310005C48007C20745B48407C60745948807C39
:10232000A0745848C07CE0740020207519E4092F7F
:1023300047D114225449A0310AA8FFF715FA1422F4
:102340005149A0310AA8FFF7F9F900250AE03DF844
:1023500015000AA931F81510884201D1701CC6B2C7
:10236000681C85B2142DF2DB142E1BD14448008862
:10237000401C434908804348007C20744148407C0D
:1023800060744048807CA0743E48C07CE07408467D
:1023900000880A2802D10220207501E00120207562
:1023A000012028E43748007C20743648407C607463
:1023B0003448807CA0743348C07CE07400202075D1
:1023C00019E40A2F5BD114222F49C8310AA8FFF75C
:1023D000CBF914222C49C8310AA8FFF7AFF9002520
:1023E0000AE03DF815000AA931F81510884201D11C
:1023F000701CC6B2681C85B2142DF2DB142E1ED1DF
:102400001F480088401C1E4908801E48007C20741C
:102410001C48407C60741B48807CA0741948C07CB8
:10242000E074084600880A2802D10220207501E0E5
:102430000120207500201249088001202EE4114857
:10244000007C20740F48407C60740E48807CA0742F
:102450000C48C07CE074002020751FE4B9F1030F24
:102460007ED1012F4ED1142208490AA8FFF77CF92A
:10247000142206490AA8FFF761F9002513E015E3C5
:10248000F809002000290020A0D4070800D8070878
:102490003DF815000AA931F81510884201D1701CC9
:1024A000C6B2681C85B2142DF2DB142E1BD1FB487A
:1024B0000088401CF9490880F948007C2074F848DD
:1024C000407C6074F648807CA074F548C07CE07461
:1024D000084600880A2802D10220207501E0012068
:1024E0002075012022E4EE48007C2074EC48407CFA
:1024F0006074EB48807CA074E948C07CE0740020E4
:10250000207513E4022F47D11422E6490AA8FFF7E9
:102510002BF91422E3490AA8FFF710F900250AE075
:102520003DF815000AA931F81510884201D1701C38
:10253000C6B2681C85B2142DF2DB142E1DD1D7480B
:102540000088401CD5490880D548007C2074D448B8
:10255000407C6074D248807CA074D148C07C00E08C
:1025600071E2E07408460088282802D10220207514
:1025700001E001202075012022E4C948007C20747C
:10258000C748407C6074C648807CA074C448C07C46
:10259000E0740020207513E4032F47D11422C149B1
:1025A00028310AA8FFF7E0F81422BE4928310AA80A
:1025B000FFF7C4F800250AE03DF815000AA931F834
:1025C0001510884201D1701CC6B2681C85B2142D4A
:1025D000F2DB142E1BD1B1480088401CAF490880A3
:1025E000AF48007C2074AE48407C6074AC48807C6E
:1025F000A074AB48C07CE074084600880A2802D169
:102600000220207501E001202075012026E4A44865
:10261000007C2074A248407C6074A148807CA07437
:102620009F48C07CE0740020207517E4042F47D138
:1026300014229C4950310AA8FFF796F814229949B0
:1026400050310AA8FFF77AF800250AE03DF8150096
:102650000AA931F81510884201D1701CC6B2681C55
:1026600085B2142DF2DB142E1BD18C480088401C3F
:102670008A4908808A48007C20748948407C6074BC
:102680008748807CA0748648C07CE0740846008837
:102690000A2802D10220207501E0012020750120C6
:1026A00027E47F48007C20747D48407C60747C482F
:1026B000807CA0747A48C07CE0740020207518E407
:1026C000052F47D11422774978310AA8FFF74CF833
:1026D0001422744978310AA8FFF730F800250AE07F
:1026E0003DF815000AA931F81510884201D1701C77
:1026F000C6B2681C85B2142DF2DB142E1BD16748BC
:102700000088401C654908806548007C2074644846
:10271000407C60746248807CA0746148C07CE07436
:10272000084600880A2802D10220207501E0012015
:102730002075012028E45A48007C20745848407CC9
:1027400060745748807CA0745548C07CE0740020B9
:10275000207519E4062F47D114225249A0310AA846
:10276000FFF702F814224F49A0310AA8FEF7E6FF4E
:1027700000250AE03DF815000AA931F81510884235
:1027800001D1701CC6B2681C85B2142DF2DB142E68
:102790001BD142480088401C404908804048007CCA
:1027A00020743F48407C60743D48807CA0743C4865
:1027B000C07CE074084600880A2802D102202075F7
:1027C00001E001202075012028E43548007C2074B8
:1027D0003348407C60743248807CA0743048C07CB0
:1027E000E0740020207519E4072F47D114222D49E9
:1027F000C8310AA8FEF7B8FF14222A49C8310AA82E
:10280000FEF79CFF00250AE03DF815000AA931F803
:102810001510884201D1701CC6B2681C85B2142DF7
:10282000F2DB142E1BD11D480088401C1B49088078
:102830001B48007C20741A48407C60741848807CD7
:10284000A0741748C07CE074084600880A2802D1AA
:102850000220207501E001202075012031E410489C
:10286000007C20740E48407C60740D48807CA0740D
:102870000B48C07CE0740020207522E4082F4DD165
:1028800014220849F0310AA8FEF76EFF1422054908
:10289000F0310AA8FEF752FF002510E0F8090020E9
:1028A0000029002028D807083DF815000AA931F8AA
:1028B0001510884201D1701CC6B2681C85B2142D57
:1028C000F2DB142E1BD1FD480088401CFB49088018
:1028D000FB48007C2074FA48407C6074F848807C97
:1028E000A074F748C07CE074084600880A2802D12A
:1028F0000220207501E001202075012029E4F04824
:10290000007C2074EE48407C6074ED48807CA074AC
:10291000EB48C07CE074002020751AE4092F45D1F3
:102920001422E8490AA8FEF71FFF1422E5490AA865
:10293000FEF704FF00250AE03DF815000AA931F86A
:102940001510884201D1701CC6B2681C85B2142DC6
:10295000F2DB142E1BD1D9480088401CD7490880CF
:10296000D748007C2074D648407C6074D448807C72
:10297000A074D348C07CE074084600880A2802D1BD
:102980000220207501E00120207501202BE4CC48B5
:10299000007C2074CA48407C6074C948807CA07464
:1029A000C748C07CE074002020751CE40A2F7DD14C
:1029B0001422C44928310AA8FEF7D6FE1422C149C0
:1029C00028310AA8FEF7BAFE00250AE03DF81500F6
:1029D0000AA931F81510884201D1701CC6B2681CD2
:1029E00085B2142DF2DB142E1ED1B4480088401C91
:1029F000B2490880B248007C2074B148407C6074C1
:102A0000AF48807CA074AE48C07CE0740846008863
:102A10000A2802D10220207501E001202075002043
:102A2000A6490880012028E4A548007C2074A44819
:102A3000407C6074A248807CA074A148C07CE07493
:102A40000020207519E4B9F1040FB0D1012F47D14E
:102A500014229D490AA8FEF787FE14229A490AA863
:102A6000FEF76CFE00250AE03DF815000AA931F8D2
:102A70001510884201D1701CC6B2681C85B2142D95
:102A8000F2DB142E1DD18D480088401C8B49088034
:102A90008B48007C20748A48407C60748848807C25
:102AA000A0748748C07CE074084600E0BBE2008860
:102AB0000A2802D10220207501E0012020750120A2
:102AC00025E47F48007C20747D48407C60747C480D
:102AD000807CA0747A48C07CE0740020207516E4E5
:102AE000022F47D11422784928310AA8FEF73CFE6C
:102AF0001422754928310AA8FEF720FE00250AE0B5
:102B00003DF815000AA931F81510884201D1701C52
:102B1000C6B2681C85B2142DF2DB142E1BD1674897
:102B20000088401C654908806548007C2074644822
:102B3000407C60746248807CA0746148C07CE07412
:102B400008460088282802D10220207501E00120D3
:102B50002075012025E45A48007C20745848407CA8
:102B600060745748807CA0745548C07CE074002095
:102B7000207516E4032F47D11422534950310AA877
:102B8000FEF7F2FD1422504950310AA8FEF7D6FD97
:102B900000250AE03DF815000AA931F81510884211
:102BA00001D1701CC6B2681C85B2142DF2DB142E44
:102BB0001BD142480088401C404908804048007CA6
:102BC00020743F48407C60743D48807CA0743C4841
:102BD000C07CE074084600880A2802D102202075D3
:102BE00001E001202075012028E43548007C207494
:102BF0003348407C60743248807CA0743048C07C8C
:102C0000E0740020207519E4042F47D114222E49C6
:102C100078310AA8FEF7A8FD14222B4978310AA8BA
:102C2000FEF78CFD00250AE03DF815000AA931F8F1
:102C30001510884201D1701CC6B2681C85B2142DD3
:102C4000F2DB142E1BD11D480088401C1B49088054
:102C50001B48007C20741A48407C60741848807CB3
:102C6000A0741748C07CE074084600880A2802D186
:102C70000220207501E001202075012032E4104877
:102C8000007C20740E48407C60740D48807CA074E9
:102C90000B48C07CE0740020207523E4052F4FD141
:102CA00014220949A0310AA8FEF75EFD1422064944
:102CB000A0310AA8FEF742FD002512E0F809002025
:102CC0000029002040D9070800DC07083DF815005E
:102CD0000AA931F81510884201D1701CC6B2681CCF
:102CE00085B2142DF2DB142E1BD1D0480088401C75
:102CF000CE490880CE48007C2074CD48407C60746A
:102D0000CB48807CA074CA48C07CE0740846008828
:102D10000A2802D10220207501E00120207501203F
:102D20002AE4C348007C2074C148407C6074C048D9
:102D3000807CA074BE48C07CE074002020751BE439
:102D4000062F45D11422BB490AA8FEF70DFD142217
:102D5000B8490AA8FEF7F2FC00250AE03DF8150084
:102D60000AA931F81510884201D1701CC6B2681C3E
:102D700085B2142DF2DB142E1BD1AC480088401C08
:102D8000AA490880AA48007C2074A948407C607445
:102D9000A748807CA074A648C07CE07408460088E0
:102DA0000A2802D10220207501E0012020750120AF
:102DB0002CE49F48007C20749D48407C60749C48B3
:102DC000807CA0749A48C07CE074002020751DE4CB
:102DD000072F47D11422974928310AA8FEF7C4FCCF
:102DE0001422944928310AA8FEF7A8FC00250AE01D
:102DF0003DF815000AA931F81510884201D1701C60
:102E0000C6B2681C85B2142DF2DB142E1BD1874884
:102E10000088401C854908808548007C20748448CF
:102E2000407C60748248807CA0748148C07CE074DF
:102E3000084600880A2802D10220207501E00120FE
:102E4000207501202CE47A48007C20747848407C6E
:102E500060747748807CA0747548C07CE074002062
:102E600020751DE4082F47D11422724950310AA859
:102E7000FEF77AFC14226F4950310AA8FEF75EFC77
:102E800000250AE03DF815000AA931F8151088421E
:102E900001D1701CC6B2681C85B2142DF2DB142E51
:102EA0001BD162480088401C604908806048007C53
:102EB00020745F48407C60745D48807CA0745C48EE
:102EC000C07CE074084600880A2802D102202075E0
:102ED00001E00120207501202CE45548007C20747D
:102EE0005348407C60745248807CA0745048C07C39
:102EF000E074002020751DE4092F47D114224D49AC
:102F000078310AA8FEF730FC14224A4978310AA821
:102F1000FEF714FC00250AE03DF815000AA931F877
:102F20001510884201D1701CC6B2681C85B2142DE0
:102F3000F2DB142E1BD13D480088401C3B49088021
:102F40003B48007C20743A48407C60743848807C60
:102F5000A0743748C07CE074084600880A2802D173
:102F60000220207501E00120207501202CE430486A
:102F7000007C20742E48407C60742D48807CA074B6
:102F80002B48C07CE074002020751DE40A2F4AD134
:102F900014222849A0310AA8FEF7E6FB142225498D
:102FA000A0310AA8FEF7CAFB00250AE03DF815008B
:102FB0000AA931F81510884201D1701CC6B2681CEC
:102FC00085B2142DF2DB142E1ED118480088401C47
:102FD000164908801648007C20741548407C6074AF
:102FE0001348807CA0741248C07CE07408460088B6
:102FF0000A2802D10220207501E00120207500205E
:103000000A490880012029E40948007C2074084806
:10301000407C60740648807CA0740548C07CE074E5
:10302000002020751AE4002018E40000F8090020B0
:1030300000290020C8DC070870B500250026264CB2
:103040002648407905022548807905432348407881
:10305000032805D021484078062801D001260CE03D
:103060001E488078022801D0012606E005211B4871
:1030700002F00EFDA84200D001261848407803282F
:1030800021D1012115480078803800EB800202EB45
:10309000801004EB4000A0F888101048C178007838
:1030A000803800EB800202EB801024F810100B48EF
:1030B00001790078803800EB800202EB801004EB8D
:1030C0004000018507E005484078062803D1034801
:1030D000C0780249C87070BD7C4F0020002B0020D2
:1030E0000146064A01EBC10000EB411032F8100026
:1030F00008B9012070470020FCE700005C4A00206E
:1031000070B50546082D3BD2DFE805F0040B121818
:103110001E252C334FF480411B4800F0E9FF044684
:103120002FE04FF40041184800F0E2FF044628E089
:103130004021164800F0DCFF044622E080211348BD
:1031400000F0D6FF04461CE04FF480710F4800F0F9
:10315000CFFF044615E04FF400710C4800F0C8FFA3
:1031600004460EE04FF48071094800F0C1FF0446A8
:1031700007E04FF40061064800F0BAFF044600E0A3
:1031800000BF00BF204670BD000C01400010014090
:103190000008014070B50025234C24484079050201
:1031A00022488079054321484078032807D01F48EA
:1031B0004078062803D001201D49088010E01B48F4
:1031C0008078022803D001201949088008E00521F1
:1031D000164802F05DFCA84202D001201449088084
:1031E000012112480078803800EB0012C2EBC010B9
:1031F00004EB4000A0F8B6100C48C1780078803885
:1032000000EB0012C2EBC01004EB400081820748C3
:1032100001790078803800EB0012C2EBC01004EB9B
:103220004000818770BD00001C580020002B00204A
:10323000FE09002010B5002150480123504A1278A1
:10324000203A02EBC20404EB421200EB4202A2F865
:1032500050304C4A1278212A03D04A4A1278222A46
:103260003CD1484A5278032A04D0464A5278062A6A
:1032700000D00121434A5278032A24D119BB0023EC
:10328000404A1278203A02EBC20404EB421200EBEF
:103290004202A2F84A3001233A4A1278203A02EB5D
:1032A000C20404EB421200EB4202A2F85030354A4D
:1032B000D3781278203A02EBC20404EB421220F8D1
:1032C000123000BF59E02F4A5278062A55D1002902
:1032D00053D12C4AD2782B4BDA704EE0294A12781F
:1032E000232A03D0274A1278242A46D1254A527825
:1032F000032A04D0234A5278062A00D00121214A09
:103300005278032A30D171BB00231E4A1278203A2A
:1033100002EBC20404EB421200EB4202A2F84A3074
:103320000123184A1278203A02EBC20404EB42123D
:1033300000EB4202A2F85030124A1278223A02EB15
:10334000C20404EB421200EB420253840D4A12788D
:10335000223A02EBC20404EB421200EB4202A2F852
:10336000423000BF09E0FFE7064A5278062A04D13E
:1033700019B9044AD278034BDA7010BD5C4A0020B8
:1033800000250020002B002010B504460CB90120B8
:1033900010BD607920B900202071204600F004F8AB
:1033A000012060710020F3E708B5094A01689142E5
:1033B0000DD100BF0749496941F04001054A5161FB
:1033C0001146496901F04001009100BF00BF08BDEE
:1033D0000030024000100240F0B5034600BF5879AB
:1033E000012801D10220F0BD0120587100BF022048
:1033F00018711868046802F0100640F6FE70B040BC
:103400008443D1E9000640EA060502F0100005FAFF
:1034100000F00443186804601868006802F01007A0
:10342000C026BE40B0431E6830601868006802F0D5
:103430001007C026BE40B0431E68306001201871DE
:1034400000BF0020587100BF00BFCCE710B5044694
:103450000CB9012010BD207920B9002060712046F0
:1034600000F008F802202071002020610120207166
:103470000020EFE710B586B00446002002900390CC
:10348000049005902249206888423ED100BF21481F
:10349000C06940F000501F49C8610846C06900F08B
:1034A0000050019000BF00BF00BF0846806940F097
:1034B000040088610846806900F00400019000BFA4
:1034C00000BF202002900320039002A9124800F0C0
:1034D0006FFC124812490860102048600021104813
:1034E00081608021C1604900016189004161202122
:1034F00081610021C16100F0E1FA08B1FEF769F8CD
:1035000000BF0748E060446200BF06B010BD000085
:1035100000740040001002400008014044040240D2
:103520009C0A00200146002291F82100022808D0C0
:103530000420886300BF002081F8200000BF012024
:1035400070470868006820F00E000B681860086873
:10355000006820F001000B68186091F840300120ED
:103560009840CB6B5860012081F8210000BF0020FB
:1035700081F8200000BF1046E2E7000070B5044665
:10358000002594F82100022803D00420A06301251F
:10359000C1E02068006820F00E0021680860206803
:1035A000006820F00100216808605C4920688842BA
:1035B00052D95A4978392068884201D1012047E020
:1035C000564964392068884201D1102040E05349AF
:1035D00050392068884201D1801539E04F493C3983
:1035E0002068884201D1801432E04C492839206893
:1035F000884202D14FF480302AE0484914392068CB
:10360000884202D14FF4801022E044492068884269
:1036100001D140041CE042492068884201D10120C8
:1036200016E03F4914312068884201D110200FE094
:103630003B4928312068884201D1801508E038498B
:103640003C312068884201D1801401E04FF4803081
:103650003349091F086051E03049783920688842B1
:1036600001D1012047E02D4964392068884201D109
:10367000102040E0294950392068884201D1801546
:1036800039E026493C392068884201D1801432E073
:10369000224928392068884202D14FF480302AE03C
:1036A0001E4914392068884202D14FF4801022E06C
:1036B0001A492068884201D140041CE0184920685A
:1036C000884201D1012016E0154914312068884252
:1036D00001D110200FE0124928312068884201D121
:1036E000801508E00E493C312068884201D18014E1
:1036F00001E04FF48030094980394860012084F8A6
:10370000210000BF002084F8200000BF606B10B1D2
:103710002046616B8847284670BD0000800002404B
:103720000804024070B50446E06B0568206806682E
:1037300094F84010042088402840002875D006F0F6
:1037400004000028FAD02068006800F0200028B9A2
:103750002068006820F0040021680860D5492068CE
:10376000884254D9D34978392068884201D104204D
:1037700049E0D04964392068884201D1402042E0C4
:10378000CC4950392068884201D100153BE0C94935
:103790003C392068884202D14FF4804033E0C5496B
:1037A00028392068884202D14FF480202BE0C1499B
:1037B00014392068884202D14FF4800023E0BD49CB
:1037C0002068884201D1C0041DE0BB4920688842BE
:1037D00001D1042017E0B84914312068884201D192
:1037E000402010E0B44928312068884201D10015FA
:1037F00009E0B1493C312068884202D14FF4804051
:1038000001E04FF48020AC49091F086054E0A94949
:1038100078392068884201D104204AE0A5496439FA
:103820002068884202D1402043E04CE0A149503951
:103830002068884201D100153BE09E493C39206850
:10384000884202D14FF4804033E09A4928392068F9
:10385000884202D14FF480202BE096491439206829
:10386000884202D14FF4800023E0924920688842C8
:1038700001D1C0041DE090492068884201D1042094
:1038800017E08D4914312068884201D1402010E0B2
:10389000894928312068884201D1001509E086490C
:1038A0003C312068884202D14FF4804001E04FF45F
:1038B0008020804980394860E06A002802D0204694
:1038C000E16A8847F4E094F84010022088402840DC
:1038D000002871D006F002000028FAD020680068A5
:1038E00000F0200040B92068006820F00A0021683C
:1038F0000860012084F821006E492068884254D96C
:103900006C4978392068884201D1022049E0694930
:1039100064392068884201D1202042E0654950394D
:103920002068884201D140153BE062493C3920685B
:10393000884202D14FF4005033E05E4928392068B4
:10394000884202D14FF400302BE05A4914392068E4
:10395000884202D14FF4001023E056492068884283
:1039600001D180041DE054492068884201D1022021
:1039700017E0514914312068884201D1202010E01D
:103980004D4928312068884201D1401509E04A4953
:103990003C312068884202D14FF4005001E04FF4DE
:1039A00000304549091F086054E0424978392068D1
:1039B000884202D102204AE057E03E49643920683B
:1039C000884201D1202042E03A495039206888429B
:1039D00001D140153BE037493C392068884202D18B
:1039E0004FF4005033E0334928392068884202D12F
:1039F0004FF400302BE02F4914392068884202D15F
:103A00004FF4001023E02B492068884201D1800444
:103A10001DE029492068884201D1022017E026498B
:103A200014312068884201D1202010E02249283139
:103A30002068884201D1401509E01F493C312068C7
:103A4000884202D14FF4005001E04FF40030194990
:103A50008039486000BF002084F8200000BFA06AC1
:103A600030B32046A16A884722E094F8401008202D
:103A700088402840E0B106F00800C8B1206800681E
:103A800020F00E002168086094F840100120884062
:103A9000E16B48600120A06384F8210000BF002092
:103AA00084F8200000BF206B10B12046216B8847AE
:103AB00070BD000080000240080402400146002260
:103AC00009B9012070471E4B086898420BD21D4B64
:103AD0000868C01A1423B0FBF3F08000086419488A
:103AE0000838C8630AE0164B0868C01A1423B0FBF4
:103AF000F3F08000086412480838C863022081F897
:103B000021000868026843F6F0708243D1E901039E
:103B10001843CB6818430B6918434B6918438B69EA
:103B20001843CB6918430243086802600020886389
:103B3000012081F82100002081F8200000BFC1E7AA
:103B400008040240080002402DE9F04104460D46F9
:103B500016461F464FF0000800BF94F820000128C9
:103B600002D10220BDE8F081012084F8200000BFCE
:103B700094F8210001282CD1022084F82100002093
:103B8000A0632068006820F00100216808603B46BF
:103B9000324629462046FDF705FDE06A30B120682F
:103BA000006840F00E00216808600BE020680068A3
:103BB00020F00400216808602068006840F00A00D6
:103BC000216808602068006840F0010021680860F2
:103BD00006E000BF002084F8200000BF4FF002087C
:103BE0004046BFE770B5044600F09AFA06462546FF
:103BF000681C10B104480078054400BF00F090FA3A
:103C0000801BA842FAD370BD0C0A00202DE9F041B8
:103C100004460E460127002500BF2648007E0128E5
:103C200002D10220BDE8F08101202249087600BFC0
:103C30002068022813D14CF25030FDF747FD90BBAD
:103C40000120FDF7C9FC4CF25030FDF73FFD07465F
:103C50001948006920F004001749086123E04CF27C
:103C60005030FDF733FDF0B94FF0FF303060A568FC
:103C700012E02846FDF7C4FC4CF25030FDF726FD5B
:103C800007460D48006920F002000B4908610FB19A
:103C9000356007E005F50065D4E9021001EBC020AE
:103CA000A842E6D800BF00BF00200249087600BF46
:103CB0003846B7E7A80F00200020024003480069FB
:103CC00040F0800001490861002070470020024058
:103CD0002DE9FE4F05468B461746984601260024DF
:103CE0000020029000BF2448007E012802D102205B
:103CF000BDE8FE8F01202049087600BF4CF250300D
:103D0000FDF7E4FC064686BB012D02D1012002909E
:103D100006E0022D02D10220029001E00420029070
:103D200000241EE02201B946C24648465146FCF72F
:103D300069FA80B20190022000FB04B00090019962
:103D4000FDF772FC4CF25030FDF7C0FC06460B4804
:103D5000006920F001000949086106B104E0601C17
:103D6000C4B202988442DDDB00BF00BF00200249DC
:103D7000087600BF3046BBE7A80F002000200240B5
:103D800000200849096901F0800151B10649054A3E
:103D90005160064951601146096901F0800101B185
:103DA000012070470020024023016745AB89EFCD19
:103DB0002DE9F847024600239C467BE14FF00108BD
:103DC00008FA03F4D1F8008008EA0400A0427DD18B
:103DD000DFF8F4A2D1F80480A8EB0A09D0453AD064
:103DE00014DCB8F1030F50D009DCB8F1000F31D06A
:103DF000B8F1010F1CD0B8F1020F49D120E0B8F1A1
:103E0000110F18D0B8F1120F42D11EE0B9F5881F7A
:103E100025D006DCB9F5803F20D0B9F5801F37D119
:103E20001AE0B9F5001F18D0B9F5041F30D117E01A
:103E3000D1F80CC02DE0D1F80C8008F1040C28E07A
:103E4000D1F80C8008F1080C23E0D1F80C8008F1BF
:103E50000C0C1EE000BF00BF00BF00BF00BF00BFD2
:103E6000D1F80880B8F1000F02D14FF0040C0BE03C
:103E7000D1F80880B8F1010F03D14FF0080C14619C
:103E800002E04FF0080C546103E04FF0000C00E03A
:103E900000BF00BFFF2801D8904601E002F10408EE
:103EA0004646FF2802D84FEA830803E0A3F108083A
:103EB0004FEA88084746D6F800804FF00F0909FA04
:103EC00007F928EA09080CFA07F900E07AE048EA5D
:103ED0000908C6F80080D1F8048008F08058B8F1CD
:103EE000805F6FD100BFDFF8E481D8F8188048F018
:103EF0000108DFF8D891C9F81880C846D8F81880AA
:103F000008F00108CDF8008000BF00BF4FEAB938C3
:103F10004FEA930958F829504FEA83784FEA187905
:103F20004FF00F0808FA09F825EA0805DFF8A08124
:103F3000424502D14FF0000824E0DFF89881424565
:103F400002D14FF001081DE0DFF88C81424502D11B
:103F50004FF0020816E0DFF88481424502D14FF0AD
:103F600003080FE0DFF87881424502D14FF00408E2
:103F700008E0DFF87081424502D14FF0050801E00A
:103F80004FF006084FEA83794FEA197908FA09F8E1
:103F900048EA0505DFF850814FEA930948F82950AF
:103FA000D1F8048008F48038B8F5803F0BD1DFF8F1
:103FB0003C81D8F8008048EA0008DFF83091C9F861
:103FC00000800AE075E0DFF82481D8F8008028EA54
:103FD0000008DFF81891C9F80080D1F8048008F4CF
:103FE0000038B8F5003F0ED1DFF8008108F1040871
:103FF000D8F8008048EA0008DFF8F09009F10409D9
:10400000C9F800800DE0DFF8E48008F10408D8F872
:10401000008028EA0008DFF8D49009F10409C9F803
:104020000080D1F8048008F48018B8F5801F0ED104
:10403000DFF8B88008F10808D8F8008048EA0008DE
:10404000DFF8A89009F10809C9F800800DE0DFF851
:104050009C8008F10808D8F8008028EA0008DFF8FA
:104060008C9009F10809C9F80080D1F8048008F49F
:104070000018B8F5001F0ED1DFF8708008F10C08A9
:10408000D8F8008048EA0008DFF8609009F10C09D0
:10409000C9F800800DE0DFF8548008F10C08D8F86A
:1040A000008028EA0008DFF8449009F10C09C9F8FB
:1040B00000805B1CD1F8008028FA03F8B8F1000FEB
:1040C0007FF47CAEBDE8F8870000111000100240BC
:1040D00000080140000C01400010014000140140A4
:1040E00000180140001C014008000140000401408C
:1040F000024693680B400BB1012000E0002070479E
:1041000010B5C26821EA020302EA010443EA04434B
:10411000036110BD0AB1016101E00B040361704746
:104120000148006870470000040A00200348006846
:10413000034909780844014908607047040A0020CF
:104140000C0A002010B50848006840F0100006492D
:104150000860032000F0CCF8002000F007F800F021
:1041600049F8002010BD00000020024070B588B062
:10417000044600250026002221462C2000F07AF873
:104180002C2000F067F800BF1648806940F400500A
:10419000144988610846806900F40050019000BF0E
:1041A00000BF02A903A800F07DF900F0B3F90546AD
:1041B0000D48B5FBF0F0461E0C480D49086040F272
:1041C000E7310B48C160466000210161816000F069
:1041D0007DFC20B9064800F0D9FC08B070BD012074
:1041E000FBE700000010024040420F000034014095
:1041F0005C0F002008B500BF1448806940F0010042
:10420000124988610846806900F00100009000BFF3
:1042100000BF00BF0846C06940F08050C861084632
:10422000C06900F08050009000BF00BF00220F2145
:10423000901E00F01FF800BF0549486820F0E060BC
:1042400040F00070486000BF08BD00000010024050
:104250000000014001460846002809DB00F01F036A
:1042600001229A4043099B0003F1E023C3F8002197
:1042700000BF70472DE9F05F80460D4616460027C7
:1042800008F050FD074639462A46334601F007003C
:10429000C0F1070ABAF1040F02D94FF0040A01E095
:1042A000C0F1070AD14600F1040ABAF1070F02D2A1
:1042B0004FF0000A01E0A0F1030AD4464FF0010AD2
:1042C0000AFA09FAAAF1010A0AEA020A0AFA0CFA37
:1042D0004FF0010B0BFA0CFBABF1010B0BEA030BDC
:1042E0004AEA0B042146404608F024FDBDE8F09F51
:1042F00000BF00F00702064B19684FF6FF03194094
:10430000044B0B4343EA0221014B196000BF704785
:104310000CED00E00000FA0570B504460D460CB93E
:10432000012070BD5A48006800F00700A8420ED274
:104330005748006820F007002843554908600846A0
:10434000006800F00700A84201D00120E9E72078CA
:1043500000F0020002281DD1207800F0040004289B
:1043600005D14C48406840F4E0604A4948602078F4
:1043700000F00800082805D14648406840F4605025
:10438000444948604348406820F0F000A168084371
:1043900040494860207800F0010078B36068012847
:1043A00006D13C48006800F4003090B90120B8E71D
:1043B0006068022806D13748006800F0007040B9F4
:1043C0000120AEE73348006800F0020008B9012080
:1043D000A7E73048406820F00300616808432D4992
:1043E0004860FFF79DFE064609E0FFF799FE801B37
:1043F00041F28831884202D9032092E707E025483C
:10440000406800F00C006168B0EB810FEDD12048EE
:10441000006800F00700A8420ED91D48006820F08F
:10442000070028431A4908600846006800F00700A2
:10443000A84201D0012074E7207800F0040004288D
:1044400007D11448406820F4E060E168084311494E
:104450004860207800F00800082808D10D4840681E
:1044600020F46050216940EAC1000A49486000F028
:1044700061F808494968C1F30311074A515CC84013
:104480000649086006480068FFF770FE002048E70C
:104490000020024000100240B40A0108000A002077
:1044A000080A00200F2202600D4A526802F003023F
:1044B00042600B4A526802F0F0028260084A526879
:1044C00002F4E062C260064A526802F46052D20806
:1044D0000261044A126802F007020A607047000095
:1044E00000100240002002400148006870470000B0
:1044F000000A002000B5FFF7F7FF04494968C1F33F
:104500000221034A515CC84000BD00000010024077
:10451000C40A010800B5FFF7E7FF04494968C1F381
:10452000C221034A515CC84000BD00000010024097
:10453000C40A0108F0B585B00FF26C0C9CE8E010DD
:1045400001A8A0E8E0101CA52D680095002100221C
:10455000002300240020194D696801F00C05F5B115
:10456000042D02D0082D19D101E0154819E001AD44
:10457000C1F38346AC5D01F4803555B10F4D6D68D4
:10458000C5F340451DF805200D4D6543B5FBF2F31D
:1045900002E00C4D04FB05F3184602E000BF08489A
:1045A00000BF00BF05B0F0BD0203040506070809FF
:1045B0000A0B0C0D0E0F101001020000001002403B
:1045C00000127A0000093D00F8B504460CB901203C
:1045D000F8BD207800F00100002878D0F848406845
:1045E00000F00C0004280CD0F548406800F00C00E6
:1045F000082811D1F248406800F48030B0F5803FBF
:104600000AD1EF48006800F4003000285FD06068ED
:1046100000285CD10120DBE700BF6068B0F5803F77
:1046200006D1E748006840F48030E549086028E09A
:10463000606858B9E248006820F48030E0490860BA
:104640000846006820F4802008601AE06068B0F531
:10465000A02F0BD1DA48006840F48020D8490860C8
:104660000846006840F4803008600AE0D4480068DA
:1046700020F48030D24908600846006820F4802089
:10468000086000BF606888B1FFF74AFD054606E094
:10469000FFF746FD401B642801D9032098E7C8486E
:1046A000006800F400300028F2D010E0FFF738FD79
:1046B000054606E0FFF734FD401B642801D90320BE
:1046C00086E7BF48006800F400300028F2D1207867
:1046D00000F00200022857D1B948406800F00C00F1
:1046E00050B1B748406800F00C00082818D1B44811
:1046F000406800F4803098B9B148006800F00200CA
:1047000020B12069012801D0012061E7AC48006890
:1047100020F0F800616940EAC100A949086033E06F
:104720002069E8B10120A7490860FFF7F9FC0546B8
:1047300006E0FFF7F5FC401B022801D9032047E7FC
:104740009F48006800F002000028F2D09C480068F2
:1047500020F0F800616940EAC1009949086013E05F
:10476000002098490860FFF7DBFC054606E0FFF7EC
:10477000D7FC401B022801D9032029E79048006894
:1047800000F002000028F2D1207800F0080008288C
:104790002DD1A069B8B101208B490860FFF7C0FC9A
:1047A000054606E0FFF7BCFC401B022801D90320A8
:1047B0000EE78348406A00F002000028F2D0012092
:1047C00001F0C4FC13E000207F490860FFF7A8FC5B
:1047D000054606E0FFF7A4FC401B022801D9032090
:1047E000F6E67748406A00F002000028F2D120780F
:1047F00000F00400042873D100277148C06900F05C
:10480000805070B900BF6E48C06940F080506C495C
:10481000C8610846C06900F08050009000BF00BF2A
:1048200001276A48006800F48070B0B967480068E2
:1048300040F4807065490860FFF772FC054606E0A9
:10484000FFF76EFC401B642801D90320C0E65F48D7
:10485000006800F480700028F2D000BFE0680128F2
:1048600006D15748006A40F001005549086227E028
:10487000E06858B95248006A20F0010050490862C7
:104880000846006A20F00400086219E0E068052884
:104890000BD14B48006A40F00400494908620846C1
:1048A000006A40F0010008620AE04548006A20F012
:1048B0000100434908620846006A20F004000862CB
:1048C00000BFE068A0B1FFF72BFC054609E0FFF749
:1048D00027FC401B41F28831884202D9032077E649
:1048E00022E03748006A00F002000028EFD012E012
:1048F000FFF716FC054608E0FFF712FC401B41F2EB
:104900008831884201D9032062E62D48006A00F010
:1049100002000028F0D1012F05D12948C06920F0FC
:1049200080502749C86100BFE069C8B32448406887
:1049300000F00C00082860D0E069022848D100206F
:1049400020490866FFF7ECFB054606E0FFF7E8FBA9
:10495000401B022801D903203AE61948006800F0FC
:1049600000700028F2D1206AB0F5803F07D11448CA
:10497000406820F40030A168084311494860D4E938
:10498000080108430E49496821F4741108430C4991
:10499000486001200B490866FFF7C2FB054607E0A7
:1049A0003DE0FFF7BDFB401B022801D903200FE6C5
:1049B0000348006800F000700028F2D02FE00000EB
:1049C0000010024000004242800442420070004059
:1049D000002014490866FFF7A3FB054606E0FFF731
:1049E0009FFB401B022801D90320F1E50E48006817
:1049F00000F000700028F2D111E0E069012800D138
:104A0000E6E50948466806F48031206A814204D10F
:104A100006F47011606A814201D00120D8E50020BF
:104A2000D6E5000000004242001002407047704787
:104A300030B502460B4600BF92F83C00012801D178
:104A4000022030BD012082F83C0000BF022082F825
:104A50003D00106844681068816824F0700418688C
:104A6000044310684460144D1068A84213D0134DDD
:104A70001068A8420FD01068B0F1804F0BD0104DD5
:104A80001068A84207D00F4D1068A84203D00E4D01
:104A90001068A84205D121F08001586801431068D0
:104AA0008160012082F83D0000BF002082F83C00B8
:104AB00000BF00BFC5E70000002C014000340140EA
:104AC0000004004000080040000C004010B50446FF
:104AD0000CB9012010BD94F83D0028B9002084F8DD
:104AE0003C00204600F026F8022084F83D00211DFD
:104AF000206807F085FA012084F8460000BF84F89A
:104B00003E0001213F200155402001554120015523
:104B100000BF00BF012084F842004320015544201B
:104B200001554520015500BF012084F83D000020BB
:104B3000D0E7000008B5124A016891420DD100BFCC
:104B40001049896941F400610E4A916111468969F1
:104B500001F40061009100BF11E00B4A016891422D
:104B60000DD100BF0749C96941F00401054AD1616F
:104B70001146C96901F00401009100BF00BF08BDE2
:104B8000002C01400010024000080040014691F84E
:104B90003D00012801D001207047022081F83D002E
:104BA0000868C06840F001000B68D860164B0868C0
:104BB000984213D0154B086898420FD00868B0F19E
:104BC000804F0BD0124B0868984207D0114B0868F1
:104BD000984203D0104B086898420CD1086880684E
:104BE00000F00702062A0CD00868006840F00100B7
:104BF0000B68186005E00868006840F001000B6869
:104C000018600020C8E70000002C0140003401407B
:104C10000004004000080040000C00402DE9F04175
:104C200004460D4600BF94F83C00012802D1022042
:104C3000BDE8F081012084F83C0000BF022084F828
:104C40003D002068866826F0770626F47F462068B7
:104C500086602868502833D00CDC202850D004DC33
:104C600000284BD0102851D149E0302849D04028A5
:104C70004CD139E060282DD0702807D0B0F5805F86
:104C800003D0B0F5005F41D10DE040E0D5E902135B
:104C90006A68206807F002FA2068866846F077069E
:104CA0002068866033E0D5E902136A68206807F05F
:104CB000F5F92068806840F480402168886026E02B
:104CC000EA686968206807F0FDF95021206807F05C
:104CD000F0F91CE0EA686968206807F006FA6021CC
:104CE000206807F0E6F912E0EA686968206807F0D2
:104CF000E9F94021206807F0DCF908E000BF00BFB7
:104D000000BF2968206807F0D4F900E000BF00BFA9
:104D1000012084F83D0000BF002084F83C0000BF63
:104D200000BF85E7704710B5044620680069C0F3EE
:104D30004000D8B12068C068C0F34000B0B16FF047
:104D4000020021680861012020772068806900F056
:104D5000030018B12046FFF7E5FF05E0204600F00C
:104D6000ADF8204600F0ABF80020207720680069FD
:104D7000C0F38000D8B12068C068C0F38000B0B133
:104D80006FF00400216808610220207720688069A4
:104D900000F4407018B12046FFF7C4FF05E020463C
:104DA00000F08CF8204600F08AF800202077206878
:104DB0000069C0F3C000D8B12068C068C0F3C0006B
:104DC000B0B16FF0080021680861042020772068E6
:104DD000C06900F0030018B12046FFF7A3FF05E00B
:104DE000204600F06BF8204600F069F8002020779C
:104DF00020680069C0F30010D8B12068C068C0F313
:104E00000010B0B16FF01000216808610820207711
:104E10002068C06900F4407018B12046FFF782FF97
:104E200005E0204600F04AF8204600F048F800204F
:104E300020772068006900F0010058B12068C06840
:104E400000F0010030B16FF00100216808612046D8
:104E500000F036F820680069C0F3C01058B120682F
:104E6000C068C0F3C01030B16FF0800021680861E5
:104E70002046FFF7DBFD20680069C0F3801058B1C1
:104E80002068C068C0F3801030B16FF04000216826
:104E90000861204600F020F820680069C0F3401047
:104EA00058B12068C068C0F3401030B16FF02000E6
:104EB000216808612046FFF7BAFD10BD70477047B2
:104EC00010B5044603492068884201D1FFF72EF946
:104ED00010BD000000340140704770B50446002545
:104EE00020684069C0F3C01594F8390021280ED11C
:104EF0006DB12068406920F0800021684861206B16
:104F000010B1206BFEF70EFB204607F08AFA2068EE
:104F10004069C0F3801594F83A0022280ED16DB193
:104F20002068406920F0400021684861606B10B142
:104F3000606BFEF7F7FA204607F053FA002070BDC9
:104F4000704700002DE9F047044620680568206896
:104F5000C668206847694FF00008C14605F00F0891
:104F6000B8F1000F0AD105F0200038B106F020009A
:104F700020B1204607F05FFABDE8F087B8F1000FD6
:104F800071D007F0010018B906F4907000286AD0BB
:104F900005F0010030B106F4807018B1E06B40F00C
:104FA0000100E06305F0040030B107F0010018B122
:104FB000E06B40F00200E06305F0020030B107F062
:104FC000010018B1E06B40F00400E06305F0080058
:104FD00048B106F0200010B907F0010018B1E06BED
:104FE00040F00800E063E06B68B305F0200028B1F2
:104FF00006F0200010B1204607F01DFA2068406935
:10500000C0F38019E06B00F0080010B9B9F1000F8F
:1050100022D0204607F0E5F92068406900F0400002
:10502000B0B12068406920F0400021684861606BA1
:1050300050B11848616B4863606BFEF79FFA10B17E
:10504000606B416B88470CE02046FFF779FF08E072
:105050002046FFF775FF04E02046FFF771FF0020B0
:10506000E06389E7FFE705F0800030B106F08000DB
:1050700018B1204607F0AEFA7EE705F0400030B1E7
:1050800006F0400018B1204607F0BBF974E700BFF6
:1050900072E700002BC3000810B504460CB90120CC
:1050A00010BDA06900B100E000BF94F8390028B934
:1050B000002084F83800204600F028F8242084F8E6
:1050C00039002068C06820F400502168C86020467C
:1050D00007F002FA2068006920F490402168086116
:1050E0002068406920F02A00216848612068C06873
:1050F00040F400502168C8600020E063202084F85C
:10510000390084F83A000020CAE7000010B586B0E4
:10511000044600200290039004900590A249206864
:1051200088423BD100BFA148C06940F480109F492C
:10513000C8610846C06900F48010019000BF00BF3C
:1051400000BF0846806940F0100088610846806909
:1051500000F01000019000BF00BF00BF084680694A
:1051600040F0200088610846806900F0200001902E
:1051700000BF00BF88140290022003900320059016
:1051800002A98B48FEF714FE042002900020039031
:10519000049002A98748FEF70BFE02E186492068C9
:1051A000884263D100BF8148806940F480407F49D4
:1051B00088610846806900F48040019000BF00BF0C
:1051C00000BF0846806940F0040088610846806995
:1051D00000F00400019000BF00BF481502900220BB
:1051E00003900320059002A97448FEF7E1FD4FF4F7
:1051F0008060029000200390049002A96F48FEF79F
:10520000D7FD6F486F4908600020486000216D4855
:1052100081608021C16000210161416120218161A3
:105220000902C161FEF74AFC08B1FCF7D2F900BFE0
:1052300064486063446200BF614814386249086092
:10524000102048600021604881608021C1600021F9
:10525000016141618161C161FEF730FC08B1FCF779
:10526000B8F900BF5848206344629AE05749206863
:10527000884249D100BF4D48C06940F400304B49D5
:10528000C8610846C06900F40030019000BF00BF4B
:1052900000BF0846806940F00400886108468069C4
:1052A00000F00400019000BF00BF04200290022023
:1052B00003900320059002A94048FEF779FD0820DD
:1052C000029000200390049002A93C48FEF770FD74
:1052D0003B4814303E4908600020486000213C48AB
:1052E00081608021C16000210161416120218161D3
:1052F0000902C161FEF7E2FB08B1FCF76AF900BFE1
:105300003348606344624CE032492068884248D1A7
:1053100000BF2648C06940F480202449C86108467F
:10532000C06900F48020019000BF00BF00BF0846A4
:10533000806940F0080088610846806900F0080034
:10534000019000BF00BF08150290022003900320C7
:10535000059002A92048FEF72BFD4FF40060029053
:1053600000200390049002A91B48FEF721FD144879
:1053700028381A49086000204860002117488160D9
:105380008021C1600021016141618161C161FEF73D
:1053900095FB08B1FCF71DF900BF1048606344623B
:1053A00000BF06B010BD00000050004000100240D9
:1053B0000010014000140140003801400008014085
:1053C00058000240700C0020B40C00200044004043
:1053D000F80C002000480040000C01403C0D00206B
:1053E00077B581B00446154694F83A00202850D18C
:1053F000029800B115B9012004B070BD00BF94F847
:105400003800012801D10220F6E7012084F8380095
:1054100000BF0298A062A5850020E063222084F8E6
:105420003A001D48616B88621C48616BC8621C4869
:10543000616B08630020616B486302AE32682368C9
:10544000191D2B46606BFEF77FFB00BF002000900C
:1054500020680068009020684068009000BF00BF8E
:1054600000BF002084F8380000BF2068C06840F406
:1054700080702168C8602068406940F001002168A0
:1054800048612068406940F0400021684861002080
:10549000B2E70220B0E700008FC30008D5C30008C0
:1054A0003FC30008704770472DE9F84F04460E4689
:1054B000174699464FF0000A94F8390020285AD12F
:1054C00006B117B90120BDE8F88F00BF94F8380085
:1054D000012801D10220F6E7012084F8380000BF3E
:1054E0000020E063212084F83900FEF719FE82468F
:1054F000A784E784A068B0F5805F04D1206910B963
:105500000025B04602E035464FF0000800BF0020FD
:1055100084F8380000BF1BE053460022802120465B
:10552000CDF8009007F08BF808B10320CBE745B920
:10553000B8F80000C0F308002168486008F10208CC
:1055400003E02878216848606D1CE08C401EE084F0
:10555000E08C0028E0D15346002240212046CDF8BF
:10556000009007F06CF808B10320ACE7202084F825
:1055700039000020A7E70220A5E710B5034693F8FD
:105580003900202823D101B10AB9012010BD00BF84
:1055900093F83800012801D10220F7E7012083F8B1
:1055A000380000BF19629A84DA840020D863212071
:1055B00083F8390000BF002083F8380000BF186866
:1055C000C06840F080001C68E0600020DEE7022038
:1055D000DCE770472DE9F0410746374D00240026EF
:1055E0006888002864D1287D06285ED10120688063
:1055F000AA7F2046611CCCB230490A5406222046BC
:10560000611CCCB22D490A5400222046611CCCB248
:105610002A490A54A5222046611CCCB227490A54C3
:105620002046611CCCB225490A542046611CCCB2EC
:1056300022490A542046611CCCB220490A54204613
:10564000611CCCB21D490A542046611CCCB21B49D6
:105650000A542046611CCCB218490A542046611CE9
:10566000CCB216490A542046611CCCB213490A54E4
:105670002046611CCCB211490A542046611CCCB2B0
:105680000E490A540E210D4800F002FA0646321265
:105690002046611CCCB209490A542046611CCCB298
:1056A00006490E540648048004E00020BDE8F0815D
:1056B0000020FBE70120F9E7A2380020163800207F
:1056C000FA090020F0B58BB00646344F344D28213E
:1056D00001A8FAF7C6FD002400BF09E004F110009C
:1056E00005F10D01085C01A921F81400601CC4B289
:1056F000287EA042F2DC287D062804D10122294917
:1057000001A8FCF731F80122264901A8FCF716F898
:10571000BDF804003074BDF80400052802DABDF8B5
:105720000400F880287D062805D108221E490DF1C5
:105730000600FCF719F808221B490DF10600FBF7DB
:10574000FDFF002424E001A9601C31F81020103076
:1057500005F10D01085C824205D0287D062802D1A2
:1057600000200BB0F0BD01A9601C31F81000082822
:105770000CDA601C31F8101007F1240020F8141026
:1057800001A9601C11F8101010303154601CC4B213
:10579000287EA042D7DC0120E3E70000603700202C
:1057A000A238002030F0070840E007082DE9F0415A
:1057B0000746384D002400266888002866D1287DD9
:1057C000062860D101206880AA7F2046611CCCB2E7
:1057D00031490A5406222046611CCCB22E490A5493
:1057E00010222046611CCCB22B490A542020425D75
:1057F0002046611CCCB228490A54A5222046611CCF
:10580000CCB225490A542046611CCCB222490A5424
:105810002046611CCCB220490A542046611CCCB2FF
:105820001D490A542046611CCCB21B490A5420462B
:10583000611CCCB218490A542046611CCCB21649EE
:105840000A542046611CCCB213490A542046611CFC
:10585000CCB211490A542046611CCCB20E490A54FC
:105860000E210D4800F014F9064632122046611C44
:10587000CCB209490A542046611CCCB206490E54E8
:105880000648048004E00020BDE8F0810020FBE72A
:105890000120F9E7A238002016380020FA0900207C
:1058A0002DE9F0410746384D00240026688800287D
:1058B00066D1287D062860D101206880AA7F204615
:1058C000611CCCB231490A5406222046611CCCB27C
:1058D0002E490A5412222046611CCCB22B490A548C
:1058E0002020425D2046611CCCB228490A54A522E2
:1058F0002046611CCCB225490A542046611CCCB21A
:1059000022490A542046611CCCB220490A54204640
:10591000611CCCB21D490A542046611CCCB21B4903
:105920000A542046611CCCB218490A542046611C16
:10593000CCB216490A542046611CCCB213490A5411
:105940002046611CCCB211490A542046611CCCB2DD
:105950000E490A540E210D4800F09AF806463212FC
:105960002046611CCCB209490A542046611CCCB2C5
:1059700006490E540648048004E00020BDE8F0818A
:105980000020FBE70120F9E7A238002016380020AC
:10599000FA0900202DE9F0410746394D0024002680
:1059A0006888002867D1287D062861D10120688099
:1059B000AA7F2046611CCCB232490A5406222046F6
:1059C000611CCCB22F490A5414222046611CCCB26F
:1059D0002C490A54EA7F2046611CCCB229490A545A
:1059E0002020425D2046611CCCB226490A54A522E3
:1059F0002046611CCCB223490A542046611CCCB21B
:105A000020490A542046611CCCB21E490A54204643
:105A1000611CCCB21B490A542046611CCCB2194906
:105A20000A542046611CCCB216490A542046611C17
:105A3000CCB214490A542046611CCCB211490A5414
:105A40002046611CCCB20F490A540E210D4800F0CB
:105A50001FF8064632122046611CCCB209490A548E
:105A60002046611CCCB207490E540748048004E06C
:105A70000020BDE8F0810020FBE70120F9E70000ED
:105A8000A238002016380020FA09002000BFFEE7E7
:105A900070B502460B46FF24FF2509E012F8010B02
:105AA00080EA04010748405C80EA05040648455C3A
:105AB000181EA3F10106B3B2F0D105EB042080B2A9
:105AC00070BD000094FD000894FE000804E0002270
:105AD00000F8012B4A1E91B20029F8DC7047000043
:105AE00070B58AB005463D4C3D4E28216846FAF710
:105AF000B8FBA17F607F41EA0020ADF800002020C4
:105B0000015DE07F41EA0020ADF802002220015D46
:105B10002120005D41EA0020ADF804002420015D51
:105B20002320005D41EA0020ADF80600207D062814
:105B300004D104222B496846FBF716FE04222949AA
:105B40006846FBF7FBFDBDF8000000122874BDF8A5
:105B500000006874BDF802000012A874BDF80200CD
:105B6000E874BDF8040000122875BDF804006875DB
:105B7000BDF806000012A875BDF80800E875297C7C
:105B8000607F814228D1697CA07F814224D1207D21
:105B9000062821D1607F1449C870A07F8870E07FFB
:105BA00048702020005D087008460168F16400BF5D
:105BB0002120005D0C49C8702220005D88702320E0
:105BC000005D48702420005D087008460168716718
:105BD00000BF01200AB070BD0020FBE7A238002002
:105BE000583F002000C007085803002070B58AB055
:105BF00005461D4E1D4C28216846FAF732FBA17F51
:105C0000607F41EA0020ADF80000207D062804D125
:105C1000012217496846FBF7A7FD0122144968468F
:105C2000FBF78CFDBDF8000000122874BDF80000E1
:105C30006874BDF800004FF6FF71884203D0BDF8CC
:105C40000000A6F86400297C607F814209D1697C4C
:105C5000A07F814205D1207D062802D101200AB013
:105C600070BD0020FBE7000060370020A238002054
:105C700040F007082DE9F0410646377896F8018094
:105C80003846FAF7CFFA3038C4B2092C01DDE01FEC
:105C9000C4B24046FAF7C6FA3038C5B2092D01DD64
:105CA000E81FC5B205EB0410C0B2BDE8F0810000EA
:105CB00010B50548054908600846FDF765FB08B1C1
:105CC000FBF787FC10BD000000300240FC01002003
:105CD0001CB50020009001900A480B490860084656
:105CE000FDF7B4FB08B1FBF774FC3C2000900020EA
:105CF0000190102269460448FDF76EFB08B1FBF7DE
:105D000068FC1CBD00740040880A002008B500BF74
:105D10001548406940F00100134948610846406950
:105D200000F00100009000BF00BF00BF08464069BE
:105D300040F0020048610846406900F0020000900F
:105D400000BF00BF002205210E20FEF793FA0E20AF
:105D5000FEF780FA002205213B20FEF78BFA3B205C
:105D6000FEF778FA08BD00000010024000B585B0CB
:105D70000020019002900390049000BF4448806985
:105D800040F02000424988610846806900F0200008
:105D9000009000BF00BF00BF0846806940F00400CB
:105DA00088610846806900F00400009000BF00BFD1
:105DB00000BF0846806940F0080088610846806995
:105DC00000F00800009000BF00BF00BF08468069D7
:105DD00040F0100088610846806900F010000090D3
:105DE00000BF00BF002213212A48FEF793F90022CA
:105DF0004FF440512848FEF78DF900224FF480619E
:105E00002648FEF787F91320019001200290002018
:105E100003900220049001A91E48FDF7C9FF4FF42A
:105E20004050019001200290002003900220049035
:105E300001A91948FDF7BCFF4FF440400190002034
:105E40000290039001A91448FDF7B2FF4FF470705F
:105E5000019000200290039001A91048FDF7A8FFCF
:105E60004FF41060019000200290039001A90948AE
:105E7000FDF79EFF4FF48060019000200290039098
:105E80000220049001A90548FDF792FF05B000BD6E
:105E90000010024000080140000C014000100140C9
:105EA00010B5002205212720FEF7E4F92720FEF790
:105EB000D1F9002205212520FEF7DCF92520FEF787
:105EC000C9F9002205212620FEF7D4F92620FEF785
:105ED000C1F9002205211E20FEF7CCF91E20FEF795
:105EE000B9F9002205211920FEF7C4F91920FEF79F
:105EF000B1F9002205211020FEF7BCF91020FEF7B1
:105F0000A9F9002205210F20FEF7B4F90F20FEF7B2
:105F1000A1F9002205210D20FEF7ACF90D20FEF7B6
:105F200099F910BD00B587B000200390049005904A
:105F300006900190029016481649086000204860BB
:105F40000021144881604FF6FF71C1604FF4007169
:105F50000161002141618161FEF7B8FD08B1FBF7E5
:105F600038FB4FF48050039003A90A48FEF756FE11
:105F700008B1FBF72EFB00200190029001A9054813
:105F8000FEF756FD08B1FBF724FB07B000BD00008B
:105F9000002C0140E00A002000B587B000200390EB
:105FA00004900590069001900290144814490860EE
:105FB000002048600021124881604FF6FF71C160E7
:105FC000002101618161FEF781FD08B1FBF701FB52
:105FD0004FF48050039003A90948FEF71FFE08B153
:105FE000FBF7F7FA00200190029001A90448FEF7A0
:105FF0001FFD08B1FBF7EDFA07B000BD0008004037
:10600000280B002010B50B480B4908604FF4E13015
:106010004860002108488160C16001610C21416134
:1060200000218161C161FFF737F808B1FBF7D1FAB0
:1060300010BD000000500040700B002010B5124849
:10604000124908604FF41650486000210F488160E3
:10605000C16001610C21416100218161C161FFF7D3
:106060001BF808B1FBF7B5FA08480068C06840F0B3
:10607000100006490968C8604FF48072044903485B
:10608000FFF7AEF910BD000000380140B00B002052
:106090000024002010B51248124908604FF4164041
:1060A000486000210F488160C16001610C2141619D
:1060B00000218161C161FEF7EFFF08B1FBF789FAAA
:1060C00008480068C06840F0100006490968C860C8
:1060D0004FF4807204490348FFF782F910BD0000B5
:1060E00000440040F00B00200027002010B51248AB
:1060F000124908604FF41650486000210F48816033
:10610000C16001610C21416100218161C161FEF723
:10611000C3FF08B1FBF75DFA08480068C06840F0AB
:10612000100006490968C8604FF4807204490348AA
:10613000FFF756F910BD000000480040300C002069
:10614000002A002000BFFEE700BFFEE708B50849AF
:106150000968C9084FF47A72B1FBF2F1414300912A
:1061600000BF00BF00994A1E00920029F9D108BD66
:10617000000A0020F0B58BB03D4D3E4F3E4E00244E
:1061800008223E4901A8FBF7D9FA00BF0FE001A899
:1061900030F814004FF6FF71884206D001A830F89D
:1061A000141005F1340020F81410601CC4B22888C3
:1061B000A042ECDC0122324901A8FBF7BFFABDF88E
:1061C00004004FF6FF71884202D0BDF80400288118
:1061D00001222B49383101A8FBF7B0FABDF80400C1
:1061E0004FF6FF71884212D000240BE04FF461702B
:1061F000C4EBC40101EB810107EB4101A1F84200AE
:10620000601CC4B22888401CA042EFDC11E00024CE
:106210000BE0BDF80400C4EBC40101EB810107EB06
:106220004101A1F84200601CC4B22888401CA04271
:10623000EFDC00240EE000203080401EF080B080B3
:10624000000C7080402106F10800FFF73FFC601C45
:10625000C4B24836082CEEDB002404E002200949D1
:106260000870601CC4B22888A042F7DC0BB0F0BDF7
:106270006037002000330020802E002020E0070837
:1062800020F007085003002070B586B004461A4E6F
:106290001A4D142101A8F9F7E4FFA97F687F41EAAC
:1062A0000020ADF80400287D062804D101221449FD
:1062B00001A8FBF759FA0020ADF8040001221049AB
:1062C00001A8FBF73BFABDF80400A6F84200BDF8B0
:1062D000040000122074BDF804006074217C687F03
:1062E000814206D1617CA87F814202D1012006B0A3
:1062F00070BD0020FBE7000000330020A238002022
:1063000058F00708F0B58BB00646344F344D2821BD
:1063100001A8F9F7A6FF002400BF09E004F110006E
:1063200005F10D01085C01A921F81400601CC4B23C
:10633000287EA042F2DC287D062804D101222949CA
:1063400001A8FBF711FA0122264901A8FBF7F6F98B
:10635000BDF804003074BDF80400052802DABDF869
:1063600004003881287D062805D108221E490DF138
:106370000600FBF7F9F908221B490DF10600FBF7AF
:10638000DDF9002424E001A9601C31F81020103050
:1063900005F10D01085C824205D0287D062802D156
:1063A00000200BB0F0BD01A9601C31F810000828D6
:1063B0000CDA601C31F8101007F1340020F81410CA
:1063C00001A9601C11F8101010303154601CC4B2C7
:1063D000287EA042D7DC0120E3E7000060370020E0
:1063E000A238002020F0070820E007082DE9FC4132
:1063F00080462F4D2F4F0024002600200090019052
:106400002888002850D1287D06284AD1AA7F204616
:10641000611CCCB228490A5406222046611CCCB229
:1064200025490A5400222046611CCCB222490A5454
:1064300010222046611CCCB21F490A54002220467B
:10644000611CCCB21C490A54FF222046611CCCB20C
:1064500019490A54A87F8DF8000006208DF8010024
:1064600000208DF8020010208DF8030000208DF828
:106470000400FF208DF8050006216846FFF708FBA1
:10648000064632122046611CCCB20B490A54204603
:10649000611CCCB208490E540848048001202880B1
:1064A00004E00020BDE8FC810020FBE70120F9E7C3
:1064B000A238002060370020D0370020FA090020E1
:1064C0002DE9F04704468F4E8F4FDFF84092DFF8FA
:1064D0004082002599F81E50012D01DB082D02DDB8
:1064E0000020BDE8F0872020E07299F81E0060745B
:1064F00007EBC510B0F87A00C0B14720A0747F2028
:10650000E074FF202075002060754720A0757F2073
:10651000E075FF202076002060764720A0767F205F
:10652000E076FF2020770020607741E007EBC51080
:10653000B0F90000000EA07407EBC510B0F9000020
:10654000000CE07407EBC5100088000A207507EB0B
:10655000C5100078607507EBC510B0F92800000E73
:10656000A07507EBC510B0F92800000CE07507EB2B
:10657000C510008D000A207607EBC51090F82800A2
:10658000607607EBC510B0F95000000EA07607EB5F
:10659000C510B0F95000000CE07607EBC510B0F85C
:1065A0005000000A207707EBC51090F85000607784
:1065B000B6F87A00D0B1472004F81E0F7F20607033
:1065C000FF20A0700020E070472020717F206071C4
:1065D000FF20A0710020E071472020727F206072B0
:1065E000FF20A0720020E0721E3C2BE0B6F90000F4
:1065F000000E04F81E0FB6F90000000C6070308821
:10660000000AA0703078E070B6F92800000E207102
:10661000B6F92800000C6071308D000AA07196F860
:106620002800E071B6F95000000E2072B6F9500053
:10663000000C6072B6F85000000AA07296F8500084
:10664000E0721E3C05EB850008EBC000C08B90B1EA
:10665000472004F82A0F7F206070FF20A0700020E0
:10666000E070472020717F206071FF20A071002022
:10667000E0712A3C43E005EB850158F83100F9F759
:10668000D1FE000E04F82A0F05EB850158F8310001
:10669000F9F7C8FE000C607005EB850158F8310071
:1066A000F9F7C0FE000AA07005EB850158F831002B
:1066B000F9F7B8FEE07005EB850108EBC1018869C8
:1066C000F9F7B0FE000E207105EB850108EBC10162
:1066D0008869F9F7A7FE000C607105EB850108EBEE
:1066E000C1018869F9F79EFE000AA07105EB8501DA
:1066F00008EBC1018869F9F795FEE0712A3C012099
:10670000EFE60000D84100205C420020A2380020C3
:10671000583F00202DE9F04F8BB00446DFF8E4A38A
:10672000F94EFA480A90DFF8E883DFF8E8B3FA4850
:106730000990FA480890FA480790FA48069001250F
:10674000002700200490814603900290012D01DB78
:10675000082D03DD00200BB0BDE8F08F002720E0FE
:106760000BF1240010F8171004980844C0B20490EC
:106770000BF1140010F81700484400F0FF090BF16A
:10678000340010F8171003980844C0B203900BF1BE
:10679000440010F8171002980844C0B20290781C08
:1067A000C7B2681EB842DBDC002705E0002107F114
:1067B00010002154781CC7B2042FF7DB05EBC5008D
:1067C00000EB45110A9800EB4100807804F8140FA3
:1067D00000206070A070E07005EBC50000EB451173
:1067E0000A9800EB410090F8400020710020607191
:1067F000A071E07105EB850000EB851018F8100022
:10680000207200206072A072E07205EB850000EB40
:10681000851008EB400090F828002073002060737A
:10682000A073E07305EB850000EB851018F81000ED
:10683000207400206074A074E07405EB850000EB08
:10684000851008EB400090F8280020750020607546
:10685000A075E075143C0498401C00EBC00101EBEE
:1068600040110A9800EB4100B0F84C0018B1032029
:1068700084F82C0006E00499491CC8B2FCF730FCEF
:1068800084F82C0009F1010000EB001000EB40013E
:10689000079800EB4100B0F85E0018B1032084F8BF
:1068A00030000CE009F1010000EB001000EB4001AA
:1068B000079800EB410090F8580084F830000398E6
:1068C000401CC0EBC00000EB8001089800EB4100C9
:1068D000408F28B1032084F8340084F8380019E090
:1068E0000398401CC0EBC00000EB8001089800EB4F
:1068F000410090F8340084F834000398401CC0EB49
:10690000C00000EB8001089800EB410090F83600D1
:1069100084F8380009F1010000EB001000EB4001A1
:10692000079800EB4100B0F85E0018B1032084F82E
:106930003C000CE009F1010000EB001000EB40010D
:10694000079800EB410090F85A0084F83C000020C2
:1069500004F82D0F6070A07020716071A07120721A
:106960006072A07220736073A07320746074A0744E
:1069700005EB850000EB851008EB400090F828003F
:10698000E074002020756075A07505EB850000EBB4
:10699000851008EB400090F82800E0750020207674
:1069A0006076A0762D3C002705E0002107F1480025
:1069B0002154781CC7B2202FF7DB05EB850006EBCE
:1069C000C000C08B38B1002004F8680F6070A07060
:1069D000E070683C13E005EB850006EBC000406802
:1069E00005909DF8140004F8680F9DF8150060707C
:1069F0009DF81600A0709DF81700E070683C05EB4C
:106A0000850006EBC000C08B38B1002004F86C0F85
:106A10006070A070E0706C3C18E00AEBC511B1F931
:106A20002A00F9F7F1FC40490190F9F77DFC059047
:106A30009DF8140004F86C0F9DF8150060709DF827
:106A40001600A0709DF81700E0706C3C05EB850007
:106A500006EBC000C08B38B1002004F8700F6070E6
:106A6000A070E070703C18E00AEBC511B1F90200AB
:106A7000F9F7CAFC2C490190F9F756FC05909DF8EE
:106A8000140004F8700F9DF8150060709DF8160052
:106A9000A0709DF81700E070703C05EB850006EBD8
:106AA000C000C08B38B1002004F8740F6070A07073
:106AB000E070743C18E00AEBC511B1F92A00F9F74F
:106AC000A3FC19490190F9F72FFC05909DF81400DB
:106AD00004F8740F9DF8150060709DF81600A07002
:106AE0009DF81700E070743C05EB850006EBC000D4
:106AF000C08BD8B1002004F8780F6070A070E070EF
:106B0000783C2CE05C420020583F00205C4A00208A
:106B10007C4F002060370020A23800200033002086
:106B2000F63800201C580020CDCCCC3D0AEBC51116
:106B3000B1F95200F9F768FC64490190F9F7F4FBE8
:106B400005909DF8140004F8780F9DF8150060700A
:106B50009DF81600A0709DF81700E070783C05EBDA
:106B6000850006EBC000C08B50B1762004F87C0F86
:106B70007F206070FF20A0700020E0707C3C14E05B
:106B8000284600EB800006EBC000806905909DF868
:106B9000140004F87C0F9DF8150060709DF8160035
:106BA000A0709DF81700E0707C3C05EB850006EBBB
:106BB000C000C08B38B1002004F8800F6070A07056
:106BC000E070803C0CE005EB850006EBC0008069BE
:106BD0000590002004F8800F6070A070E070803C89
:106BE00005EB850006EBC000C08B38B1002004F82F
:106BF000840F6070A070E070843C0CE005EB8500B1
:106C000006EBC00080690590002004F8840F6070D6
:106C1000A070E070843C05EB850006EBC000C08BE3
:106C200038B1002004F8880F6070A070E070883CD4
:106C30000CE005EB850006EBC000806905900020A4
:106C400004F8880F6070A070E070883C05EB850048
:106C500006EBC000C08B38B1002004F88C0F6070C8
:106C6000A070E0708C3C13E005EB850006EBC000E3
:106C7000806905909DF8140004F88C0F9DF81500AC
:106C800060709DF81600A0709DF81700E0708C3CB5
:106C900005EB850006EBC000C08B38B1002004F87E
:106CA000900F6070A070E070903C0CE005EB8500E8
:106CB00006EBC00080690590002004F8900F60701A
:106CC000A070E070903C012045E50000CDCCCC3DAB
:106CD00078B50246FE4B0121002400BF05E0A52542
:106CE00004F110001554601CC4B2082CF7DD002418
:106CF00012E00020182505EB84055055192505EBF9
:106D0000840550551A2505EB840550551B2505EBC8
:106D100084055055601CC4B2082CEADD0121FDE356
:106D200001EB810003EBC000C08B28B30025481E97
:106D300000EB400606EBC000382606EB8000155439
:106D4000481E00EB400606EBC000392606EB80002B
:106D50001554481E00EB400606EBC0003A2606EB31
:106D600080001554481E00EB400606EBC0003B2691
:106D700006EB8000155430E001EB810053F8300041
:106D800000909DF80050481E00EB400606EBC00046
:106D9000382606EB800015549DF80150481E00EB84
:106DA000400606EBC000392606EB800015549DF81E
:106DB0000250481E00EB400606EBC0003A2606EBE8
:106DC000800015549DF80350481E00EB400606EB6A
:106DD000C0003B2606EB8000155401EB810003EB5D
:106DE000C000C08B28B30025481E00EB400606EB10
:106DF000C0003C2606EB80001554481E00EB400600
:106E000006EBC0003D2606EB80001554481E00EB43
:106E1000400606EBC0003E2606EB80001554481ED7
:106E200000EB400606EBC0003F2606EB8000155441
:106E300031E001EB810003EBC000806800909DF819
:106E40000050481E00EB400606EBC0003C2606EB57
:106E5000800015549DF80150481E00EB400606EBDB
:106E6000C0003D2606EB800015549DF80250481ED8
:106E700000EB400606EBC0003E2606EB80001554F2
:106E80009DF80350481E00EB400606EBC0003F266D
:106E900006EB8000155401EB810003EBC000C08BB2
:106EA00028B30025481E00EB400606EBC000402634
:106EB00006EB80001554481E00EB400606EBC000B0
:106EC000412606EB80001554481E00EB400606EBF9
:106ED000C000422606EB80001554481E00EB400619
:106EE00006EBC000432606EB8000155431E001EBB1
:106EF000810003EBC000C06800909DF80050481E60
:106F000000EB400606EBC000402606EB800015545F
:106F10009DF80150481E00EB400606EBC0004126DC
:106F200006EB800015549DF80250481E00EB400609
:106F300006EBC000422606EB800015549DF8035076
:106F4000481E00EB400606EBC000432606EB80001F
:106F5000155401EB810003EBC000C08B28B3002562
:106F6000481E00EB400606EBC000442606EB8000FE
:106F70001554481E00EB400606EBC000452606EB04
:106F800080001554481E00EB400606EBC000462664
:106F900006EB80001554481E00EB400606EBC000CF
:106FA000472606EB8000155431E001EB810003EB2E
:106FB000C000006900909DF80050481E00EB40069C
:106FC00006EBC000442606EB800015549DF80150E6
:106FD000481E00EB400606EBC000452606EB80008D
:106FE00015549DF80250481E00EB400606EBC00009
:106FF000462606EB800015549DF80350481E00EB12
:10700000400606EBC000472606EB8000155401EB56
:10701000810003EBC000C08B28B30025481E00EBA5
:10702000400606EBC000482606EB80001554481EBB
:1070300000EB400606EBC000492606EB8000155425
:10704000481E00EB400606EBC0004A2606EB800017
:107050001554481E00EB400606EBC0004B2606EB1D
:107060008000155431E001EB810003EBC000406962
:1070700000909DF80050481E00EB400606EBC00053
:10708000482606EB800015549DF80150481E00EB81
:10709000400606EBC000492606EB800015549DF81B
:1070A0000250481E00EB400606EBC0004A2606EBE5
:1070B000800015549DF80350481E00EB400606EB77
:1070C000C0004B2606EB8000155401EB810001E067
:1070D000583F002003EBC000C08B40B37625481E0C
:1070E00000EB400606EBC0004C2606EB8000155472
:1070F0007F25481E00EB400606EBC0004D2606EB40
:1071000080001554FF25481E00EB400606EBC0002A
:107110004E2606EB800015540025481E00EB400665
:1071200006EBC0004F2606EB8000155431E001EB62
:10713000810003EBC000806900909DF80050481E5C
:1071400000EB400606EBC0004C2606EB8000155411
:107150009DF80150481E00EB400606EBC0004D268E
:1071600006EB800015549DF80250481E00EB4006C7
:1071700006EBC0004E2606EB800015549DF8035028
:10718000481E00EB400606EBC0004F2606EB8000D1
:10719000155401EB810003EBC000C08B40B3762592
:1071A000481E00EB400606EBC000502606EB8000B0
:1071B00015547F25481E00EB400606EBC000512603
:1071C00006EB80001554FF25481E00EB400606EB39
:1071D000C000522606EB800015540025481E00EB27
:1071E000400606EBC000532606EB8000155431E044
:1071F00001EB810003EBC000806900909DF8005016
:10720000481E00EB400606EBC000502606EB80004F
:1072100015549DF80150481E00EB400606EBC000D7
:10722000512606EB800015549DF80250481E00EBD5
:10723000400606EBC000522606EB800015549DF870
:107240000350481E00EB400606EBC000532606EB39
:107250008000155401EB810003EBC000C08B40B3EC
:107260007625481E00EB400606EBC000542606EBD0
:10727000800015547F25481E00EB400606EBC00039
:10728000552606EB80001554FF25481E00EB4006EE
:1072900006EBC000562606EB800015540025481E5C
:1072A00000EB400606EBC000572606EB80001554A5
:1072B00031E001EB810003EBC000806900909DF894
:1072C0000050481E00EB400606EBC000542606EBBB
:1072D000800015549DF80150481E00EB400606EB57
:1072E000C000552606EB800015549DF80250481E3C
:1072F00000EB400606EBC000562606EB8000155456
:107300009DF80350481E00EB400606EBC0005726D0
:1073100006EB8000155401EB810003EBC000C08B2D
:1073200040B37625481E00EB400606EBC000582609
:1073300006EB800015547F25481E00EB400606EB47
:10734000C000592606EB80001554FF25481E00EBAF
:10735000400606EBC0005A2606EB800015540025B7
:10736000481E00EB400606EBC0005B2606EB8000E3
:10737000155431E001EB810003EBC00080690090FF
:107380009DF80050481E00EB400606EBC000582652
:1073900006EB800015549DF80150481E00EB400696
:1073A00006EBC000592606EB800015549DF80250EC
:1073B000481E00EB400606EBC0005A2606EB800094
:1073C00015549DF80350481E00EB400606EBC00024
:1073D0005B2606EB8000155401EB810003EBC00037
:1073E000C08B40B37625481E00EB400606EBC0007C
:1073F0005C2606EB800015547F25481E00EB4006F6
:1074000006EBC0005D2606EB80001554FF25481EE4
:1074100000EB400606EBC0005E2606EB800015542C
:107420000025481E00EB400606EBC0005F2606EB79
:107430008000155431E001EB810003EBC00080694E
:1074400000909DF80050481E00EB400606EBC0007F
:107450005C2606EB800015549DF80150481E00EB99
:10746000400606EBC0005D2606EB800015549DF833
:107470000250481E00EB400606EBC0005E2606EBFD
:10748000800015549DF80350481E00EB400606EBA3
:10749000C0005F2606EB8000155401EB810003EB72
:1074A000C000C08B40B37625481E00EB400606EBBB
:1074B000C000602606EB800015547F25481E00EBB7
:1074C000400606EBC000612606EB80001554FF2540
:1074D000481E00EB400606EBC000622606EB80006B
:1074E00015540025481E00EB400606EBC00063263D
:1074F00006EB8000155433E001EB810003EBC00084
:10750000806900909DF80050481E00EB400606EB95
:10751000C000602606EB8000155400E022E09DF8D4
:107520000150481E00EB400606EBC000612606EB4A
:10753000800015549DF80250481E00EB400606EBF3
:10754000C000622606EB800015549DF80350481ECB
:1075500000EB400606EBC000632606EB80001554E6
:10756000481CC1B204297FF7DBAB012078BD0000C5
:107570002DE9F04F8BB00446DFF8E4A3F94EFA484A
:107580000A90DFF8E883DFF8E8B3FA480990FA4890
:107590000890FA480790FA48069002250027002034
:1075A0000490814603900290012D01DB082D03DD3C
:1075B00000200BB0BDE8F08F002720E00BF1240085
:1075C00010F8171004980844C0B204900BF114008E
:1075D00010F81700484400F0FF090BF1340010F8D0
:1075E000171003980844C0B203900BF1440010F840
:1075F000171002980844C0B20290781CC7B2681EE7
:10760000B842DBDC002705E0002107F1100021541F
:10761000781CC7B2042FF7DB05EBC50000EB451162
:107620000A9800EB4100807804F8140F0020607085
:10763000A070E07005EBC50000EB45110A9800EB67
:10764000410090F84000207100206071A071E0714D
:1076500005EB850000EB851018F810002072002063
:107660006072A072E07205EB850000EB851008EBFC
:10767000400090F82800207300206073A073E0732E
:1076800005EB850000EB851018F810002074002031
:107690006074A074E07405EB850000EB851008EBC6
:1076A000400090F82800207500206075A075E075F6
:1076B000143C0498401C00EBC00101EB40110A98F7
:1076C00000EB4100B0F84C0018B1032084F82C0006
:1076D00006E00499491CC8B2FBF702FD84F82C00AF
:1076E00009F1010000EB001000EB4001079800EBEE
:1076F0004100B0F85E0018B1032084F830000CE0BF
:1077000009F1010000EB001000EB4001079800EBCD
:10771000410090F8580084F830000398401CC0EBFA
:10772000C00000EB8001089800EB4100408F28B1B9
:10773000032084F8340084F8380019E00398401CD2
:10774000C0EBC00000EB8001089800EB410090F80E
:10775000340084F834000398401CC0EBC00000EBF8
:107760008001089800EB410090F8360084F838005A
:1077700009F1010000EB001000EB4001079800EB5D
:107780004100B0F85E0018B1032084F83C000CE022
:1077900009F1010000EB001000EB4001079800EB3D
:1077A000410090F85A0084F83C00002004F82D0FA6
:1077B0006070A07020716071A07120726072A07200
:1077C00020736073A07320746074A07405EB85004F
:1077D00000EB851008EB400090F82800E0740020D2
:1077E00020756075A07505EB850000EB851008EB32
:1077F000400090F82800E075002020766076A076A2
:107800002D3C002705E0002107F148002154781C99
:10781000C7B2202FF7DB05EB850006EBC000C08B5D
:1078200038B1002004F8680F6070A070E070683C08
:1078300013E005EB850006EBC000406805909DF85D
:10784000140004F8680F9DF8150060709DF816008C
:10785000A0709DF81700E070683C05EB850006EB12
:10786000C000C08B38B1002004F86C0F6070A070AD
:10787000E0706C3C18E00AEBC511B1F92A00F8F78A
:10788000C3FD40490190F8F74FFD05909DF81400A5
:1078900004F86C0F9DF8150060709DF81600A0703C
:1078A0009DF81700E0706C3C05EB850006EBC0000E
:1078B000C08B38B1002004F8700F6070A070E070C9
:1078C000703C18E00AEBC511B1F90200F8F79CFD15
:1078D0002C490190F8F728FD05909DF8140004F854
:1078E000700F9DF8150060709DF81600A0709DF84F
:1078F0001700E070703C05EB850006EBC000C08B04
:1079000038B1002004F8740F6070A070E070743C0F
:1079100018E00AEBC511B1F92A00F8F775FD19490D
:107920000190F8F701FD05909DF8140004F8740F1C
:107930009DF8150060709DF81600A0709DF8170066
:10794000E070743C05EB850006EBC000C08BD8B13D
:10795000002004F8780F6070A070E070783C2CE094
:107960005C420020583F00205C4A00207C4F0020F1
:1079700060370020A238002000330020F6380020B5
:107980001C580020CDCCCC3D0AEBC511B1F95200FA
:10799000F8F73AFD60490190F8F7C6FC05909DF8AC
:1079A000140004F8780F9DF8150060709DF816001B
:1079B000A0709DF81700E070783C05EB850006EBA1
:1079C000C000C08B50B1762004F87C0F7F2060701F
:1079D000FF20A0700020E0707C3C14E0284600EB03
:1079E000800006EBC000806905909DF8140004F843
:1079F0007C0F9DF8150060709DF81600A0709DF832
:107A00001700E0707C3C05EB850006EBC000C08BE6
:107A100038B1002004F8800F6070A070E070803CE6
:107A20000CE005EB850006EBC000806905900020A6
:107A300004F8800F6070A070E070803C05EB85005A
:107A400006EBC000C08B38B1002004F8840F6070D2
:107A5000A070E070843C0CE005EB850006EBC000F4
:107A600080690590002004F8840F6070A070E070B9
:107A7000843C05EB850006EBC000C08B38B10020CC
:107A800004F8880F6070A070E070883C0CE005EB93
:107A9000850006EBC00080690590002004F8880F7F
:107AA0006070A070E070883C05EB850006EBC000BC
:107AB000C08B38B1002004F88C0F6070A070E070AB
:107AC0008C3C0CE005EB850006EBC000806905905E
:107AD000002004F88C0F6070A070E0708C3C05EB07
:107AE000850006EBC000C08B38B1002004F8900F71
:107AF0006070A070E070903C0CE005EB850006EB38
:107B0000C00080690590002004F8900F6070A0709C
:107B1000E070903C01204CE5CDCCCC3DF8B5014661
:107B2000FD4BFE4EFE4C0322002500BF05E0002762
:107B300005F110000F54681CC5B2042DF7DB02EBF1
:107B4000C20000EB421006EB4000807801F8140FF1
:107B5000002048708870C87002EBC20000EB421031
:107B600006EB400090F840000871002048718871D1
:107B7000C87102EB820000EB821014F8100008724A
:107B8000002048728872C87202EB820000EB8210FB
:107B900004EB400090F828000873002048738873B5
:107BA000C87302EB820000EB821014F81000087416
:107BB000002048748874C87402EB820000EB8210C5
:107BC00004EB400090F8280008750020487588757F
:107BD000C87502EB820000EB821014F810000876E2
:107BE000002048768876C87602EB820000EB82108F
:107BF00004EB400090F82800087700204877887749
:107C0000C87702EB820000EB821014F8100081F8B4
:107C10002000002081F8210081F8220081F8230053
:107C200002EB820000EB821004EB400090F8280089
:107C300081F82400002081F8250081F8260081F8D1
:107C4000270002EB820000EB821004EB400090F86A
:107C5000280081F82800002081F8290081F82A00F6
:107C600081F82B0002EB820000EB821004EB400055
:107C700090F8280081F82C00002081F82D0081F870
:107C80002E0081F82F0002EB820000EB821004EB43
:107C9000400090F8280081F83000002081F8310081
:107CA00081F8320081F833001439002505E00027FF
:107CB00005F148000F54681CC5B2202DF7DB02EB1C
:107CC000820003EBC000C08B38B1002001F8680FC0
:107CD00048708870C870683912E002EB820053F86F
:107CE000300000909DF8000001F8680F9DF8010039
:107CF00048709DF8020088709DF80300C8706839CC
:107D000002EB820003EBC000C08B38B1002001F809
:107D10006C0F48708870C8706C3913E002EB8200F9
:107D200003EBC000806800909DF8000001F86C0F24
:107D30009DF8010048709DF8020088709DF80300CE
:107D4000C8706C3902EB820003EBC000C08B38B105
:107D5000002001F8700F48708870C870703913E007
:107D600002EB820003EBC000C06800909DF80000A9
:107D700001F8700F9DF8010048709DF802008870AE
:107D80009DF80300C870703902EB820003EBC0005D
:107D9000C08B38B1002001F8740F48708870C8702B
:107DA000743913E002EB820003EBC000006900901D
:107DB0009DF8000001F8740F9DF8010048709DF8CF
:107DC000020088709DF80300C870743902EB8200CD
:107DD00003EBC000C08B38B1002001F8780F487069
:107DE0008870C870783913E002EB820003EBC000A2
:107DF000406900909DF8000001F8780F9DF801009F
:107E000048709DF8020088709DF80300C8707839AA
:107E100002EB820003EBC000C08B50B1762001F86A
:107E20007C0F7F204870FF2088700020C8707C394C
:107E300013E002EB820003EBC000806900909DF824
:107E4000000001F87C0F9DF8010048709DF80200C9
:107E500088709DF80300C8707C3902EB820003EB48
:107E6000C000C08B38B1002001F8800F48708870C6
:107E7000C87080390CE002EB820003EBC00080691F
:107E80000090002001F8800F48708870C870803919
:107E900002EB820003EBC000C08B38B1002001F878
:107EA000840F48708870C87084390CE002EB82003F
:107EB00003EBC00080690090002001F8840F487037
:107EC0008870C870843902EB820003EBC000C08B5D
:107ED00038B1002001F8880F48708870C870883960
:107EE0000CE002EB820003EBC000806900900020F0
:107EF00001F8880F48708870C870883902EB8200DA
:107F000003EBC000C08B68B1002001F88C0F4870F3
:107F10008870C8708C3912E0583F00205C4A0020FD
:107F20007C4F002002EB820003EBC00080690090D0
:107F3000002001F88C0F48708870C8708C3902EBF3
:107F4000820003EBC000C08B38B1002001F8900F15
:107F500048708870C87090390CE002EB820003EB27
:107F6000C00080690090002001F8900F4870887070
:107F7000C87090390120F8BDF8B50146FD4BFE4EA2
:107F8000FE4C0422002500BF05E0002705F110008B
:107F90000F54681CC5B2042DF7DB02EBC20000EBE6
:107FA000421006EB4000807801F8140F0020487062
:107FB0008870C87002EBC20000EB421006EB400074
:107FC00090F840000871002048718871C87102EB78
:107FD000820000EB821014F8100008720020487232
:107FE0008872C87202EB820000EB821004EB400042
:107FF00090F828000873002048738873C87302EB58
:10800000820000EB821014F81000087400204874FD
:108010008874C87402EB820000EB821004EB40000D
:1080200090F828000875002048758875C87502EB1F
:10803000820000EB821014F81000087600204876C9
:108040008876C87602EB820000EB821004EB4000D9
:1080500090F828000877002048778877C87702EBE7
:10806000820000EB821014F8100081F8200000203C
:1080700081F8210081F8220081F8230002EB8200C0
:1080800000EB821004EB400090F8280081F82400F7
:10809000002081F8250081F8260081F8270002EBF6
:1080A000820000EB821004EB400090F8280081F879
:1080B0002800002081F8290081F82A0081F82B008F
:1080C00002EB820000EB821004EB400090F82800E5
:1080D00081F82C00002081F82D0081F82E0081F815
:1080E0002F0002EB820000EB821004EB400090F8BE
:1080F000280081F83000002081F8310081F832003A
:1081000081F833001439002505E0002705F1480007
:108110000F54681CC5B2202DF7DB02EB820003EB85
:10812000C000C08B38B1002001F8680F487088701B
:10813000C870683912E002EB820053F830000090FA
:108140009DF8000001F8680F9DF8010048709DF847
:10815000020088709DF80300C870683902EB820045
:1081600003EBC000C08B38B1002001F86C0F4870E1
:108170008870C8706C3913E002EB820003EBC0001A
:10818000806800909DF8000001F86C0F9DF80100D8
:1081900048709DF8020088709DF80300C8706C3923
:1081A00002EB820003EBC000C08B38B1002001F865
:1081B000700F48708870C870703913E002EB82004D
:1081C00003EBC000C06800909DF8000001F8700F3C
:1081D0009DF8010048709DF8020088709DF803002A
:1081E000C870703902EB820003EBC000C08B38B15D
:1081F000002001F8740F48708870C870743913E05B
:1082000002EB820003EBC000006900909DF80000C3
:1082100001F8740F9DF8010048709DF80200887005
:108220009DF80300C870743902EB820003EBC000B4
:10823000C08B38B1002001F8780F48708870C87082
:10824000783913E002EB820003EBC0004069009034
:108250009DF8000001F8780F9DF8010048709DF826
:10826000020088709DF80300C870783902EB820024
:1082700003EBC000C08B50B1762001F87C0F7F204B
:108280004870FF2088700020C8707C3913E002EB32
:10829000820003EBC000806900909DF8000001F8A7
:1082A0007C0F9DF8010048709DF8020088709DF8D1
:1082B0000300C8707C3902EB820003EBC000C08B66
:1082C00038B1002001F8800F48708870C87080397C
:1082D0000CE002EB820003EBC000806900900020FC
:1082E00001F8800F48708870C870803902EB8200F6
:1082F00003EBC000C08B38B1002001F8840F487038
:108300008870C87084390CE002EB820003EBC00077
:1083100080690090002001F8840F48708870C87050
:10832000843902EB820003EBC000C08B38B100201F
:1083300001F8880F48708870C87088390CE002EB2B
:10834000820003EBC00080690090002001F8880FD4
:1083500048708870C870883902EB820003EBC00057
:10836000C08B68B1002001F88C0F48708870C8700D
:108370008C3912E0583F00205C4A00207C4F0020DE
:1083800002EB820003EBC00080690090002001F83E
:108390008C0F48708870C8708C3902EB820003EB38
:1083A000C000C08B38B1002001F8900F4870887071
:1083B000C87090390CE002EB820003EBC0008069CA
:1083C0000090002001F8900F48708870C8709039B4
:1083D0000120F8BDF8B50146FD4BFE4EFE4C0522CE
:1083E000002500BF05E0002705F110000F54681CB0
:1083F000C5B2042DF7DB02EBC20000EB421006EB26
:108400004000807801F8140F002048708870C87010
:1084100002EBC20000EB421006EB400090F8400077
:108420000871002048718871C87102EB820000EB6E
:10843000821014F810000872002048728872C87206
:1084400002EB820000EB821004EB400090F8280061
:108450000873002048738873C87302EB820000EB36
:10846000821014F810000874002048748874C874CE
:1084700002EB820000EB821004EB400090F8280031
:108480000875002048758875C87502EB820000EBFE
:10849000821014F810000876002048768876C87696
:1084A00002EB820000EB821004EB400090F8280001
:1084B0000877002048778877C87702EB820000EBC6
:1084C000821014F8100081F82000002081F82100AB
:1084D00081F8220081F8230002EB820000EB821079
:1084E00004EB400090F8280081F82400002081F877
:1084F000250081F8260081F8270002EB820000EBBE
:10850000821004EB400090F8280081F82800002039
:1085100081F8290081F82A0081F82B0002EB820003
:1085200000EB821004EB400090F8280081F82C004A
:10853000002081F82D0081F82E0081F82F0002EB39
:10854000820000EB821004EB400090F8280081F8D4
:108550003000002081F8310081F8320081F83300CA
:108560001439002505E0002705F148000F54681C68
:10857000C5B2202DF7DB02EB820003EBC000C08BFD
:1085800038B1002001F8680F48708870C8706839E9
:1085900012E002EB820053F8300000909DF80000DA
:1085A00001F8680F9DF8010048709DF8020088707E
:1085B0009DF80300C870683902EB820003EBC0002D
:1085C000C08B38B1002001F86C0F48708870C870FB
:1085D0006C3913E002EB820003EBC000806800906E
:1085E0009DF8000001F86C0F9DF8010048709DF89F
:1085F000020088709DF80300C8706C3902EB82009D
:1086000003EBC000C08B38B1002001F8700F487038
:108610008870C870703913E002EB820003EBC00071
:10862000C06800909DF8000001F8700F9DF80100EF
:1086300048709DF8020088709DF80300C87070397A
:1086400002EB820003EBC000C08B38B1002001F8C0
:10865000740F48708870C870743913E002EB8200A0
:1086600003EBC000006900909DF8000001F8740F52
:108670009DF8010048709DF8020088709DF8030085
:10868000C870743902EB820003EBC000C08B38B1B4
:10869000002001F8780F48708870C870783913E0AE
:1086A00002EB820003EBC000406900909DF80000DF
:1086B00001F8780F9DF8010048709DF8020088705D
:1086C0009DF80300C870783902EB820003EBC0000C
:1086D000C08B50B1762001F87C0F7F204870FF20BE
:1086E00088700020C8707C3913E002EB820003EB35
:1086F000C000806900909DF8000001F87C0F9DF893
:10870000010048709DF8020088709DF80300C87051
:108710007C3902EB820003EBC000C08B38B1002033
:1087200001F8800F48708870C87080390CE002EB47
:10873000820003EBC00080690090002001F8800FE8
:1087400048708870C870803902EB820003EBC0006B
:10875000C08B38B1002001F8840F48708870C87051
:1087600084390CE002EB820003EBC00080690090CA
:10877000002001F8840F48708870C870843902EBBB
:10878000820003EBC000C08B38B1002001F8880FD5
:1087900048708870C87088390CE002EB820003EBE7
:1087A000C00080690090002001F8880F4870887030
:1087B000C870883902EB820003EBC000C08B68B13F
:1087C000002001F88C0F48708870C8708C3912E056
:1087D000583F00205C4A00207C4F002002EB8200C2
:1087E00003EBC00080690090002001F88C0F4870F6
:1087F0008870C8708C3902EB820003EBC000C08B1C
:1088000038B1002001F8900F48708870C870903916
:108810000CE002EB820003EBC000806900900020B6
:1088200001F8900F48708870C87090390120F8BD29
:10883000F8B50146FD4BFE4EFE4C0622002500BF5A
:1088400005E0002705F110000F54681CC5B2042D87
:10885000F7DB02EBC20000EB421006EB4000807831
:1088600001F8140F002048708870C87002EBC20035
:1088700000EB421006EB400090F840000871002029
:1088800048718871C87102EB820000EB821014F805
:1088900010000872002048728872C87202EB8200D1
:1088A00000EB821004EB400090F8280008730020D1
:1088B00048738873C87302EB820000EB821014F8CF
:1088C00010000874002048748874C87402EB820099
:1088D00000EB821004EB400090F82800087500209F
:1088E00048758875C87502EB820000EB821014F899
:1088F00010000876002048768876C87602EB820061
:1089000000EB821004EB400090F82800087700206C
:1089100048778877C87702EB820000EB821014F862
:10892000100081F82000002081F8210081F8220049
:1089300081F8230002EB820000EB821004EB400080
:1089400090F8280081F82400002081F8250081F8A3
:10895000260081F8270002EB820000EB821004EB76
:10896000400090F8280081F82800002081F82900B4
:1089700081F82A0081F82B0002EB820000EB8210C4
:1089800004EB400090F8280081F82C00002081F8CA
:108990002D0081F82E0081F82F0002EB820000EB01
:1089A000821004EB400090F8280081F8300000208D
:1089B00081F8310081F8320081F833001439002544
:1089C00005E0002705F148000F54681CC5B2202DB2
:1089D000F7DB02EB820003EBC000C08B38B1002054
:1089E00001F8680F48708870C870683912E002EBAF
:1089F000820053F8300000909DF8000001F8680FE5
:108A00009DF8010048709DF8020088709DF80300F1
:108A1000C870683902EB820003EBC000C08B38B12C
:108A2000002001F86C0F48708870C8706C3913E032
:108A300002EB820003EBC000806800909DF800000C
:108A400001F86C0F9DF8010048709DF802008870D5
:108A50009DF80300C8706C3902EB820003EBC00084
:108A6000C08B38B1002001F8700F48708870C87052
:108A7000703913E002EB820003EBC000C068009085
:108A80009DF8000001F8700F9DF8010048709DF8F6
:108A9000020088709DF80300C870703902EB8200F4
:108AA00003EBC000C08B38B1002001F8740F487090
:108AB0008870C870743913E002EB820003EBC000C9
:108AC000006900909DF8000001F8740F9DF8010006
:108AD00048709DF8020088709DF80300C8707439D2
:108AE00002EB820003EBC000C08B38B1002001F81C
:108AF000780F48708870C870783913E002EB8200F4
:108B000003EBC000406900909DF8000001F8780F69
:108B10009DF8010048709DF8020088709DF80300E0
:108B2000C870783902EB820003EBC000C08B50B1F3
:108B3000762001F87C0F7F204870FF20887000208D
:108B4000C8707C3913E002EB820003EBC00080693F
:108B500000909DF8000001F87C0F9DF8010048701E
:108B60009DF8020088709DF80300C8707C3902EB04
:108B7000820003EBC000C08B38B1002001F8800FE9
:108B800048708870C87080390CE002EB820003EBFB
:108B9000C00080690090002001F8800F4870887044
:108BA000C870803902EB820003EBC000C08B38B183
:108BB000002001F8840F48708870C87084390CE078
:108BC00002EB820003EBC00080690090002001F8F6
:108BD000840F48708870C870843902EB820003EB00
:108BE000C000C08B38B1002001F8880F4870887031
:108BF000C87088390CE002EB820003EBC00080698A
:108C00000090002001F8880F48708870C87088397B
:108C100002EB820003EBC000C08B68B1002001F8BA
:108C20008C0F48708870C8708C3912E0583F002053
:108C30005C4A00207C4F002002EB820003EBC00066
:108C400080690090002001F88C0F48708870C8700F
:108C50008C3902EB820003EBC000C08B38B10020DE
:108C600001F8900F48708870C87090390CE002EBE2
:108C7000820003EBC00080690090002001F8900F93
:108C800048708870C87090390120F8BDF8B5014669
:108C9000FD4BFE4EFE4C0722002500BF05E00027DD
:108CA00005F110000F54681CC5B2042DF7DB02EB70
:108CB000C20000EB421006EB4000807801F8140F70
:108CC000002048708870C87002EBC20000EB4210B0
:108CD00006EB400090F84000087100204871887150
:108CE000C87102EB820000EB821014F810000872C9
:108CF000002048728872C87202EB820000EB82107A
:108D000004EB400090F82800087300204873887333
:108D1000C87302EB820000EB821014F81000087494
:108D2000002048748874C87402EB820000EB821043
:108D300004EB400090F828000875002048758875FD
:108D4000C87502EB820000EB821014F81000087660
:108D5000002048768876C87602EB820000EB82100D
:108D600004EB400090F828000877002048778877C7
:108D7000C87702EB820000EB821014F8100081F833
:108D80002000002081F8210081F8220081F82300D2
:108D900002EB820000EB821004EB400090F8280008
:108DA00081F82400002081F8250081F8260081F850
:108DB000270002EB820000EB821004EB400090F8E9
:108DC000280081F82800002081F8290081F82A0075
:108DD00081F82B0002EB820000EB821004EB4000D4
:108DE00090F8280081F82C00002081F82D0081F8EF
:108DF0002E0081F82F0002EB820000EB821004EBC2
:108E0000400090F8280081F83000002081F83100FF
:108E100081F8320081F833001439002505E000277D
:108E200005F148000F54681CC5B2202DF7DB02EB9A
:108E3000820003EBC000C08B38B1002001F8680F3E
:108E400048708870C870683912E002EB820053F8ED
:108E5000300000909DF8000001F8680F9DF80100B7
:108E600048709DF8020088709DF80300C87068394A
:108E700002EB820003EBC000C08B38B1002001F888
:108E80006C0F48708870C8706C3913E002EB820078
:108E900003EBC000806800909DF8000001F86C0FA3
:108EA0009DF8010048709DF8020088709DF803004D
:108EB000C8706C3902EB820003EBC000C08B38B184
:108EC000002001F8700F48708870C870703913E086
:108ED00002EB820003EBC000C06800909DF8000028
:108EE00001F8700F9DF8010048709DF8020088702D
:108EF0009DF80300C870703902EB820003EBC000DC
:108F0000C08B38B1002001F8740F48708870C870A9
:108F1000743913E002EB820003EBC000006900909B
:108F20009DF8000001F8740F9DF8010048709DF84D
:108F3000020088709DF80300C870743902EB82004B
:108F400003EBC000C08B38B1002001F8780F4870E7
:108F50008870C870783913E002EB820003EBC00020
:108F6000406900909DF8000001F8780F9DF801001D
:108F700048709DF8020088709DF80300C870783929
:108F800002EB820003EBC000C08B50B1762001F8E9
:108F90007C0F7F204870FF2088700020C8707C39CB
:108FA00013E002EB820003EBC000806900909DF8A3
:108FB000000001F87C0F9DF8010048709DF8020048
:108FC00088709DF80300C8707C3902EB820003EBC7
:108FD000C000C08B38B1002001F8800F4870887045
:108FE000C87080390CE002EB820003EBC00080699E
:108FF0000090002001F8800F48708870C870803998
:1090000002EB820003EBC000C08B38B1002001F8F6
:10901000840F48708870C87084390CE002EB8200BD
:1090200003EBC00080690090002001F8840F4870B5
:109030008870C870843902EB820003EBC000C08BDB
:1090400038B1002001F8880F48708870C8708839DE
:109050000CE002EB820003EBC0008069009000206E
:1090600001F8880F48708870C870883902EB820058
:1090700003EBC000C08B68B1002001F88C0F487072
:109080008870C8708C3912E0583F00205C4A00207C
:109090007C4F002002EB820003EBC000806900904F
:1090A000002001F88C0F48708870C8708C3902EB72
:1090B000820003EBC000C08B38B1002001F8900F94
:1090C00048708870C87090390CE002EB820003EBA6
:1090D000C00080690090002001F8900F48708870EF
:1090E000C87090390120F8BDF8B50146FD4BFE4E21
:1090F000FE4C0822002500BF05E0002705F1100006
:109100000F54681CC5B2042DF7DB02EBC20000EB64
:10911000421006EB4000807801F8140F00204870E0
:109120008870C87002EBC20000EB421006EB4000F2
:1091300090F840000871002048718871C87102EBF6
:10914000820000EB821014F81000087200204872B0
:109150008872C87202EB820000EB821004EB4000C0
:1091600090F828000873002048738873C87302EBD6
:10917000820000EB821014F810000874002048747C
:109180008874C87402EB820000EB821004EB40008C
:1091900090F828000875002048758875C87502EB9E
:1091A000820000EB821014F8100008760020487648
:1091B0008876C87602EB820000EB821004EB400058
:1091C00090F828000877002048778877C87702EB66
:1091D000820000EB821014F8100081F820000020BB
:1091E00081F8210081F8220081F8230002EB82003F
:1091F00000EB821004EB400090F8280081F8240076
:10920000002081F8250081F8260081F8270002EB74
:10921000820000EB821004EB400090F8280081F8F7
:109220002800002081F8290081F82A0081F82B000D
:1092300002EB820000EB821004EB400090F8280063
:1092400081F82C00002081F82D0081F82E0081F893
:109250002F0002EB820000EB821004EB400090F83C
:10926000280081F83000002081F8310081F83200B8
:1092700081F833001439002505E0002705F1480086
:109280000F54681CC5B2202DF7DB02EB820003EB04
:10929000C000C08B38B1002001F8680F487088709A
:1092A000C870683912E002EB820053F83000009079
:1092B0009DF8000001F8680F9DF8010048709DF8C6
:1092C000020088709DF80300C870683902EB8200C4
:1092D00003EBC000C08B38B1002001F86C0F487060
:1092E0008870C8706C3913E002EB820003EBC00099
:1092F000806800909DF8000001F86C0F9DF8010057
:1093000048709DF8020088709DF80300C8706C39A1
:1093100002EB820003EBC000C08B38B1002001F8E3
:10932000700F48708870C870703913E002EB8200CB
:1093300003EBC000C06800909DF8000001F8700FBA
:109340009DF8010048709DF8020088709DF80300A8
:10935000C870703902EB820003EBC000C08B38B1DB
:10936000002001F8740F48708870C870743913E0D9
:1093700002EB820003EBC000006900909DF8000042
:1093800001F8740F9DF8010048709DF80200887084
:109390009DF80300C870743902EB820003EBC00033
:1093A000C08B38B1002001F8780F48708870C87001
:1093B000783913E002EB820003EBC00040690090B3
:1093C0009DF8000001F8780F9DF8010048709DF8A5
:1093D000020088709DF80300C870783902EB8200A3
:1093E00003EBC000C08B50B1762001F87C0F7F20CA
:1093F0004870FF2088700020C8707C3913E002EBB1
:10940000820003EBC000806900909DF8000001F825
:109410007C0F9DF8010048709DF8020088709DF84F
:109420000300C8707C3902EB820003EBC000C08BE4
:1094300038B1002001F8800F48708870C8708039FA
:109440000CE002EB820003EBC0008069009000207A
:1094500001F8800F48708870C870803902EB820074
:1094600003EBC000C08B38B1002001F8840F4870B6
:109470008870C87084390CE002EB820003EBC000F6
:1094800080690090002001F8840F48708870C870CF
:10949000843902EB820003EBC000C08B38B100209E
:1094A00001F8880F48708870C87088390CE002EBAA
:1094B000820003EBC00080690090002001F8880F53
:1094C00048708870C870883902EB820003EBC000D6
:1094D000C08B68B1002001F88C0F48708870C8708C
:1094E0008C3912E0583F00205C4A00207C4F00205D
:1094F00002EB820003EBC00080690090002001F8BD
:109500008C0F48708870C8708C3902EB820003EBB6
:10951000C000C08B38B1002001F8900F48708870EF
:10952000C87090390CE002EB820003EBC000806948
:109530000090002001F8900F48708870C870903932
:109540000120F8BD2DE9F04F87B00446FD48069094
:10955000FD4EFE480590DFF8F893FE4FFE4804905C
:10956000FE4803904FF0000A0025A8460020029014
:1095700083460190059890F81EB0BBF1010F02DB05
:10958000BBF1080F03DD002007B0BDE8F08F00201D
:10959000019023E006F12400019910F811005044D5
:1095A00000F0FF0A06F11400019910F81100284498
:1095B000C5B206F13400019910F81100404400F0E2
:1095C000FF0806F14400019910F8111002980844B0
:1095D000C0B202900198401CC0B20190ABF10100F2
:1095E00001998842D6DC2820E0720598807F60745B
:1095F0000AF1010000EBC00101EB4011049800EBFF
:109600004100B0F84C0010B10320A07405E00AF14D
:109610000101C8B2F9F764FDA074681C00EB0010EA
:1096200000EB400007EB4000B0F85E0010B10320F3
:10963000E07409E0681C00EB001000EB400007EB51
:10964000400090F85800E074FAF76AFDC4490860D9
:1096500008F10100C0EBC00000EB800009EB400006
:10966000408F18B103202075607515E008F10100E6
:10967000C0EBC00000EB800009EB400090F8340024
:10968000207508F10100C0EBC00000EB800009EB81
:10969000400090F836006075681C00EB001000EB8D
:1096A000400007EB4000B0F85E0010B10320A07549
:1096B00009E0681C00EB001000EB400007EB4000E5
:1096C00090F85A00A0750298401C00EB800101EB55
:1096D0008011069800EB4100B0F8840010B103201F
:1096E000E0750BE00298401C00EB800101EB80115B
:1096F000069800EB410090F87E00E075039890F822
:10970000F20020760AF1010000EBC00101EB4011EC
:10971000049800EB4100B0F84C0060B10AF1010080
:1097200000EBC00101EB4011049800EB410090F800
:10973000220060760BE00AF1010000EBC00101EBB2
:109740004011049800EB410090F822006076A520BB
:10975000A076E076ABF1010006F1240131F81000AB
:10976000012815DD0AF1020000EBC00101EB4011F8
:10977000049800EB4100B0F84C0010B103202077B2
:1097800008E00AF10201C8B2F9F7AAFC207701E06B
:10979000A5202077ABF1010006F1140131F810008B
:1097A000012824DDA81C00EB001000EB400007EBB3
:1097B0004000B0F85E0020B10320607784F82000FC
:1097C00019E0A81C00EB001000EB400007EB400084
:1097D00090F858006077A81C00EB001000EB4000E8
:1097E00007EB400090F85A0084F8200003E0A52021
:1097F000607784F82000ABF1010006F1340131F804
:109800001000012824DD08F10200C0EBC00000EBCD
:10981000800009EB4000408F18B10320A077E0776B
:1098200019E008F10200C0EBC00000EB800009EB7A
:10983000400090F83400A07708F10200C0EBC000AF
:1098400000EB800009EB400090F83600E07702E082
:10985000A520A077E077A52004F8210F6070A07004
:10986000E0702071213CABF1010006F1240131F8D8
:109870001000022817DD0AF1030000EBC00101EB24
:109880004011049800EB4100B0F84C0018B10320DF
:1098900084F826000AE00AF10301C8B2F9F720FCB7
:1098A00084F8260002E0A52084F82600ABF1010030
:1098B00006F1140131F81000022826DDE81C00EB47
:1098C000001000EB400007EB4000B0F85E0028B14C
:1098D000032084F8270084F82A001BE0E81C00EB32
:1098E000001000EB400007EB400090F8580084F8AF
:1098F0002700E81C00EB001000EB400007EB4000E5
:1099000090F85A0084F82A0004E0A52084F8270083
:1099100084F82A00ABF1010006F1340131F810009F
:10992000022838DD08F10300C0EBC00000EB800026
:1099300009EB4000408FA8B1032084F8280084F888
:1099400029002DE07C4F002060370020A238002045
:1099500000330020F63800205C4A00201C5800200C
:109960005403002008F10300C0EBC00000EB8000AE
:1099700009EB400090F8340084F8280008F1030057
:10998000C0EBC00000EB800009EB400090F836000F
:1099900084F8290004E0A52084F8280084F8290030
:1099A000A52004F82B0F6070A070E07020712B3C94
:1099B000ABF1010006F1240131F81000032817DD96
:1099C0000AF1040000EBC00101EB4011049800EB28
:1099D0004100B0F84C0018B1032084F830000AE0D0
:1099E0000AF10401C8B2F9F77BFB84F8300002E009
:1099F000A52084F83000ABF1010006F1140131F824
:109A00001000032825DD281D00EB001000EB4000AE
:109A100007EB4000B0F85E0020B1032084F831006D
:109A200084F83400281D00EB001000EB400007EB29
:109A3000400090F8580084F83100281D00EB001019
:109A400000EB400007EB400090F85A0084F8340027
:109A500004E0A52084F8310084F83400ABF1010063
:109A600006F1340131F81000042828DD08F1040063
:109A7000C0EBC00000EB800009EB4000408F28B134
:109A8000032084F8320084F833001DE008F104005C
:109A9000C0EBC00000EB800009EB400090F8340000
:109AA00084F8320008F10400C0EBC00000EB800035
:109AB00009EB400090F8360084F8330004E0A5205C
:109AC00084F8320084F83300A52004F8350F607064
:109AD000A070E0702071353C0F480068B0F5005F61
:109AE00018D20020153404F8010C207060706070EA
:109AF000A0706072A072E072E0722073E074207552
:109B000060756075A0756077A077E077E07784F87E
:109B10002000153C012037E5540300202DE9F041D9
:109B20000446934D934EDFF85082944FB87F5028EF
:109B30003BDDB87F5F2838DA607C503800EB80006E
:109B400008EBC000C08B40B14720A0747F20E074B8
:109B5000FF2020750020607507E1617C503901EB22
:109B6000810158F83100F6F75DFC000EA074617CAD
:109B7000503901EB810158F83100F6F753FC000C25
:109B8000E074617C503901EB810158F83100F6F73F
:109B900049FC000A2075617C503901EB810158F8BD
:109BA0003100F6F73FFC6075DFE0B87F60287DDDAF
:109BB000B87F6F287ADA607C603806EBC010B0F8A6
:109BC0007A00B8B14720A0747F20E074FF20207590
:109BD000002060754720A0757F20E075FF2020766B
:109BE000002060764720A0767F20E076FF20207757
:109BF00000206077607C603806EBC010B0F9000090
:109C0000000EA074607C603806EBC010B0F9000054
:109C1000000CE074607C603806EBC0100088000A1D
:109C20002075607C603806EBC01000786075607C41
:109C3000603806EBC010B0F92800000EA075607CFB
:109C4000603806EBC010B0F92800000CE075607CAD
:109C5000603806EBC010008D000A2076607C60380A
:109C600006EBC01090F828006076607C603806EB48
:109C7000C010B0F95000000EA076607C603806EB92
:109C8000C010B0F95000000CE076607C603806EB44
:109C9000C010B0F85000000A2077607C603806EBF6
:109CA000C01090F8500060775FE0FFE7B87F702841
:109CB00002DDB87F7F2858DBB87F802802DDB87FBF
:109CC0008F2852DBB87FE02849DDB87FE32846DAE9
:109CD000B5F87A00C0B14720A0747F20E074FF205F
:109CE0002075002060754720A0757F20E075FF205B
:109CF0002076002060764720A0767F20E076FF2047
:109D000020770020607730E0B5F90000000EA074E5
:109D1000B5F90000000CE0742888000A2075287846
:109D20006075B5F92800000EA074B5F92800000C84
:109D3000E074288D000A207595F828006075B5F943
:109D40005000000EA074B5F95000000CE074B5F896
:109D50005000000A207595F85000607505E0B87F46
:109D6000E42802D00020BDE8F0810120FBE70000DC
:109D7000D84100205C420020583F0020A23800203B
:109D80000246002124E0144850F82100000E102360
:109D900003EB8103D054104850F82100C0F307436F
:109DA000012000EB8100103013540B4830F82100E3
:109DB000C0F30723022000EB810010301354064843
:109DC00010F82130032000EB810010301354491C9F
:109DD0000829D8DB012070475C030020F8B5044651
:109DE000264D0026B5F90000F6F70EFB074624497C
:109DF000F6F79AFA00909DF8000020749DF8010093
:109E000060749DF80200A0749DF80300E074B5F939
:109E10002800F6F7F9FA07461949F6F785FA00908F
:109E20009DF8000020759DF8010060759DF8020006
:109E3000A0759DF80300E075B5F95000F6F7E4FA57
:109E400007460F49F6F770FA00909DF8000020765B
:109E50009DF8010060769DF80200A0769DF8030051
:109E6000E07600BF05E0A52106F11C002154701C1E
:109E7000C6B2E42EF7DB0120F8BD0000D841002077
:109E80000000B43B72B621E0012080F3138800BFCC
:109E900000BF00BF00BF00BF00BFBFF34F8F00BFB8
:109EA00000BF00BF0A48006800F4E06009490843A9
:109EB000001D0749086000BF00BF00BFBFF34F8F00
:109EC00000BF00BF00BF00BF00BFFDE7DCE7000030
:109ED0000CED00E00000FA052DE9FC5F0446DFF818
:109EE000F491DFF8F4A17D480190002000908346B2
:109EF0008046002500260027AA20207000206070E0
:109F0000A120A0701120E0700020207100BFCEE0E1
:109F10007806050E0021681D2154A81D2154002635
:109F200046E0701C4044C0EBC00000EB80000AEB30
:109F30004000408F30B1681D205C40F01001681D6A
:109F400021540FE0701C4044C0EBC00000EB8000C7
:109F50000AEB4000808E28B1681D205C40F00101B2
:109F6000681D2154B9F80A0000B3701C4044C0EBCE
:109F7000C00000EB80000AEB4000C08F30B1681DCC
:109F8000205C40F02001681D21540FE0701C40440B
:109F9000C0EBC00000EB80000AEB4000C08E28B18F
:109FA000681D205C40F00201681D2154701CC6B27F
:109FB00009F1340030F81700B042B2DC08EB0600BB
:109FC00000F0FF0800263BE0701C584400EB001036
:109FD00000EB4001019800EB4100B0F85E0060B179
:109FE000681D205C40F08001681D2154A81D205C84
:109FF00040F05501A81D215420E0701C584400EB8E
:10A00000001000EB4001019800EB4100B0F858004F
:10A0100028B1681D205C40F00801681D2154701CA7
:10A02000584400EB001000EB4001019800EB4100A8
:10A03000B0F85A0010B10121A81D2154701CC6B2FD
:10A0400009F1140030F81700B042BDDC0BEB06003C
:10A0500000F0FF0B00261DE0711C009A1144C8B2ED
:10A06000F9F73EF8012806D1681D205C40F0040194
:10A07000681D21540CE0711C009A1144C8B2F9F714
:10A080002FF828B1681D205C00F04001681D2154A4
:10A09000701CC6B209F1240030F81700B042DBDCB6
:10A0A00000983044C0B200900026781CC7B2082F38
:10A0B000FFF62EAF0A480068B0F5005F08D200270F
:10A0C00004E00021781D2154781CC7B2102FF8DB62
:10A0D000BDE8FC9F6037002000330020F6380020E8
:10A0E00054030020F0B585B004461B4E1B4F1C4D99
:10A0F00014216846F6F7B5F8A97F687F41EA002089
:10A10000ADF80000287D062804D1012215496846D3
:10A11000F7F72AFB012213496846F7F70FFBBDF852
:10A120000000A6F84000BDF80000A7F86000BDF8E8
:10A13000000000122074BDF800006074217C687F6C
:10A14000814206D1617CA87F814202D1012005B005
:10A15000F0BD0020FBE7000000330020F6380020AF
:10A16000A238002064F0070800BF012003F0F8FACD
:10A17000FBE700001CB54FF00008C14600BF0024FB
:10A18000A246FD480190FD480090FD4EFD4DFE4F5A
:10A1900000BFA3460020FD49088016E005F1140029
:10A1A000FA49098830F8110050441FFA80FA05F185
:10A1B0002400F649098830F8110058441FFA80FB42
:10A1C000F2480088401CF14908802888EF49098836
:10A1D0008842E3DC0020ED49088000BF0A2003F03C
:10A1E000BFFA4FF48061EA48F9F78AFFE94800783E
:10A1F00028B34FF0000AD3460020E449088016E057
:10A2000005F11400E149098830F8110050441FFAA3
:10A2100080FA05F12400DD49098830F8110058441E
:10A220001FFA80FBD9480088401CD849088028883C
:10A23000D64909888842E3DC0020D6490870009896
:10A24000408800287DD1B8F1000F53D1288A00281A
:10A250004ED0A88802284BD00621CF48FBF718FC27
:10A2600004462012CC498871CC7100224FF48051F1
:10A27000CA48F9F74FFF502002F02EFF0822C649C6
:10A28000C748FBF77AF902E0012003F069FAC448F5
:10A2900090F839002128F7D001221103BF48F9F7BF
:10A2A00039FFBD480078103800EB001000EB40008B
:10A2B00006EB4000B0F86400401C81B2B64800785C
:10A2C000103800EB001000EB400006EB4000A0F857
:10A2D0006410B14800781038504505DAAE4800786F
:10A2E000401CAD49087005E01120AB49087001E041
:10A2F0004FF00308B8F1030F37D1B5F86C0088B3FD
:10A300000621A848FBF7C4FB04462012A549887122
:10A31000CC7100224FF48051A048F9F7FBFE502089
:10A3200002F0DAFE642308229E499D48FBF7BCF840
:10A33000502002F0D1FE012211039848F9F7EAFEFD
:10A3400000E0C7E0B7F87E003C2805DD3C20A7F818
:10A350007E00A7F8780008E0B7F87E00401CA7F858
:10A360007E0002E0FFE74FF00608B8F1060F24D1A7
:10A37000E88900B306218C48FBF78AFB04462012CB
:10A3800089498871CC7100224FF480518348F9F7D4
:10A39000C1FE502002F0A0FE6423082282498048BA
:10A3A000FBF782F8502002F097FE012211037B4850
:10A3B000F9F7B0FE01E04FF00908B8F1090F5FD1DD
:10A3C000688A00285AD0E888F0B30E217748FBF756
:10A3D0005FFB0446201275498873CC7300224FF44A
:10A3E00080516E48F9F796FE502002F075FE642306
:10A3F00010226E496A48FBF757F8502002F06CFEB5
:10A40000012211036548F9F785FE68480078203875
:10A4100000EBC00101EB4011019800EB4100B0F8E6
:10A42000500032281BDC61480078203800EBC00166
:10A4300001EB4011019800EB4100B0F85000401CC6
:10A4400081B25A48007800E018E0203800EBC002E2
:10A4500002EB4012019800EB4200A0F85010534864
:10A4600000782138584505DA50480078401C4F499B
:10A47000087005E021204D49087001E04FF00C08FC
:10A48000B8F10C0F5ED1B5F86E0000B30621484854
:10A49000FBF7FEFA0446201245498871CC71002270
:10A4A0004FF480513D48F9F735FE502002F014FE7C
:10A4B000642308223E493A48FAF7F6FF502002F09A
:10A4C0000BFE012211033548F9F724FE3AE04FF064
:10A4D000000883E6B9F1030F1DD100224FF480512B
:10A4E0002E48F9F717FE502002F0F6FD3148028899
:10A4F00031492B48FBF741F802E0012003F030F925
:10A50000274890F839002128F7D001221103234869
:10A51000F9F700FE06E0B9F1060F03D1002100981B
:10A520004180894609F1010000F0FF0923480068D5
:10A53000012807D1B9F1030F04DD00210098418003
:10A5400089464BE61D48006801287CD100201B4944
:10A5500008601B480078102876DB194800781F280F
:10A5600072DC174840790402154880790443144886
:10A57000407803282ED025E05C4A0020A238002035
:10A58000F638002060370020D84100201403002056
:10A5900000100140F802002090010020000C014052
:10A5A000300C0020D2010020DA0100209A010020A6
:10A5B000CA010020FA090020163800204C030020B0
:10A5C000002B00209E484078062803D001209D499A
:10A5D000088010E09A488078022803D00120994929
:10A5E000088008E005219648FBF752FAA04202D005
:10A5F0000120944908809348008800287ED10021DA
:10A600008F480078103800EB001000EB400006EB9C
:10A610004000A0F85C108A480078103800EB001069
:10A6200000EB400006EB4000A0F85E108448407844
:10A6300003281ED18248C1780078103800EB001042
:10A6400000EB400001E0A5E017E026F810107C4880
:10A6500001790078103800EB001000EB400006EBA9
:10A660004000018576490978103988B202F048FA2D
:10A6700000E000BF4FF00308B0E571480078702893
:10A6800068DB6F4800787F2864DC6D48C07904027D
:10A690006B48007A04430120A7F87E0068484078A0
:10A6A000032807D066484078062803D00120654972
:10A6B00008800DE062488078082803DB01206149AA
:10A6C000088005E05E488078C11C5D48FBF7E0F932
:10A6D0005C48008890B95A484078032856D15A48B7
:10A6E000008814282EDA0020A7F878005448007952
:10A6F0005349C97840EA012000B200E029E05249FC
:10A70000098827F811004E4880794D49497940EA77
:10A71000012001B207F128004B4A128820F81210DC
:10A720004748007A4649C97940EA012001B207F159
:10A730005000454A128820F8121043480088401CF7
:10A74000414908804048008814281FD100203E4914
:10A7500008801BE03A480078202806DB384800785B
:10A760002F2802DCF8F766FD10E035480078E42871
:10A7700002D1F8F70FFD09E031480078812805DBA8
:10A780002F4800788F2801DCF8F756FC00202D496F
:10A79000088046E0B8F1020F43D12C480078112818
:10A7A00003D12B48A0F800A004E028480078113815
:10A7B000274908802648008800EB001000EB400085
:10A7C00006EB4000B0F85C00401C2149098801EB11
:10A7D000011101EB410106EB4101A1F85C001C48AD
:10A7E000008800EB001000EB400006EB4000B0F8E2
:10A7F0005C00032815DD0B201549098801EB0111C8
:10A8000001EB410106EB4101A1F85C000120104978
:10A81000098801EB011101EB410106EB4101A1F8AF
:10A820005E00B8F10F0F04DA08F1010000F0FF0834
:10A8300001E04FF00008282002F092FFCEE4000073
:10A84000002B002018030020160300209001002098
:10A85000140300201FB54FF0000A0020039081462A
:10A8600002900024DFF8F4B3FD480090FD4DFE4E49
:10A87000FE4FDFF8FC8300BFB6F86600022802D165
:10A880000320A6F866000020FA49088011E006F1CE
:10A890003400F849098830F8110050441FFA80FA52
:10A8A00009F101001FFA80F9F2480088401CF149C3
:10A8B00008803088EF4909888842E8DC96F866000D
:10A8C00010B9CDF80C9005E096F8660000FB09F091
:10A8D00080B203900020E749088000BF0A2002F000
:10A8E0003FFF4FF48061E448F9F70AFCE348007841
:10A8F00098B34FF0000AD146B6F86600022802D19C
:10A900000320A6F866000020DA49088011E006F16D
:10A910003400D849098830F8110050441FFA80FAF1
:10A9200009F101001FFA80F9D2480088401CD14982
:10A9300008803088CF4909888842E8DC96F86600AC
:10A9400010B9CDF80C9005E096F8660000FB09F010
:10A9500080B203900020C949087000980088002840
:10A9600074D1C7480078002879D1B089002873D005
:10A970003089022870D00621C248FBF789F8C24905
:10A980000880084600880012BE498871BE480078D9
:10A99000C87100224FF40051BC48F9F7BBFB5020AE
:10A9A00002F09AFB0822B749B948FAF7E6FD02E03F
:10A9B000012002F0D5FEB64890F839002128F7D0E2
:10A9C00001225103B148F9F7A5FBAE4800783038B1
:10A9D000C0EBC00000EB800005EB4000B0F8440085
:10A9E000401C81B2A74800783038C0EBC00000EBB3
:10A9F000800005EB4000A0F844103089D8B9A14888
:10AA00000078302813D19F480178A2480278007856
:10AA1000401CA04B187088189A49087008460078A6
:10AA2000303850451BDB01201946087017E03020F4
:10AA30009449087013E0934800783038504507DA9D
:10AA400090480078401C8F49087008E0C7E103E097
:10AA500031208C49087002E0032089490870884839
:10AA6000007803287ED1708901287CD106218A488C
:10AA7000FBF70EF8844908800846008800128649D2
:10AA8000887181480078C87100224FF400517F48D6
:10AA9000F9F740FB502002F01FFB3089012805D157
:10AAA0000A2302227D497A48FAF7FEFC6423082231
:10AAB00079497748FAF7F8FC3089012805D10A234B
:10AAC000022276497248FAF7EFFC502002F004FBAC
:10AAD000012251036D48F9F71DFB6F48007840389B
:10AAE000C0EBC00000EB800005EB4000B0F8440074
:10AAF0003C2816DD3C21684800784038C0EBC00097
:10AB000000EB800005EB4000A0F84410624800789C
:10AB10004038C0EBC00000EB800005EB40008187AF
:10AB200017E05D4800784038C0EBC00000EB8000C3
:10AB300005EB4000B0F84400401C81B25648007854
:10AB40004038C0EBC00000EB800005EB4000A0F8EF
:10AB50004410514800784138AAF10101884208DACE
:10AB60004D4801E00CE008E00078401C4A490870BC
:10AB700006E041204849087002E00620404908707C
:10AB80003F480078062805D1B6F8640018B90920B6
:10AB90003B490870CCE0B6F8640001284CD106218E
:10ABA0003F48FAF775FF38490880084600880012C8
:10ABB0003B49887134480078C87100224FF4005135
:10ABC0003248F9F7A7FA502002F086FA08223449F1
:10ABD0002F48FAF7D2FC02E0012002F0C1FD2C4818
:10ABE00090F839002128F7D0012251032748F9F7BE
:10ABF00091FA2B480078503800EB800007EBC0003A
:10AC0000408C401C81B226480078503800EB800010
:10AC100007EBC0004184224800785138A9F10101B6
:10AC2000884205DA1E480078401C1D4908707FE004
:10AC300051201B4908707BE0B6F86400022874D1EB
:10AC400006211848FAF724FF0F49088008460088B3
:10AC50000012144988710C48007825E0802E0020ED
:10AC6000A23800200033002060370020583F002029
:10AC70005C4200201E03002000100140F80200206A
:10AC80001A030020AA0100202C030020000C014020
:10AC9000B00B00201C030020BE0100209801002002
:10ACA000EA010020E2010020C87100224FF40051A7
:10ACB000FE48F9F72FFA502002F00EFA0822FC495C
:10ACC000FC48FAF75AFC02E0012002F049FDF9487D
:10ACD00090F839002128F7D001225103F348F9F701
:10ACE00019FAF3480078503800EB800007EBC000F9
:10ACF000408C401C81B2EE480078503800EB800058
:10AD000007EBC0004184EA4800785038A9F10101FE
:10AD1000884206DAE6480078401CE549087007E0FA
:10AD200003E05120E249087002E00920E24908707E
:10AD3000E1480078092849D1B6F86600F0B3062149
:10AD4000DE48FAF7A5FEDE490880084600880012B2
:10AD5000DA498871DA480078C87100224FF400514E
:10AD6000D248F9F7D7F9502002F0B6F90822D349B2
:10AD7000D048FAF702FC02E0012002F0F1FCCD48D5
:10AD800090F839002128F7D001225103C748F9F77C
:10AD9000C1F9CA480078603808EBC010B0F87E00EE
:10ADA000401C81B2C5480078603808EBC010A0F89C
:10ADB0007E10C24800786038039900E00BE08842BA
:10ADC00005DABE480078401CBC4908703CE06120B0
:10ADD000BA49087038E00020B74908707EE5B948E4
:10ADE000007803281CD100224FF40051AF48F9F736
:10ADF00091F9502002F070F9B3480288B349AD4888
:10AE0000FAF7BBFB02E0012002F0AAFCA94890F887
:10AE100039002128F7D001225103A448F9F77AF923
:10AE2000A8480078401CA7490870A9480068012874
:10AE30000AD108460078032806DD00210098018029
:10AE40000020A049087049E5A148006801287DD18B
:10AE500000209F4908609F4908709F4880780190B2
:10AE60000198C01C9C49085C000295490880019823
:10AE7000001D9949085C9249098808439049088057
:10AE80009548005D30287CDB9348005D3F2878DCE6
:10AE90009149601C085C032807D0601C085C0628E8
:10AEA00003D001208B49087013E08B49A01C085C7B
:10AEB000042803D00120874908700AE0072186484A
:10AEC000FAF7E6FD7E490988884202D001208149CF
:10AED00008708149E01C095C7F4A201D105C41EA32
:10AEE000002002901146601C085C03287ED179483E
:10AEF00000780028FAD100211046005D3038C0EB00
:10AF0000C00000EB800005EB400001871046005DAB
:10AF10003038C0EBC00000EB800005EB40004187FB
:10AF20001046015D0298F5F745FB6B48005D30382F
:10AF300000EBC0000BEBC000B0F9060000280EDBF0
:10AF40006548005D303800EBC00000E05FE30BEBCC
:10AF5000C000B0F9060046F67811884217DB5E485B
:10AF6000005D3038C0EBC00000EB800005EB400016
:10AF7000008F401C81B25848005D3038C0EBC000E3
:10AF800000E0C4E000EB800005EB40000187308961
:10AF900020B95149085D0021F5F7ECFB4E48005DF2
:10AFA000303800EBC0000BEBC000B0F90600002801
:10AFB0000CDA4948005D303800EBC0000BEBC000F4
:10AFC000B0F9060046F6781188426DDC4248005D13
:10AFD000303800EBC0000BEBC000B0F90600404277
:10AFE000B5F8421088420EDC3B4800E0BEE2005D4E
:10AFF000303800EBC0000BEBC000B0F90600B5F82C
:10B000004210884216DD3448005D3038C0EBC00085
:10B0100000EB800005EB4000008E401C81B22E4802
:10B02000005D3038C0EBC00000EB800005EB400055
:10B0300001860AE000212848005D3038C0EBC000DE
:10B0400000EB800005EB400001862348005D3038AE
:10B05000C0EBC00000EB800005EB4000018E1E48F5
:10B06000005D3038C0EBC00000EB800005EB400015
:10B07000B0F8400081423BDB1748005D3038C0EB40
:10B08000C00000EB800005EB4000B0F84010124813
:10B09000005D3038C0EBC00000EB800005EB4000E5
:10B0A000018601210C4819E02DE00000000C014050
:10B0B000E2010020B00B00201A030020F201002062
:10B0C0002C0300201B030020FA090020D0370020A9
:10B0D000440300201D03002000250020005D3038BF
:10B0E000C0EBC00000EB800005EB400081860AE069
:10B0F0000021F748005D3038C0EBC00000EB800055
:10B1000005EB400081860320F249087066E6F048AE
:10B11000005D40287EDBEE48005D4F287ADC002190
:10B12000EB48005D3038C0EBC00000EB800005EB61
:10B13000400081870121E648005D4038C0EBC00037
:10B1400000EB800005EB4000A0F84410E049601CD3
:10B15000085C032807D0601C085C062803D0012087
:10B16000DD49087013E0DA49A01C085C042803D00C
:10B170000120D94908700AE00721D548FAF788FC70
:10B18000D6490988884202D00120D3490870D049A5
:10B19000601C085C032855D1CF480078D8BB0B460B
:10B1A000221D9B5C8C46E21C1CF8022043EA022014
:10B1B0000A46115DF5F7FEF9C9480088082839DA12
:10B1C000C349201D085C0102C148005D4038C0EB46
:10B1D000C00000EB800005EB40001030C04A128830
:10B1E00020F81210BA48005D4038C0EBC00000EBF8
:10B1F000800005EB40001030B949098830F8110093
:10B20000B34AE11C515C08431146095D4039C1EB6A
:10B21000C10101E01BE015E001EB810105EB4101FB
:10B220001031AF4A128821F81200AD480088401C46
:10B23000AB490880AA480088082804D10020A84902
:10B24000088000E000BF0620A2490870C6E5A048BB
:10B25000007850287BDB9E4800785F2877DCB6F8C2
:10B260006400012874D1012199480078503800EB1E
:10B27000800007EBC00041840021954800785038D9
:10B2800000EB800007EBC0008183914840780428E0
:10B2900003D001209049087012E08D488078202862
:10B2A00003D001208C4908700AE023218848FAF76E
:10B2B000EFFB8A490988884202D00120864908703C
:10B2C0008349601C085C042879D183480078E8BB76
:10B2D00008464079834908707D48807948707C48E9
:10B2E000C07888707A480079C87008460168784844
:10B2F000005D503800EB800047F830107448407B08
:10B30000784908707248807B48707148C07A8870AC
:10B310006F48007BC870084601686D48005D503872
:10B3200000EB800007EBC00081606948407C6D49FC
:10B3300008706748807C48706548C07B88706448A6
:10B34000007CC87008460168614802E037E092E07E
:10B3500036E0005D503800EB800007EBC0008160F4
:10B360005B48407D5F4908705948807D4870584867
:10B37000C07C88705648007DC870084601685448F3
:10B38000005D503800EB800007EBC00001615048C1
:10B39000407E544908704E48807E48704C48C07DBD
:10B3A00088704B48007EC870084601684848005DB8
:10B3B000503800EB800007EBC000416157E056E0D9
:10B3C000B6F86400022852D1012141480078503873
:10B3D00000EB800007EBC000418400213C4800786E
:10B3E000503800EB800007EBC0008183384840787C
:10B3F000042803D001203849087012E034488078CE
:10B40000042803D00120344908700AE0072130489D
:10B41000FAF73EFB31490988884202D001202E49C3
:10B42000087007212A48FAF733FBA6F86800284974
:10B43000601C085C042819D127480078B0B9084678
:10B440000079284908702248C078487020488079DF
:10B4500088701F484079C870084601681C48005D24
:10B46000503800EB800047F8301000E000BF0920A2
:10B4700018490870B2E416480078602876DB144852
:10B4800000786F2872DC012117480078603808EBDB
:10B49000C010A0F87E10002113480078603808EB37
:10B4A000C010A0F878100A484078032807D0084850
:10B4B0004078062803D0012007490870A3E004481B
:10B4C0008078022812D00120034908709BE0000018
:10B4D000002500201A0300201D0300202C0300205B
:10B4E0002203002030030020F201002005219B48A8
:10B4F000FAF7CEFA9A490988884203D0012099497F
:10B50000087080E09549601C085C03287BD1954851
:10B51000007850BBB6F86600012828D108460079AB
:10B52000C97840EA012001B28C48005D603808EB20
:10B53000C0104180894800798849C97840EA0120D3
:10B5400001B28648005D603808EBC0104185834831
:10B5500000798249C97840EA012001B27F48005D44
:10B56000603808EBC010A0F852104CE0E5E0B6F8E7
:10B570006600032847D17948005D61387A49088020
:10B5800008460088032190FBF1F201FB120020B174
:10B59000012813D0022834D121E073480088032108
:10B5A00090FBF1F0401C08EBC0116C4800796B4A2D
:10B5B000D27840EA022000B2488023E06A4800883E
:10B5C000032190FBF1F0401C08EBC010634909799E
:10B5D000624AD27841EA022109B2418512E062480A
:10B5E0000088032190FBF1F0401C08EBC0105B4980
:10B5F00009795A4AD27841EA022109B2A0F85210D8
:10B6000000E000BF00BF0020584908701BE4574805
:10B61000007802285DD13089E0B95548007830289B
:10B6200014D154480078012803D14F48A0F800A055
:10B630001DE05048007828B14E480078401E4A4925
:10B64000088014E001204849088010E000204649A5
:10B6500008800CE046480078312803D14248A0F821
:10B6600000A004E04248007831383F4908803E4855
:10B670000088C0EBC00000EB800005EB4000008FAD
:10B68000401C39490988C1EBC10101EB810105EB7F
:10B690004101088734480088C0EBC00000EB8000FF
:10B6A00005EB4000008F032813DD0B202E4909888D
:10B6B000C1EBC10101EB810105EB410108870120CC
:10B6C00029490988C1EBC10101EB810105EB410169
:10B6D00048872648007808282FD1B6F8640001284A
:10B6E00004D1254800782049088007E0B6F86400B6
:10B6F000022803D1214800781B490880B6F864006D
:10B70000D8B119480088512803D11748A0F80090F3
:10B7100004E0154800885138134908801248008811
:10B7200000EB800007EBC000808B401C0E490988AD
:10B7300001EB810107EBC10188830C4800780C28DC
:10B7400005DA0A480078401C0849087002E0002029
:10B7500006490870282002F003F8D7E400250020ED
:10B760002C0300201D0300201E0300201A030020CC
:10B77000AA0100201C030020EA010020E2010020B1
:10B780000EB5F94C4FF00009CA4600BFCB46002069
:10B7900002900190F54D00BF322001F0E1FF4FF41F
:10B7A0008061F348F8F7ACFCF248006801287AD1D0
:10B7B0000020F0490860F04800783A2843D1EE486C
:10B7C000407833283FD1EC48807839283BD1EA488B
:10B7D000C078302837D1E9480068832805D0E84888
:10B7E0000068401CE6490860D6E7002610E0E24900
:10B7F000491C01EB4600FAF73DFAE2498855DE495B
:10B80000491C01EB4600FAF735FADF498855761CEA
:10B81000DA490968C81E00EBD071B6EB610FE6DBB0
:10B82000D6480068C01E009000EBD0704210D64988
:10B83000D148F4F7FDFCD1490968C81E00EBD0716E
:10B840004910CE4A1160CD480068052800DAA3E708
:10B85000CA480068401EC849085C4FEA0029C7482A
:10B860000068801E085C40EA0909C4480088801E00
:10B8700081B2C148FAF70CF9BF480078392813D0D3
:10B88000BD48407801280FDCBB48807895280BDC48
:10B89000B948C078502807DCE888401CE8800120BF
:10B8A000B749086047E0A2E2B3484079012806D0D2
:10B8B000E888401CE8800120B14908603BE0AE48C0
:10B8C000C07903280AD0AC48C079062806D0E88899
:10B8D000401CE8800120AA4908602CE00020E88094
:10B8E000A7490860A94908800DE0A348A74909882D
:10B8F000415C05F10D00A54A12888154A3480088D7
:10B90000401CA2490880A14800884028EDDB0020A7
:10B910009E4908800BE098489C490988405C9B49F7
:10B920000988605499480088401C984908809748C5
:10B9300000881028EFDB9248006800287DD18E48EF
:10B94000007A688168894FF6FF7101EA00206881FA
:10B9500068898949497A08436881688973286DD064
:10B9600036DC29286BD012DCA0F11000192867D230
:10B97000DFE800F0787B7C7D6666666666666666F4
:10B9800066666666868B8C8D8E8F90959A0052289F
:10B9900071D00EDC43286FD006DC40286DD04128E2
:10B9A0006CD042284CD1A1E0502868D05128F9D160
:10B9B000BCE070286FD006DC53286DD054286CD0C2
:10B9C0005528EFD1E8E0712868D07228EAD1EEE07E
:10B9D000B0F5BF7F72D01CDC7A2870D008DCA0F1F3
:10B9E00074000628C3D2DFE800F0F2FAEFEEEDECC7
:10B9F0007E2876D006DC7B2874D07C2873D07D2806
:10BA0000D0D12EE1A0F2211000286DD00128C9D19B
:10BA10004DE141F29512811A904271D01ADC41F247
:10BA20002112A0EB020190426BD00EDCB0F5C07F7A
:10BA300068D0B0F5C87F77D003E0D5E1BCE034E052
:10BA4000FBE0B0F5087FADD132E172296DD07329EA
:10BA5000A8D13CE107298AD2DFE801F0EFEEEDEC56
:10BA6000EBEAE900FEF70EFA5AE159E158E14848DD
:10BA7000FEF732FA54E15EE039E017E035E037E0F6
:10BA80002046FDF75FFD82464AE149E148E147E192
:10BA900046E145E144E184E07CE07CE082E0204650
:10BAA000FAF70EFD82463BE13AE139E12046F4F730
:10BAB000BBFF82460020354908800DE0DFE0BDE095
:10BAC0002D4832490988405C3049098860542F4824
:10BAD0000088401C2D4908802C4800884028EFDB56
:10BAE0001EE1C5E0AFE0B5E0E0E019E118E117E1E3
:10BAF000204600F0E1FE82460020244908800EE046
:10BB0000EAE0DAE0C2E01C4820490988405C1F49AD
:10BB1000098860541D480088401C1C4908801B4847
:10BB200000884028EFDBFBE0B8E0CBE0204600F0E7
:10BB300017FF8246F4E02046FAF758FC82460020C0
:10BB4000124908800BE00C4810490988405C0F49F5
:10BB5000098860540D480088401C0C4908800B4837
:10BB600000884028EFDBDBE090000020A2380020B6
:10BB70000010014048030020002900203803002065
:10BB8000100300201C000020000E002034030020C1
:10BB9000800E0020C4E0C3E02046FDF7BFFF8246D0
:10BBA000BEE0BDE02046F5F703F88246B8E0204647
:10BBB000FAF76AFB8246B3E02046FEF793FA824624
:10BBC000AEE02CE023E01AE011E008E0FFE72046B9
:10BBD000F5F740F88246012085490870A0E020462C
:10BBE000FAF790FB824601208149087098E02046D0
:10BBF00000F012FF824601207D49087090E0204647
:10BC0000F9F760FD824601207949087088E02046F6
:10BC1000F9F7ECFF824601207549087080E0204664
:10BC2000F4F7BEFE824601207149087078E071E0A9
:10BC30006BE065E05FE059E053E070E0204600F023
:10BC400025FB82466CE02046F9F7B0FD01206849EB
:10BC5000087065E02046F9F79DFE012064490870F0
:10BC60005EE02046F9F71CFE01206149087057E0AC
:10BC70002046F9F7AFFC01205D49087050E02046EE
:10BC800000F048FA01205A49087049E02046F5F7CB
:10BC9000B1FD824601205649087041E02046F9F77F
:10BCA0001FFF824601205249087000BF38E037E08C
:10BCB0002046FEF765F8824632E02046FBF708F89A
:10BCC00083462DE02046FAF725FD029028E0204625
:10BCD000FBF74EFC029023E02046FBF71FFF02908B
:10BCE0001EE02046FCF748F9029019E02046FCF7D8
:10BCF00071FB029014E02046FCF79AFD02900FE0E1
:10BD00002046FCF7C3FF02900AE02046FDF7ECF95D
:10BD1000029005E02046FEF761F8019000E000BFC8
:10BD200000BF00276889132803D1DFF8C8803E27A9
:10BD30002CE0029820B100200290A046942725E034
:10BD4000019820B100200190A04660271EE0BBF1C1
:10BD5000000F09D04FF0000B002084F8E80084F8B1
:10BD6000E900A046EA2711E0BAF1000F07D0002051
:10BD700084F83C0084F83D00A0463E2706E0FF2002
:10BD800084F83C0084F83D00A0463E274FF0000AAE
:10BD900057B339464046F9F77BFE81464FEA2920E2
:10BDA00008F80700781C08F80090002210211248BB
:10BDB000F8F7B0F9502001F08FF9B81C82B2414673
:10BDC0000E48F9F7DAFB02E0012001F0C9FC0B484C
:10BDD00090F839002128F7D0502001F07DF9012298
:10BDE00010210548F8F796F9002005490860D3E4CA
:10BDF000F8020020800E002000080140F00B002017
:10BE000048030020244E254FDFF89480DFF89490FB
:10BE100000BF4FF480612448F8F772F9F4F70CFD85
:10BE2000002434E0052C19D2DFE804F00304090EE5
:10BE3000130014E0DFF86880DFF868900FE0DFF8A7
:10BE40006C80DFF86C900AE0DFF86880DFF86890BB
:10BE500005E0DFF86880DFF8689000E000BF00BF11
:10BE600004EB840156F8310023464A464146F4F774
:10BE70002BFF054604EB840006EBC00085612046DD
:10BE8000F5F794FA642001F06BFC601CC4B23888AA
:10BE9000A042BEDDC6E70000583F0020603700200A
:10BEA00080030020740401080010014010050020E8
:10BEB00004060108A00600209407010830080020AD
:10BEC0002409010800BF012001F04AFCFBE700BF84
:10BED000012001F045FCFBE700BF012001F040FC20
:10BEE000FBE700BF012001F03BFCFBE700BF0120A6
:10BEF00001F036FCFBE700BF012001F031FCFBE75D
:10BF000000BF4FF4FA7001F02BFC07480068401C9A
:10BF10000549086001210548F8F7F2F84FF48061FF
:10BF20000348F8F7EDF8ECE70400002000080140B2
:10BF30000010014010B500BF502080F31188BFF3FE
:10BF40004F8FBFF36F8F00BF03F090FC18B14FF01D
:10BF500080500449086000BF002080F3118800BFB2
:10BF600010BD000004ED00E000B58FB0282105A849
:10BF7000F4F777F914216846F4F773F90120059076
:10BF800000040690002007900120099002200C90E8
:10BF9000C1030D914FF4E0110E9105A8F8F714FBC1
:10BFA00008B1F5F716FB0F20009002200190002049
:10BFB00002904FF4806003900020049002216846B4
:10BFC000F8F7AAF908B1F5F704FB0FB000BD704708
:10BFD00010B50248F8F7A7FE10BD0000E00A0020E7
:10BFE00010B50248F8F79FFE10BD0000280B002096
:10BFF00010B50248F8F797FE10BD00005C0F002056
:10C0000010B50268204B98420ED0204B98420BD0BE
:10C01000B0F1804F08D01E4B984205D01D4B98427E
:10C0200002D01D4B984203D122F070024B681A4394
:10C03000154B98420ED0154B98420BD0B0F1804F63
:10C0400008D0134B984205D0124B984202D0124BA5
:10C05000984203D122F44072CB681A4322F0800345
:10C060004C6943EA040202608B68C3620B68836216
:10C07000054B984202D0054B984201D10B690363EE
:10C080000123436110BD0000002C01400034014039
:10C090000004004000080040000C004030B50C4691
:10C0A000816821F47F4142EA0325254329438160C9
:10C0B00030BD0A46816821F0700142F00703194340
:10C0C0008160704730B50B461446026A056A25F058
:10C0D00001050562816921F0F00141EA041122F0B5
:10C0E0000A021A438161026230BD30B50B46144624
:10C0F000056A25F0100505628169026A21F4704124
:10C1000041EA043122F0A00242EA03128161026294
:10C1100030BD00002DE9F0410446514D0027514843
:10C12000877C4FF6FF7000EA07274E48C07C074324
:10C13000012F48D16888002845D1287D062842D1A2
:10C14000012068804748007D4749088008460088EC
:10C150004FF6FF7101EA0020434908804148407DC5
:10C160000988084340490880084602883D4916313D
:10C170003E48F4F75DF8002609E03D48006810B13C
:10C18000688800B906E0012001F0EAFA761CB6F5ED
:10C19000967FF2DB00BF3648006888B135480088DA
:10C1A000000A2075334800786075324832490268C9
:10C1B00004F11600F4F73CF800203049086002E072
:10C1C000002020756075002F48D12888002845D1AF
:10C1D000287D062842D1012028802248007D22495E
:10C1E0000880084600884FF6FF7101EA00201E49CA
:10C1F00008801C48407D098808431B490880084680
:10C200000288184916311E48F4F712F8002609E092
:10C210001A48006810B1288800B906E0012001F032
:10C220009FFA761CB6F5967FF2DB00BF13480068D4
:10C2300088B114480088000A20751248007860759B
:10C2400010481149026804F11600F3F7F1FF0020CD
:10C250000A49086002E0002020756075BDE8F081A1
:10C26000A238002000290020FA09002016380020FA
:10C270004C0300203C030020002B0020440300203E
:10C28000D0370020400300200025002070B58AB080
:10C2900005461D4E1D4C28216846F3F7E2FF617FDD
:10C2A000A07F41EA0020ADF80000207D062804D1DF
:10C2B000012217496846F5F757FA012214496846E2
:10C2C000F5F73CFABDF8000000126874BDF80000F4
:10C2D0002874BDF800004FF6FF71884203D0BDF806
:10C2E0000000A6F86600297C607F814209D1697C44
:10C2F000A07F814205D1207D062802D101200AB00D
:10C3000070BD0020FBE7000060370020A23800204D
:10C3100048F0070870B50546284602F07FFA044643
:10C3200014B1D4E90010884770BD70B505466C6A39
:10C330000020E085E0842046F8F702FE70BD70B56D
:10C3400006460025746A20684069C0F3C01594F859
:10C350003900212805D125B10020E084204600F0D5
:10C3600060F820684069C0F3801594F83A002228EC
:10C3700005D125B10020E085204600F032F8E06BC1
:10C3800040F01000E0632046F8F7DAFD70BD70B5AC
:10C3900005466C6A2868006800F02000B0B90020EB
:10C3A000E0852068C06820F480702168C86020683B
:10C3B000406920F00100216848612068406920F050
:10C3C000400021684861202084F83A002046F9F7AF
:10C3D00069F870BD70B50446656A2846F9F763F8D8
:10C3E00070BD0168C96821F490710268D16001686C
:10C3F000496921F0010102685161202180F83A1059
:10C40000704710B504462068C06820F040002168DD
:10C41000C860202084F839002046F9F7DAF80020B7
:10C4200010BD0168C96821F0C0010268D1602021F7
:10C4300080F83910704770B5044694F83A00222805
:10C4400047D1A068B0F5805F0CD1206950B90025B4
:10C45000A66A20684068C0F308003080A06A801C8B
:10C46000A06215E0A56A0026A068B0F5805F03D041
:10C47000A06828B9206918B920684068287004E0CD
:10C480002068406800F07F002870A06A401CA0620D
:10C49000E08D401E80B2E085C8B92068C06820F0F9
:10C4A00020002168C8602068C06820F4807021687E
:10C4B000C8602068406920F00100216848612020A0
:10C4C00084F83A002046F8F7EDFF002070BD002008
:10C4D000FCE70220FAE7000070B50446216809690C
:10C4E00021F44051E2681143226811612269A16878
:10C4F0001143626941EA02052168C96841F20C6290
:10C50000914329432268D1602168496921F440712F
:10C51000A2691143226851612D4A2168914202D1DA
:10C52000F7F7F8FF01E0F7F7E5FF00EBC00101EBDB
:10C53000001162689200B1FBF2F100EBC00202EB65
:10C54000001263689B00B2FBF3F26423B2FBF3F2C8
:10C5500002EBC20303EB0212A1EB8201322202EBD7
:10C5600001116422B1FBF2F101F0F00100EBC00215
:10C5700002EB001263689B00B2FBF3F26423B2FB90
:10C58000F3F201EB021200EBC00101EB0011636852
:10C590009B00B1FBF3F100EBC00303EB00136668F3
:10C5A000B600B3FBF6F36426B3FBF6F303EBC30666
:10C5B00006EB0313A1EB8301322303EB0111642388
:10C5C000B1FBF3F101F00F0111442268916070BDDD
:10C5D00000380140014691F8390021282DD18868A2
:10C5E000B0F5805F0BD1086948B90A6A1088C0F3BA
:10C5F00008000B685860086A801C086205E00B6A36
:10C60000581C086218780B685860C88C401E80B2AD
:10C61000C88420B1C88C4FF6FA7398420BD90868C9
:10C62000C06820F080000B68D8600868C06840F0DF
:10C6300040000B68D860002070470220FCE72DE91D
:10C64000F04104460D4617469846069E21E0701CB0
:10C65000F8B12EB1F7F764FDA0EB0800B04218D98D
:10C660002068C06820F4D0702168C86020684069E4
:10C6700020F0010021684861202084F8390084F806
:10C680003A0000BF002084F8380000BF0320BDE856
:10C69000F081206800682840A84201D1012000E014
:10C6A0000020B842D3D00020F1E7000008B51848B8
:10C6B00000680068C0F3001028B300BF002000909D
:10C6C00013480068006800901148006840680090B6
:10C6D00000BF00BF0E48F8F700FC0E480068406835
:10C6E000C0F580700C49086008460C4902680C4887
:10C6F000F3F79EFD4FF4807208490548F8F770FE85
:10C700000120084908600248F8F71CFC08BD000039
:10C71000B00B0020700C00204003002000240020FB
:10C72000002500204403002008B518480068006870
:10C73000C0F3001028B300BF002000901348006829
:10C7400000680090114800684068009000BF00BF7A
:10C750000E48F8F7C2FB0E4800684068C0F58070CC
:10C760000C49086008460C4902680C48F3F760FD64
:10C770004FF4807208490548F8F732FE0120084955
:10C7800008600248F8F7DEFB08BD0000F00B00204F
:10C79000F80C00203803002000270020002900208A
:10C7A0004803002008B51848F8F7CCFB1648006885
:10C7B0000068C0F3001028B300BF002000901248AA
:10C7C000006800680090104800684068009000BF52
:10C7D00000BF0D48F8F781FB0C4800684068C0F5C1
:10C7E00080700B49086008460A4902680A48F3F756
:10C7F0001FFD4FF4807207490348F8F7F1FD01204F
:10C800000649086008BD0000300C00203C0D0020E7
:10C810003C030020002A0020002B00204C030020B5
:10C8200000BFFEE730B58BB01F4D282101A8F3F7FC
:10C8300018FD002401221D4901A8F4F77FFFBDF86F
:10C8400004004FF6FF71884202D0BDF80400A880B2
:10C850000822174901A8F4F771FF00240FE001A88E
:10C8600030F814004FF6FF71884206D001A830F866
:10C87000141005F1140020F81410601CC4B22888AC
:10C88000A042ECDC00240AE005F1140030F81400AA
:10C8900008490988084407490880601CC4B22888F0
:10C8A000A042F1DC0BB030BD6037002028F0070853
:10C8B00000E007087C0300202DE9F0418046254D6B
:10C8C000002400270026688800283ED1287D0628FD
:10C8D00038D101206880AA7F2046611CCCB21E4955
:10C8E0000A5406222046611CCCB21B490A5400227D
:10C8F0002046611CCCB218490A5402222046611C11
:10C90000CCB215490A5400222046611CCCB212490F
:10C910000A5401222046611CCCB20F490A54C8199E
:10C920000621F9F7B5F8064632122046611CCCB252
:10C9300009490A542046611CCCB207490E540748E5
:10C94000048004E00020BDE8F0810020FBE7012026
:10C95000F9E70000A238002016380020FA0900206C
:10C960002DE9F0478146284D284F0024A046002697
:10C970006888002844D1287D06283ED1012068809F
:10C98000B888012800D100BFAA7F2046611CCCB224
:10C990001F490A5406222046611CCCB21C490A5485
:10C9A00000222046611CCCB219490A5410222046AC
:10C9B000611CCCB216490A54EA7F2046611CCCB2F5
:10C9C00013490A542020425D2046611CCCB2104914
:10C9D0000A5401EB08000621F9F75AF8064632120C
:10C9E0002046611CCCB20A490A542046611CCCB2D4
:10C9F00007490E540748048004E00020BDE8F08792
:10CA00000020FBE70120F9E7A23800206037002072
:10CA100016380020FA090020F0B58BB00646344FD6
:10CA2000344D282101A8F3F71CFC002400BF09E0C5
:10CA300004F1100005F10D01085C01A921F81400B2
:10CA4000601CC4B2287EA042F2DC287D062804D1F6
:10CA50000122294901A8F4F787FE0122264901A8ED
:10CA6000F4F76CFEBDF804003074BDF8040005282E
:10CA700002DABDF80400B880287D062805D1082216
:10CA80001E490DF10600F4F76FFE08221B490DF157
:10CA90000600F4F753FE002424E001A9601C31F8DD
:10CAA0001020103005F10D01085C824205D0287D70
:10CAB000062802D100200BB0F0BD01A9601C31F89E
:10CAC000100008280CDA601C31F8101007F114006F
:10CAD00020F8141001A9601C11F810101030315406
:10CAE000601CC4B2287EA042D7DC0120E3E700002E
:10CAF00060370020A238002028F0070800E007086F
:10CB000010B502467C4800BFD1B201EB011303EB24
:10CB1000430330F81330012B35D1002301EB01140E
:10CB200004EB440400EB4404A4F8523001EB01137D
:10CB300003EB430300EB4303B3F850305B1C01EB02
:10CB4000011404EB440400EB4404A4F8503001EB5E
:10CB5000011303EB430300EB4303B3F85030022B04
:10CB600011DB002301EB011404EB440400EB44044B
:10CB7000A4F85030012301EB011404EB440400EB52
:10CB80004404A4F8583001EB011303EB430330F8DD
:10CB90001330A3BB002301EB011404EB440400EBAE
:10CBA0004404A4F8503001EB011303EB430300EB02
:10CBB0004303B3F852305B1C01EB011404EB440453
:10CBC00000EB4404A4F8523001EB011303EB4303E0
:10CBD00000EB4303B3F85230022B10DB002301EBD0
:10CBE000011404EB440400EB4404A4F8523001EBBC
:10CBF000011404EB440400EB4404A4F8583001EBA6
:10CC0000011303EB430300EB43031B8D012B35D1D1
:10CC1000002301EB011404EB440400EB4404A4F8EA
:10CC2000563001EB011303EB430300EB4303B3F86E
:10CC300054305B1C01EB011404EB440400EB44048E
:10CC4000A4F8543001EB011303EB430300EB43035F
:10CC5000B3F85430022B11DB002301EB011404EB79
:10CC6000440400EB4404A4F85430012301EB011404
:10CC700004EB440400EB4404A4F85A3001EB011324
:10CC800003EB430300EB43031B8DA3BB002301EB2A
:10CC9000011404EB440400EB4404A4F8543001EB09
:10CCA000011303EB430300EB4303B3F856305B1C63
:10CCB00001EB011404EB440400EB4404A4F85630E7
:10CCC00001EB011303EB430300EB4303B3F85630CE
:10CCD000022B10DB002301EB011404EB440400EBF6
:10CCE0004404A4F8563001EB011404EB440400EBB7
:10CCF0004404A4F85A3010BDF63800200FB4084B95
:10CD000010B504A902AA039800F040F8044602A94D
:10CD1000002000F0DCF9204610BC5DF814FB000098
:10CD2000CFD0000802480068C0F30220704700001E
:10CD30000CED00E010B5002804DB0A07130E054ACD
:10CD4000135406E00A07140E034A00F00F031B1FDA
:10CD5000D45410BD00E400E018ED00E0EFF31180C2
:10CD60007047EFF305807047EFF31080704702E0E3
:10CD700008C8121F08C1002AFAD170477047002066
:10CD800001E001C1121F002AFBD170472DE9FF4FBE
:10CD90008BB088460546002606E025280BD0DDE945
:10CDA0000D1290476D1C761C28780028F5D10FB025
:10CDB0003046BDE8F08F0024A146A2460122AE49CC
:10CDC00000E0044315F8013F203B02FA03F008425B
:10CDD000F7D128782A2810D06FF02F022878A0F1F8
:10CDE0003001092915D809EB890102EB410144F012
:10CDF000020400EB01096D1CF0E758F8041B5FEA20
:10CE0000010903D544F40054C9F1000944F00204B7
:10CE10006D1C28782E2817D115F8010F44F0040452
:10CE20002A280ED06FF02F022878A0F130010929AE
:10CE30000AD80AEB8A0102EB410100EB010A6D1CE2
:10CE4000F2E758F804AB6D1C28786C280FD006DC8C
:10CE50004C2817D068280DD06A2814D104E0742813
:10CE600010D07A280FD10DE044F400140AE044F405
:10CE7000801401E044F440146978814202D104F541
:10CE800080146D1C6D1C2878692865D006DC00288C
:10CE90008DD0632827D0642806D15DE06E2808D0A5
:10CEA00073282AD0752877D0DDE90D129047761CBB
:10CEB000E0E0C4F30250022809D003280DD0D8F8CE
:10CEC000001004280DD00E6008F10408D2E0D8F854
:10CED0000010F217C1E90062F6E7D8F800100E80E2
:10CEE000F2E70E70F0E718F8041B8DF80010002030
:10CEF0008DF80100EB46012003E058F804BB4FF029
:10CF0000FF3061074FF0000701D40AE07F1C57454E
:10CF10000DDA8742FADB1BF807100029F6D106E08C
:10CF20007F1C8742FCDB1BF807100029F8D1DDE9E4
:10CF30000D23A9EB07008146214600F0B1F83044EB
:10CF4000C61904E0DDE90D121BF8010B90477F1EA6
:10CF5000F8D22146484688E058F8040BC4F3025141
:10CF60004FF00A0B032900D100B2042900D140B2CE
:10CF7000002802DA40422D2102E0210505D52B21AF
:10CF80008DF82410012104E006E0E10710D02021F3
:10CF9000F6E708AF089113E058F8040BC4F3025108
:10CFA0004FF00A0B032900D180B2042900D1C0B28E
:10CFB0000021EEE75946F3F76DFA303107F8011D0D
:10CFC0000028F7D1ADEB070000F1200B600702D578
:10CFD00024F4803401E04FF0010ADA4502DDAAEBC7
:10CFE0000B0000E00020824600EB0B010898014492
:10CFF000A9EB01000A90E00306D4DDE90D232146E8
:10D000000A9800F04DF806444FF0000908E009A91D
:10D0100011F80900DDE90D12904709F10109761CAC
:10D0200008998945F3DBE0030CD5DDE90D232146A2
:10D030000A9800F035F8064404E0DDE90D123020CE
:10D040009047761CBAF10001AAF1010AF5DC05E06F
:10D05000DDE90D1217F8010B9047761CBBF10001BA
:10D06000ABF1010BF4DC0A982146DDE90D2300F059
:10D0700005F806446D1C97E6092801002DE9F041EA
:10D08000044600251E461746880404D405E03946A8
:10D090002020B0476D1C641EF9D52846BDE8F081FC
:10D0A0002DE9F041044600251E469046C80301D5EF
:10D0B000302700E02027880404D505E041463846A3
:10D0C000B0476D1C641EF9D52846BDE8F0810A689A
:10D0D000531C0B6010707047C200002100BF01E0BC
:10D0E00000BF491C9142FBD3704700001FB50020D0
:10D0F0000090019002900390F7F724F8F3F7FCFEFC
:10D10000F9F738F8FFF78EFBF3F7FEFCFEF72CFF7C
:10D11000F8F72CFEF8F7FAFDF8F790FFF8F772FF32
:10D12000F8F7B8FFF8F7E2FFF8F7C2FDF8F7D0FD1F
:10D13000F8F7F8FEF8F730FFF8F7B2FE01225103D6
:10D14000EF48F6F7E7FF01221103ED48F6F7E2FF9B
:10D1500001221021EB48F6F7DDFF4FF480600090CC
:10D16000002001900290022003906946E648F6F7FD
:10D170001FFE00224FF40051E148F6F7CBFF0022DA
:10D180004FF40051DE48F6F7C5FF00224FF48051FE
:10D19000DB48F6F7BFFF00221021DA48F6F7BAFFA6
:10D1A0000220F6F71FFD2021D848F3F75AF8052290
:10D1B000D7A1D648FFF7A2FD0446A2B24FF496735A
:10D1C000D249D848F8F770F901225103CC48F6F754
:10D1D000A1FF01221103CA48F6F79CFF012210218A
:10D1E000C848F6F797FF00F007FBCF4800F0A2FB16
:10D1F000CE490860CE4800F09DFBCE490860CE487D
:10D2000000F098FBCD490860CD4800F093FBCD4974
:10D210000860CD4800F08EFBCC490860CC4800F097
:10D2200089FBCC490860CC4800F084FBCB490860FE
:10D23000CB4800F07FFBCB490860CB4800F07AFB7D
:10D24000CA490860CA4800F075FBCA490860CA4864
:10D2500000F070FBC9490860C94800F06BFBC94980
:10D260000860C94A0121084600F0CCFBC7490860A4
:10D27000C74A0121084600F0C5FBC6490860C64AF6
:10D280000121084600F0BEFBC4490860C44A0121E0
:10D29000084600F0B7FBC3490860C34A01210846AD
:10D2A00000F0B0FBC1490860C14A0121084600F006
:10D2B000A9FBC0490860C04A0121084600F0A2FB52
:10D2C000BE490860BE4A0121084600F09BFBBD49EB
:10D2D0000860BD4A0221084600F094FBBB49086083
:10D2E000BB4A0221084600F08DFBBA490860BA4AE1
:10D2F0000221084600F086FBB8490860B84A0221BE
:10D30000084600F07FFBB7490860B74B00220121B7
:10D31000B64800F05BFCB6490860B64B002201211C
:10D32000B54800F053FCB5490860B54B0022012117
:10D33000B44800F04BFCB4490860B44B0022012112
:10D34000B34800F043FCB3490860B34B002201210D
:10D35000B24800F03BFCB2490860B24B0022012108
:10D36000B14800F033FCB1490860B14B0022012103
:10D37000B04800F02BFCB0490860B04B00220121FE
:10D38000AF4800F023FCAF490860AF4B00220121F9
:10D39000AE4800F01BFCAE490860AE4B00220121F4
:10D3A000AD4800F013FCAD490860AD4A02211020E1
:10D3B00000F064FAAB490860AB4A0221102000F08B
:10D3C0005DFAAA490860AA4A0221102000F056FA24
:10D3D000A8490860A84A0221102000F04FFAA74986
:10D3E0000860A74A0221102000F048FAA549086009
:10D3F000A54A0221102000F041FAA4490860A44A7D
:10D400000021A44800F074FBA3490860A34A00214E
:10D41000A34800F06DFBA3490860A34A0021A3487C
:10D4200000F066FBA2490860A24A0021A24800F071
:10D430005FFBA2490860A24A0021A24800F058FB05
:10D44000A1490860A14A0021A14800F051FBA1496F
:10D450000860A14A0021A14800F04AFBA0490860E9
:10D46000A04A0021A04800F043FBA0490860A04A60
:10D470000021A04800F03CFB9F4908609F4A002122
:10D480009F4800F035FB9F4908609F4A00219F4854
:10D4900000F02EFB9E4908609E4A00219E4800F045
:10D4A00027FB9E4908609E4800F076F99D49086078
:10D4B0009D4800F071F99D4908609D4800F06CF9A5
:10D4C0009C4908609C4800F067F99C4908609C48AA
:10D4D00000F062F99B4908609B4800F05DF99B49A8
:10D4E00008609B4800F058F99A4908609A4800F093
:10D4F00053F99A49086000F09FF900BFFEE7000069
:10D50000000C01400008014000100140800D002087
:10D510007379737974656D2072657365742E2E2E20
:10D5200025356400F00B002074020108740200200D
:10D530008402010878020020940201087C02002085
:10D54000A402010880020020B40201088402002025
:10D55000C402010888020020D40201088C020020C5
:10D56000E402010890020020F40201089402002065
:10D570000403010898020020140301089C02002003
:10D5800024030108A002002034030108A4020020A3
:10D5900044030108A802002054030108AC02002043
:10D5A00064030108B002002074030108B4020020E3
:10D5B00084030108B802002094030108BC02002083
:10D5C000A4030108C0020020B4030108C402002023
:10D5D000C4030108C8020020D4030108CC020020C3
:10D5E000E4030108D0020020D4010108E50E000880
:10D5F0004C020020E4010108E90E0008500200205E
:10D60000F4010108EB0E0008540200200402010896
:10D61000ED0E00085802002014020108EF0E000869
:10D620005C02002024020108F10E000860020020C4
:10D6300034020108F30E00086402002044020108CD
:10D64000F50E00086802002054020108F70E0008D9
:10D650006C02002064020108E70E0008700200203E
:10D6600044010108340200205C0101083802002056
:10D67000740101083C0200208C01010840020020D6
:10D68000A401010844020020BC0101084802002056
:10D6900094FF000869A1000804020020B8FF0008F8
:10D6A00075A1000808020020DCFF000855A800084A
:10D6B0000C0200200000010881B7000810020020C1
:10D6C0002400010805BE00081402002048000108DB
:10D6D000C5BE0008180200206C000108CFBE00087B
:10D6E0001C02002090000108D9BE00082002002082
:10D6F000B4000108E3BE000824020020D80001089D
:10D70000EDBE000828020020FC000108F7BE00085A
:10D710002C0200202001010801BF00083002002077
:10D72000F4030108D402002004040108D8020020F8
:10D7300014040108DC02002024040108E002002097
:10D7400034040108E402002044040108E802002037
:10D7500054040108EC02002064040108F0020020D7
:10D7600070B50546FFF7FDFA48B9FFF7FDFA30B985
:10D7700008480068022805D1FFF7F0FA10B16FF0F1
:10D78000050404E0002415B1284601F023FA2046E0
:10D7900070BD0000600A002070B504460026FFF747
:10D7A000E0FA00BBFFF7E0FAE8B912480068022887
:10D7B00002D1FFF7D3FAB0B94FF0FF3564B1A068DA
:10D7C00020B1E068202801D3012506E0A06820B937
:10D7D000E06810B9002500E00025012D04D1A06803
:10D7E00001F02FFB064603E015B901F01BFB0646CE
:10D7F000304670BD600A002010B5FFF7B2FA48B994
:10D80000FFF7B2FA30B90B480068022805D1FFF7DC
:10D81000A5FA10B16FF0050409E00648006820B9C8
:10D82000012004490860002401E04FF0FF34204645
:10D8300010BD0000600A002010B5FFF792FA48B949
:10D84000FFF792FA30B90C480068022805D1FFF7BB
:10D8500085FA10B16FF005040CE007480068012854
:10D8600006D102200449086001F030FA002401E0EA
:10D870004FF0FF34204610BD600A00202DE9F84328
:10D8800005460E4614464FF00009FFF76AFA0028D5
:10D890004BD1FFF769FA002847D1254800680228D4
:10D8A00003D1FFF75BFA00283FD1002D3DD0002EB9
:10D8B0003BD04FF0FF37BCB1A06858B1E0685028AA
:10D8C00008D3206930B105FB06F06169814201D3BC
:10D8D00001270AE0A06840B9E06830B9206920B9A2
:10D8E000606910B9002700E00027012F09D100204E
:10D8F000009031462846A368226901F000FC814669
:10D9000006E02FB900223146284601F0C9FB8146C6
:10D91000B9F1000F09D014B1D4F8008001E04FF044
:10D9200000084146484601F0E7F84846BDE8F8835C
:10D93000600A00202DE9F04704460026FFF711FA9F
:10D94000002859D1FFF710FA002855D12C4800685B
:10D95000022803D1FFF702FA00284DD10CB1676805
:10D9600000E0002707F0010008B1012500E00025D4
:10D9700007F0080008283FD04FF0FF3874B1A068C6
:10D9800028B1E068502802D34FF0010808E0A068F1
:10D9900030B9E06820B94FF0000801E04FF000080E
:10D9A000B8F1010F0CD12DB10420A16801F063FB87
:10D9B000064612E00120A16801F05DFB06460CE07E
:10D9C000B8F1000F09D125B1042001F043FB064650
:10D9D00003E0012001F03EFB06464EB114B1D4F83D
:10D9E000009001E04FF000094946304601F084F80C
:10D9F00016B10DB146F001063046BDE8F0870000D3
:10DA0000600A00202DE9F84305460F4614464FF002
:10DA10000008FFF7A6F9002864D1FFF7A5F9002850
:10DA200060D132480068022803D1FFF797F9002837
:10DA300058D1002D56D0AF4254D84FF0FF3664B1C4
:10DA4000A06820B1E068502801D3012606E0A06854
:10DA500020B9E06810B9002600E00026701C70B301
:10DA6000012D23D1012E09D103200090002211465F
:10DA70000120A36801F043FB804605E0032200215A
:10DA8000012001F00DFB8046B8F1000F1DD0E7B179
:10DA900000231A461946404601F0ECFB012814D039
:10DAA000404601F03FF84FF000080EE0012E07D18C
:10DAB00039462846A26801F09BFA804605E011E04D
:10DAC0003946284601F066FA8046B8F1000F09D0C1
:10DAD00014B1D4F8009001E04FF0000949464046E7
:10DAE00001F00AF84046BDE8F8830000600A002013
:10DAF0002DE9F04786B08046894614460020049000
:10DB0000FFF72FF900285DD1FFF72EF9002859D132
:10DB10002D480068022803D1FFF720F9002851D1D1
:10DB2000B8F1000F4ED080261825002005900DF189
:10DB3000140A471E44B3206808B1D4F800A0A069B5
:10DB400000B1A5692DB1382D03D8207900F001006E
:10DB500018B1002006B0BDE8F087606908B16069BF
:10DB60008608A06840B1E0685C2805D3206918B138
:10DB7000606908B1012708E0A06830B9E06820B901
:10DB8000206910B9002700E00027012F0CD121697E
:10DB9000A0684B463246CDE90051029051464046BE
:10DBA00001F0F2FD04900DE067B904A8B2B24B4653
:10DBB0005146CDE90050404601F0B4FD012801D0A6
:10DBC000002004900498C5E7600A00202DE9FE4F6C
:10DBD0000646894692461C4600200290FFF7C1F88F
:10DBE000002851D1FFF7C0F800284DD1284800681F
:10DBF000022803D1FFF7B2F8002845D1002E43D008
:10DC0000082000F06DFD0546002D3DD02E60C5F8C2
:10DC100004A0B9F1000F01D1002700E001274FF067
:10DC2000FF384FF0000B94B1206808B1D4F800B071
:10DC3000A06828B1E068302802D34FF0010808E05E
:10DC4000A06830B9E06820B94FF0000801E04FF05B
:10DC50000008B8F1010F0BD10E49A0682B463A46D7
:10DC6000CDE900100121584601F0DDFF02900BE0E4
:10DC7000B8F1000F08D107482B463A460121009021
:10DC8000584601F0B5FF02900298BDE8FE8F0000F3
:10DC9000600A002015C300082DE9F04105460E4634
:10DCA0001948076800201949096881F85A0017487F
:10DCB0000068001D00F0DAFD681C38B936B1134861
:10DCC0000168091D124800F028FE1AE07C190F486F
:10DCD00000684460BC4207D20C480168091D0D4829
:10DCE000006800F000FE0CE008480168091D0A48C1
:10DCF000006800F0F8FD09480068844201D2074836
:10DD00000460BDE8F0810000240A0020100A002011
:10DD1000EC5D0020180A0020140A0020400A0020B0
:10DD200010B5044600F006FE24480068401C234954
:10DD300008602348006840B921480460084600682C
:10DD400001280DD100F030FA0AE01E48006838B909
:10DD50001B480068C06AE16A884201D8184804601C
:10DD600019480068401C184908600846006860644B
:10DD70001649E06A0968884202D91449E06A0860D5
:10DD8000E16A01EB8101124A02EB8100211D00F0E2
:10DD9000C4FD00F0F9FD0B48006868B10848006850
:10DDA000C06AE16A884207D24FF080500949086092
:10DDB000BFF34F8FBFF36F8F10BD0000200A00200C
:10DDC000100A00202C0A00203C0A0020280A00200B
:10DDD0003C59002004ED00E008B500F0ABFD12480E
:10DDE0000068E8B9114800F06EFD114800F06BFDC5
:10DDF0000E48104908600E480F49086000200F4B7C
:10DE00000F4A102100900A2001F079F906490860B4
:10DE10000846006820B10BA10348006800F06CFEC2
:10DE200000F0B2FD08BD0000540A0020005E002092
:10DE3000145E00204C0A0020500A0020285E0020BA
:10DE4000785E0020546D72510000000010B516E09D
:10DE500000F070FD0C48C068C468201D00F006FD8D
:10DE60000A480068401E0949086009480068401EC9
:10DE70000749086000F088FD204600F05EF804487D
:10DE800000680028E4D110BDD85D0020200A0020E1
:10DE90001C0A002070B504460D46206C70B1216C40
:10DEA000E0680844E0606168E068884201D3206867
:10DEB000E0602846226CE168F2F7BAF970BD2DE9FE
:10DEC000F04104460F4615464FF00008A66B206C43
:10DED00040B9206860BB606801F06AFD80460020A0
:10DEE000606025E07DB93946226CA068F2F7A0F9A0
:10DEF000216CA0680844A060D4E90110884217D3BF
:10DF00002068A06014E03946226CE068F2F790F9CE
:10DF1000216CE068401AE0602168E068884203D222
:10DF2000216C6068401AE060022D01D106B1761EB6
:10DF3000701CA0634046BDE8F08110B5044694F81B
:10DF4000590030B9206B00F03DFD204600F03AFD4D
:10DF50001AE094F85900012803D1204600F032FD60
:10DF600012E094F85900022801D1012000E00020BD
:10DF700050B900BF502080F31188BFF34F8FBFF31B
:10DF80006F8F00BF00BFFEE710BD00000146084ACA
:10DF9000126812680AB9012200E000220A600A68C9
:10DFA00022B9034A1268D268106800E00020704766
:10DFB0004C0A002030B54FF48043174800F00704A6
:10DFC0002CB1C01D20F00700134C041B1B1B024684
:10DFD000124C22600024114D6C60D018083820F0DB
:10DFE00007000F4C206000240D4D2D686C600C4D17
:10DFF0002D682C601146441A4C60094C24680C6052
:10E00000084D4C682C60084D4C682C604FF0004463
:10E01000064D2C6030BD0000D0650020640A002051
:10E020006C0A0020740A0020700A0020780A002080
:10E0300000BFFFF70BFF07480068012807D94FF022
:10E04000805005490860BFF34F8FBFF36F8F00F01A
:10E0500039FCEEE73C59002004ED00E010B5044621
:10E060004CB1002060602060E06000231A46194631
:10E07000204601F0FFF810BD2DE9F04106460D469F
:10E0800017469846069C0DB9246000E02760E663B9
:10E0900025640121204601F0A1F884F84C80BDE8F8
:10E0A000F0812DE9F05F82460F4690469B460A9E1E
:10E0B0000C9C4FEA8801A522206BF2F7CBF8A8F15F
:10E0C0000100216B01EB800929F0070909F0070025
:10E0D00008B9012000E0002050B900BF502080F3B3
:10E0E0001188BFF34F8FBFF36F8F00BF00BFFEE7F4
:10E0F000002507E0795D04F134004155785D00B9F1
:10E1000002E06D1C102DF5D300BF00214320015506
:10E11000382E00D33726E662E66400202065201DF5
:10E1200000F0DEFB04F1180000F0DAFB2461C6F118
:10E130003800A06164620020606584F8580084F8AB
:10E140005A005A465146484600F07EFB20600B9824
:10E1500008B10B980460BDE8F09F2DE9F047064632
:10E160000D4617469846DDE908940DB1012000E000
:10E17000002050B900BF502080F31188BFF34F8FAB
:10E18000BFF36F8F00BF00BFFEE75CB1FFF724FE57
:10E190002660A561E761C4F82080C4F82490201DA2
:10E1A00000F09EFBBDE8F08710B5002407E004EB0B
:10E1B00084010F4A02EB810000F085FB641C382CBF
:10E1C000F5D30C4800F07FFB0B4800F07CFB0B48BC
:10E1D00000F079FB0A4800F076FB0A4800F073FB78
:10E1E00004480949086004480849086010BD000057
:10E1F0003C5900209C5D0020B05D0020C45D0020E3
:10E20000D85D0020EC5D0020140A0020180A0020D0
:10E2100010B50146164800E0006803688B42FBD346
:10E220000246436813448B4204D143684C6823443C
:10E23000436001460A464B6813440468A34211D167
:10E240000C4C03682468A34208D04B6804686468D7
:10E2500023444B6003681B680B6005E0054B1B689B
:10E260000B6001E003680B60884200D0016010BDC4
:10E27000640A00206C0A00202DE9F04104460D4696
:10E2800016461F464FF0000865602461B5420CD861
:10E29000F01BA169884202D34FF0010811E0211D53
:10E2A0000948006800F01FFB0BE0BE4204D2BD42EB
:10E2B00002D34FF0010804E0211D0448006800F07B
:10E2C00012FB4046BDE8F081500A00204C0A0020B5
:10E2D00070B5054600F02EFBA86B08B9012400E0DC
:10E2E000002400F051FB204670BD70B5054600F0DB
:10E2F00021FBA86BE96B884201D1012400E00024D6
:10E3000000F042FB204670BDF8B505460F461648A2
:10E310000068C068C468201D00F0A8FAE069012800
:10E320001DD1A06941192B463A462046FFF7A4FFAC
:10E33000A8B1002003462A4601460090204601F07D
:10E34000E7FC064656B900BF502080F31188BFF3A2
:10E350004F8FBFF36F8F00BF00BFFEE700BF2046A7
:10E36000616A8847F8BD00004C0A0020F0B587B00C
:10E3700082E00398002811DA04AE56B900BF50209D
:10E3800080F31188BFF34F8FBFF36F8F00BF00BFC3
:10E39000FEE7D6E90020B168904700BF0398002847
:10E3A0006ADB059C606908B9012000E0002010B913
:10E3B000201D00F05BFA02A800F0C0F805460398A3
:10E3C0000A2857D2DFE800F009050731334F060865
:10E3D000323400BF00BF00BF00BF0498A26981189B
:10E3E00003462A462046FFF747FFE8B12046616A08
:10E3F0008847E069012817D1002000900498A1699E
:10E40000421800231946204601F082FC074657B9FE
:10E4100000BF502080F31188BFF34F8FBFF36F8F81
:10E4200000BF00BFFEE700BF25E000BF23E000BF44
:10E430000498A061A06908B1012000E0002050B953
:10E4400000BF502080F31188BFF34F8FBFF36F8F51
:10E4500000BF00BFFEE7A06941192B462A462046AF
:10E46000FFF70AFF07E094F82C0010B9204600F0EF
:10E47000A9FA00E000BF00BF002203A90448006819
:10E4800001F048F800287FF474AF07B0F0BD000039
:10E49000540A0020F8B505460C4600F073FC6846A7
:10E4A00000F04CF80646009820BB44B9B54206D8A7
:10E4B00001F01CFB31462846FFF726FF1CE03CB16B
:10E4C0000E480068006808B9012000E000200446FA
:10E4D000A91B22460A48006800F056FB01F006FB23
:10E4E00050B94FF0805007490860BFF34F8FBFF31A
:10E4F0006F8F01E001F0FAFAF8BD0000500A002029
:10E50000540A002004ED00E00A490968096809B9C5
:10E51000012100E0002121B14FF0FF31064A1160D6
:10E5200006E004490968C968C868034A416811607F
:10E5300070470000140A0020400A002070B504460D
:10E5400001F08EF9054607480068854204D200F0C4
:10E550000BF80120206001E00020206001480560E8
:10E56000284670BD5C0A00202DE9F84332E02448BB
:10E570000068C068056822480068C068C468201D3B
:10E5800000F074F92046616A8847E069012821D1CA
:10E59000A0694619AE4207D966602461211D18485A
:10E5A000006800F0A0F915E0002003462A46014665
:10E5B0000090204601F0ACFB074657B900BF502041
:10E5C00080F31188BFF34F8FBFF36F8F00BF00BF81
:10E5D000FEE700BF0A480068006808B9012000E0B3
:10E5E00000200028C3D00648D0F800800548006805
:10E5F000034908600348C0F80080BDE8F8830000C4
:10E600004C0A0020500A00200E480068401C08B93F
:10E61000012000E0002050B900BF502080F3118895
:10E62000BFF34F8FBFF36F8F00BF00BFFEE700BF88
:10E63000502080F31188BFF34F8FBFF36F8F00BF5F
:10E6400000BFFEE77C0A002008B500BF6846FFF760
:10E650009DFC044620460099FFF71CFFFFF786FE4D
:10E66000F4E770B5044600F065F994F9455010E000
:10E67000606A08B9012000E0002038B904F12400E4
:10E6800001F0E8F918B100F0DFFA00E003E0681EDD
:10E6900045B2002DECDC00BFFF2084F8450000F0FF
:10E6A00073F900F047F994F9445010E0206908B973
:10E6B000012000E0002048B904F1100001F0CAF97F
:10E6C00008B100F0C1FA681E45B200E001E0002D7B
:10E6D000ECDC00BFFF2084F8440000F055F970BD69
:10E6E0002DE9F04104464FF0000800F04BFB46488E
:10E6F000006808B9FFF75EFC444800682040002825
:10E700006BD1D4B1083404F00700B0B104F00700B5
:10E71000C0F10800044404F0070008B9012000E03B
:10E72000002050B900BF502080F31188BFF34F8FF5
:10E73000BFF36F8F00BF00BFFEE7002C4DD0344801
:10E740000068844249D8334E3046056801E02E46C1
:10E750002D686868A04202D228680028F7D12A48AC
:10E760000068854239D0306800F1080828683060B8
:10E770006868001B102819D92F1907F0070008B97D
:10E78000012000E0002050B900BF502080F3118824
:10E79000BFF34F8FBFF36F8F00BF00BFFEE7686806
:10E7A000001B78606C603846FFF732FD18496868D6
:10E7B0000968081A16490860084600681649096879
:10E7C000884203D212480068134908600F496868FC
:10E7D0000968084368600020286001F087F908F0A4
:10E7E000070008B9012000E0002050B900BF502008
:10E7F00080F31188BFF34F8FBFF36F8F00BF00BF4F
:10E80000FEE74046BDE8F0816C0A0020780A00204F
:10E81000700A0020640A0020740A002070B50446C3
:10E82000254654B900BF502080F31188BFF34F8FA5
:10E83000BFF36F8F00BF00BFFEE700F07BF82E6ACA
:10E8400000F0A2F8304670BD001F4FF080730360E7
:10E85000001F21F001030360001F034B0360143805
:10E86000026020387047000009E6000801460A6986
:10E87000D1E901309860D1E90103586050688842BD
:10E8800001D188685060002008611068401E106047
:10E8900010687047034B0360034B0B6080231360C9
:10E8A00070470000185F0020745F0020034B036076
:10E8B000034B0B604FF4807313607047746100204A
:10E8C000D0610020704700F1080141604FF0FF3136
:10E8D000816000F10801C1600161002101607047A1
:10E8E00000210161704710B502460B685C1C0CB931
:10E8F000106907E002F1080000E0406844682468FD
:10E900009C42FAD944684C604C68A16088604160C0
:10E910000A611468641C146010BD42684A60936800
:10E920008B60936859609160086103685B1C0360A9
:10E930007047000000BF502080F31188BFF34F8F55
:10E94000BFF36F8F00BF0E480068401C0C49086081
:10E9500008460068012812D10A480068C0B208B908
:10E96000012000E0002050B900BF502080F3118842
:10E97000BFF34F8FBFF36F8F00BF00BFFEE770473D
:10E980007C0A002004ED00E00D48006850B900BF8B
:10E99000502080F31188BFF34F8FBFF36F8F00BFFC
:10E9A00000BFFEE706480068401E054908600846AB
:10E9B000006820B9002080F3118800BF00BF7047B5
:10E9C0007C0A002070B506463546002E3FD0083D33
:10E9D0002C461F4960680968084008B1012000E022
:10E9E000002050B900BF502080F31188BFF34F8F33
:10E9F000BFF36F8F00BF00BFFEE7206808B901209A
:10EA000000E0002050B900BF502080F31188BFF310
:10EA10004F8FBFF36F8F00BF00BFFEE70C496068E8
:10EA20000968084098B1206888B909496068096890
:10EA30008843606000F0A6F90649606809680844E8
:10EA4000044908602046FFF7E3FB01F04FF870BD72
:10EA5000780A0020700A002000204FF0E0210861B1
:10EA60008861064800684FF47A71B0FBF1F0401EEF
:10EA70004FF0E0214861072008617047000A00203C
:10EA800070B5F1F7A9FB0446102C16D304F1E02071
:10EA900090F8F05315480078854201DB012000E032
:10EAA000002050B900BF502080F31188BFF34F8F72
:10EAB000BFF36F8F00BF00BFFEE70D48006800F492
:10EAC000E0600C490968884201D8012000E000207C
:10EAD00050B900BF502080F31188BFF34F8FBFF3B0
:10EAE0006F8F00BF00BFFEE770BD0000800A0020EE
:10EAF0000CED00E0840A0020024600200BE0084BE9
:10EB000053F8303033B9064B43F8301003EBC003F1
:10EB10005A6002E0401C0828F1D300BF7047000093
:10EB2000FC58002070B50446254655B900BF50205A
:10EB300080F31188BFF34F8FBFF36F8F00BF00BF0B
:10EB4000FEE7284600F008F895F8460010B9284678
:10EB5000FFF738FF70BD0000014600200EE0094AB3
:10EB600002EBC00252688A4207D10022054B43F8EB
:10EB7000302003EBC0035A6002E0401C0828EED3AB
:10EB800000BF7047FC5800202DE9F04105460E46B5
:10EB900017462C46FFF7CEFE94F94400401C10B9EE
:10EBA000002084F8440094F94500401C10B900206E
:10EBB00084F84500FFF7E8FEA06B28B93A463146D5
:10EBC00004F1240000F062F82046FFF74AFDBDE89A
:10EBD000F081000070B504460025D4B112480068E9
:10EBE00008B9012000E0002050B900BF502080F398
:10EBF0001188BFF34F8FBFF36F8F00BF00BFFEE7D9
:10EC000000F0C0F800212046FFF746F800F06EFF44
:10EC100005463DB94FF0805004490860BFF34F8F5F
:10EC2000BFF36F8F70BD0000480A002004ED00E0C4
:10EC300003490968016003490968416070470000A1
:10EC4000380A0020240A002001200149086070478A
:10EC5000340A002070B504460D4654B900BF502058
:10EC600080F31188BFF34F8FBFF36F8F00BF00BFDA
:10EC7000FEE70548016818312046FFF734FE012100
:10EC80002846FFF709F870BD100A002070B5054648
:10EC90000E46144655B900BF502080F31188BFF3CB
:10ECA0004F8FBFF36F8F00BF00BFFEE706480168BC
:10ECB00018312846FFF731FE0CB14FF0FF362146E0
:10ECC0003046FEF7E9FF70BD100A002010B586B08F
:10ECD00000200590049003AA04A905A8FFF7DAFD17
:10ECE0000022DDE904101346CDE9002102901EA1A7
:10ECF0001F48039A00F048FD1E4908600846006856
:10ED000008B1012400E00024012C02D100F0C4FF6E
:10ED10000446012C15D100BF502080F31188BFF3A9
:10ED20004F8FBFF36F8F00BF4FF0FF301249086065
:10ED300001201249086000201149086000F0AEF877
:10ED400010E0601C08B1012000E0002050B900BFB5
:10ED5000502080F31188BFF34F8FBFF36F8F00BF38
:10ED600000BFFEE706B010BD49444C45000000005E
:10ED700031E00008440A0020400A00202C0A00204C
:10ED8000240A002002480068401C014908607047BE
:10ED9000480A00201E48006818B101201D4908607B
:10EDA00034E000201B4908601B4801680CE051B9A1
:10EDB00000BF502080F31188BFF34F8FBFF36F8FD8
:10EDC00000BF00BFFEE7491E01EB8100134A52F865
:10EDD000200008B9012000E000200028E7D101EB65
:10EDE00081020E4B03EB820042685268426000F1E0
:10EDF00008024368934202D1426852684260426806
:10EE0000D268074B1A600448016000BF70470000D9
:10EE1000480A0020340A0020280A00203C5900201B
:10EE2000100A002010B52020FFF75AFC044634B128
:10EE300000202060201DFFF746FD0020207720469F
:10EE400010BD38B5054655B900BF502080F3118874
:10EE5000BFF34F8FBFF36F8F00BF00BFFEE72020CF
:10EE600000900098202801D1012000E0002050B936
:10EE700000BF502080F31188BFF34F8FBFF36F8F17
:10EE800000BF00BFFEE72C4634B100202060201DEB
:10EE9000FFF719FD01202077204638BD1CB5384901
:10EEA000084600780190FF200A4610700846007856
:10EEB00000909DF8000000F0F0009DF800209042C6
:10EEC00001D1012000E0002050B900BF502080F3A4
:10EED0001188BFF34F8FBFF36F8F00BF00BFFEE7F6
:10EEE0009DF8000000F05000264A10700720264AC6
:10EEF000106009E024480068401E234A10609DF815
:10EF000000004006000E00909DF8000000F0800018
:10EF10008028EFD01C480068C0F10700042801D108
:10EF2000012000E0002050B900BF502080F311887C
:10EF3000BFF34F8FBFF36F8F00BF00BFFEE71248D4
:10EF400000680002104A10601046008800F4E0607B
:10EF500010600B4A019810700C48006840F4700073
:10EF60000A4908600846006840F070400860FFF7F2
:10EF700073FD002006490860F1F7F8F800201CBD79
:10EF800000E400E0800A0020840A002020ED00E078
:10EF90007C0A002070B505460E460DB1012000E048
:10EFA000002050B900BF502080F31188BFF34F8F6D
:10EFB000BFF36F8F00BF00BFFEE7AE4201D8012054
:10EFC00000E0002050B900BF502080F31188BFF34B
:10EFD0004F8FBFF36F8F00BF00BFFEE702220021FB
:10EFE000284600F05DF8044604B1A663204670BDD3
:10EFF000F8B505460E4617460DB1012000E0002089
:10F0000050B900BF502080F31188BFF34F8FBFF37A
:10F010006F8F00BF00BFFEE7AE4201D8012000E0C5
:10F02000002050B900BF502080F31188BFF34F8FEC
:10F03000BFF36F8F00BF00BFFEE702203B460022F8
:10F0400011460090284600F05AF8044604B1A66321
:10F050002046F8BD2DE9F04104460126002722464E
:10F060000021012000F01CF805462846FEF7F6FFB7
:10F070002846BDE8F0812DE9F84304460D460127F6
:10F080004FF000082B46002211460120009400F0AA
:10F0900036F806463046FEF7E1FF3046BDE8F88315
:10F0A0002DE9F84305460E4690460DB1012000E0DB
:10F0B000002050B900BF502080F31188BFF34F8F5C
:10F0C000BFF36F8F00BF00BFFEE70EB9002701E05E
:10F0D00005FB06F707F15000FFF702FB04465CB1A1
:10F0E00004F15009002084F8460043464A46314660
:10F0F00028460094FEF7C0FF2046BDE8F8832DE9BE
:10F10000F84380460E4617461D46DDF82090B8F1BC
:10F11000000F01D0012000E0002050B900BF5020B6
:10F1200080F31188BFF34F8FBFF36F8F00BF00BF15
:10F13000FEE70DB1012000E0002050B900BF5020D3
:10F1400080F31188BFF34F8FBFF36F8F00BF00BFF5
:10F15000FEE707B10EB1012000E0002050B900BF6A
:10F16000502080F31188BFF34F8FBFF36F8F00BF24
:10F1700000BFFEE707B90EB9012000E0002050B93A
:10F1800000BF502080F31188BFF34F8FBFF36F8F04
:10F1900000BF00BFFEE7502000900098502801D12A
:10F1A000012000E0002050B900BF502080F31188FA
:10F1B000BFF34F8FBFF36F8F00BF00BFFEE72C463A
:10F1C0004CB1012084F846004B463A463146404651
:10F1D0000094FEF751FF2046BDE8F88370B5054660
:10F1E0000E462C4654B900BF502080F31188BFF35F
:10F1F0004F8FBFF36F8F00BF00BFFEE7FFF79AFB93
:10F20000D4E90F12206801FB020060600020A063B7
:10F210002068A060E06B401E226C216800FB021099
:10F22000E060FF2084F8440084F845009EB920691E
:10F2300008B9012000E00020A8B904F1100000F096
:10F2400009FC80B14FF0805009490860BFF34F8F2F
:10F25000BFF36F8F07E004F11000FFF734FB04F1F8
:10F260002400FFF730FBFFF78FFB012070BD00008B
:10F2700004ED00E02DE9FF4383B0064688461D46B5
:10F280004FF00009344654B900BF502080F3118874
:10F29000BFF34F8FBFF36F8F00BF00BFFEE7B8F122
:10F2A000000F01D1206C08B9012000E0002050B906
:10F2B00000BF502080F31188BFF34F8FBFF36F8FD3
:10F2C00000BF00BFFEE7022D02D1E06B012801D193
:10F2D000012000E0002050B900BF502080F31188C9
:10F2E000BFF34F8FBFF36F8F00BF00BFFEE700F08B
:10F2F000A7FA08B9059808B9012000E0002050B924
:10F3000000BF502080F31188BFF34F8FBFF36F8F82
:10F3100000BF00BFFEE700BFFFF70CFBA06BE16B77
:10F32000884201D3022D28D12A4641462046FEF7C5
:10F33000C6FD0746606A08B9012000E0002068B9F0
:10F3400004F1240000F086FB88B14FF08050324970
:10F350000860BFF34F8FBFF36F8F08E03FB14FF0EE
:10F3600080502D490860BFF34F8FBFF36F8FFFF7B9
:10F370000BFB012007B0BDE8F083059818B9FFF733
:10F3800003FB0020F6E7B9F1000F04D101A8FFF755
:10F390004FFC4FF00109FFF7F7FAFFF7F3FCFFF717
:10F3A000C9FA94F94400401C10B9002084F84400C4
:10F3B00094F94500401C10B9002084F84500FFF77F
:10F3C000E3FA05A901A800F059F9F0B92046FEF7C3
:10F3D0008CFFA0B104F110000599FFF73BFC20461B
:10F3E000FFF73FF900F082FB002895D14FF08050E5
:10F3F00009490860BFF34F8FBFF36F8F8CE720463A
:10F40000FFF72FF900F072FB86E72046FFF729F996
:10F4100000F06CFB0020ADE704ED00E02DE9F05FAB
:10F4200007468A4690461E463C4654B900BF5020C7
:10F4300080F31188BFF34F8FBFF36F8F00BF00BF02
:10F44000FEE7BAF1000F01D1206C08B9012000E0FD
:10F45000002050B900BF502080F31188BFF34F8FB8
:10F46000BFF36F8F00BF00BFFEE7022E02D1E06B3B
:10F47000012801D1012000E0002050B900BF502038
:10F4800080F31188BFF34F8FBFF36F8F00BF00BFB2
:10F49000FEE7FFF7F5FA00BF5021EFF3118081F38B
:10F4A0001188BFF34F8FBFF36F8F00BF0546A06B6E
:10F4B000E16B884201D3022E23D194F945B0324644
:10F4C00051462046FEF7FBFC0BF1010088B9606A4B
:10F4D00008B9012000E0002080B904F1240000F008
:10F4E000B9FA58B1B8F1000F08D00120C8F80000EF
:10F4F00004E00BF1010040B284F845004FF001092F
:10F5000001E04FF0000900BF85F3118800BF4846B5
:10F51000BDE8F09F2DE9F74183B005460E464FF058
:10F5200000082C4654B900BF502080F31188BFF367
:10F530004F8FBFF36F8F00BF00BFFEE70EB9206C87
:10F5400008B9012000E0002050B900BF502080F32E
:10F550001188BFF34F8FBFF36F8F00BF00BFFEE76F
:10F5600000F06EF908B9059808B9012000E0002004
:10F5700050B900BF502080F31188BFF34F8FBFF305
:10F580006F8F00BF00BFFEE700BFFFF7D3F9A76B87
:10F59000F7B131462046FEF77DFC781EA063206956
:10F5A00008B9012000E0002060B904F1100000F06B
:10F5B00051FA38B14FF080502F490860BFF34F8F98
:10F5C000BFF36F8FFFF7E0F9012006B0BDE8F081CF
:10F5D000059818B9FFF7D8F90020F6E7B8F1000F41
:10F5E00004D101A8FFF724FB4FF00108FFF7CCF985
:10F5F000FFF7C8FBFFF79EF994F94400401C10B9CF
:10F60000002084F8440094F94500401C10B9002003
:10F6100084F84500FFF7B8F905A901A800F02EF815
:10F62000F0B92046FEF754FEA0B104F1240005997C
:10F63000FFF710FB2046FFF714F800F057FA0028F8
:10F64000A3D14FF080500C490860BFF34F8FBFF338
:10F650006F8F9AE72046FFF704F800F047FA94E727
:10F660002046FEF7FEFF00F041FA2046FEF730FE8E
:10F6700000288AD00020A8E704ED00E070B5064617
:10F680000C4656B900BF502080F31188BFF34F8F4E
:10F69000BFF36F8F00BF00BFFEE754B900BF50201B
:10F6A00080F31188BFF34F8FBFF36F8F00BF00BF90
:10F6B000FEE7FFF73FF9184802687068131A174809
:10F6C000006890F85A0030B100201449096881F8A8
:10F6D0005A0001251CE02068401C08B9002517E0ED
:10F6E0000F4930680968884204D07068904201D898
:10F6F00001250DE02068984207D92068C01A2060D3
:10F700003046FFF795FA002502E000202060012531
:10F71000FFF73AF9284670BD240A0020100A00209D
:10F72000380A00202DE9FF4F85B0804689461746EC
:10F73000DDE912ABB800FEF7D3FF064656B15C20F8
:10F74000FEF7CEFF04460CB1266304E03046FFF717
:10F7500039F900E000248CB1002084F85900CDE98B
:10F7600000ABCDE902403A4649464046089BFEF7C9
:10F7700098FC2046FEF7D4FA012501E04FF0FF3552
:10F78000284609B0BDE8F08F2DE9F04F85B0074657
:10F79000884691469A46DDE90EB6109C0EB10120CE
:10F7A00000E0002050B900BF502080F31188BFF363
:10F7B0004F8FBFF36F8F00BF00BFFEE70CB101207A
:10F7C00000E0002050B900BF502080F31188BFF343
:10F7D0004F8FBFF36F8F00BF00BFFEE75C20039029
:10F7E00003985C2801D1012000E0002050B900BF3F
:10F7F000502080F31188BFF34F8FBFF36F8F00BF8E
:10F8000000BFFEE7B4B1AEB125462C462E63022000
:10F8100085F85900002004A953464A46CDE900B1B5
:10F82000CDE9025041463846FEF73BFC2846FEF73C
:10F8300077FA01E000200490049805B0BDE8F08F4D
:10F840000549096809B9012005E00449096809B9B1
:10F85000022000E0002070472C0A0020480A002007
:10F860000149086870470000240A00202DE9F04192
:10F870004FF0000843480068002876D142480068ED
:10F88000451C4148056015BB40480068006808B940
:10F89000012000E0002050B900BF502080F3118803
:10F8A000BFF34F8FBFF36F8F00BF00BFFEE7374836
:10F8B00007683748006835490860354807603548AB
:10F8C0000068401C33490860FEF71EFE00BF324846
:10F8D000006885423BD300BF2C480068006808B927
:10F8E000012000E0002020B14FF0FF302A490860DD
:10F8F0002CE026480068C068C4686668B54202D239
:10F900002548066022E0201DFEF7B0FFA06A18B16E
:10F9100004F11800FEF7AAFF2049E06A096888424E
:10F9200002D91E49E06A0860E16A01EB81011C4AC4
:10F9300002EB8100211DFEF7F0FF1A49E06A096819
:10F94000C96A8842C8D34FF00108C5E700BF15480F
:10F950000068C06A00EB8000114951F820000128BE
:10F9600001D94FF0010805E0FFE70F480068401C8F
:10F970000D4908600D48006808B14FF00108404685
:10F98000BDE8F081480A0020240A0020140A002063
:10F99000180A0020380A0020400A0020280A002007
:10F9A0003C590020100A0020300A0020340A0020B0
:10F9B00070B505462C460026002D43D0224800682D
:10F9C000844201D1012000E0002050B900BF502046
:10F9D00080F31188BFF34F8FBFF36F8F00BF00BF5D
:10F9E000FEE7206D50B900BF502080F31188BFF3AF
:10F9F0004F8FBFF36F8F00BF00BFFEE7206D401E2B
:10FA00002065E16CE06A88421CD0206DD0B9201DD1
:10FA1000FEF72CFFE06CE062E06AC0F13800A06104
:10FA20000A49E06A0968884202D90849E06A086020
:10FA3000E16A01EB8101064A02EB8100211DFEF71C
:10FA40006CFF0126304670BD100A0020280A0020F5
:10FA50003C59002070B50646F068C46854B900BF30
:10FA6000502080F31188BFF34F8FBFF36F8F00BF1B
:10FA700000BFFEE704F11800FEF7F8FE1548006825
:10FA8000A0B9201DFEF7F2FE1349E06A096888421A
:10FA900002D91149E06A0860E16A01EB81010F4A6D
:10FAA00002EB8100211DFEF738FF04E004F118018C
:10FAB0000B48FEF732FF0B49E06A0968C96A8842C1
:10FAC00004D9012501200849086000E000252846E6
:10FAD00070BD0000480A0020280A00203C59002080
:10FAE000C45D0020100A0020340A002070B50024F4
:10FAF00000263648006850B900BF502080F31188B6
:10FB0000BFF34F8FBFF36F8F00BF00BFFEE7FEF75D
:10FB100011FF2E480068401E2C4908600846006806
:10FB200000284ED12A48006800284AD023E02948FE
:10FB3000C068C46804F11800FEF798FE201DFEF7A7
:10FB400095FE2549E06A0968884202D92249E06A9F
:10FB50000860E16A01EB8101204A02EB8100211D6E
:10FB6000FEF7DBFE1E49E06A0968C96A884202D3D3
:10FB700001201C4908601748006808B9012000E00E
:10FB800000200028D3D00CB1FEF7BEFC1648056853
:10FB900065B100BFFFF76AFE10B10120114908608E
:10FBA0006D1E002DF6D100200F4908600D48006839
:10FBB00038B1012630070D490860BFF34F8FBFF3FE
:10FBC0006F8FFEF7E1FE304670BD0000480A00204E
:10FBD000200A0020C45D0020280A00203C59002093
:10FBE000100A0020340A0020300A002004ED00E052
:10FBF0002DE9FC4705460E4617469846DDF8289045
:10FC00003020FEF76DFD044654B143463A46314676
:10FC10002846CDE90094FEF7A0FA002084F82C00D5
:10FC20002046BDE8FC872DE9FC4706460F46904676
:10FC30009946DDE90AA5302001900198302801D1CC
:10FC4000012000E0002050B900BF502080F311884F
:10FC5000BFF34F8FBFF36F8F00BF00BFFEE755B9F3
:10FC600000BF502080F31188BFF34F8FBFF36F8F19
:10FC700000BF00BFFEE72C4654B14B464246394612
:10FC80003046CDE900A4FEF768FA012084F82C0084
:10FC90002046BDE8FC87000010B586B00024FEF7C2
:10FCA0009BF816480068D0B100200590049003AA84
:10FCB00004A905A8FEF7FAFD0222DDE904100023DD
:10FCC000CDE9002102900EA10F48039AFFF75CFDD9
:10FCD0000E4908600846006800B1012400BF54B90D
:10FCE00000BF502080F31188BFF34F8FBFF36F8F99
:10FCF00000BF00BFFEE7204606B010BD540A00203A
:10FD0000546D72205376630049E60008580A0020BB
:10FD10002DE9FF4704460D4616461F46DDF83080A4
:10FD20004FF0000954B900BF502080F31188BFF391
:10FD30004F8FBFF36F8F00BF00BFFEE7144800680E
:10FD400010B3009501960294062D15DAFFF778FDA1
:10FD5000022808D10023424669460D480068FFF793
:10FD600089FA814610E000231A466946084800686F
:10FD7000FFF780FA814607E000233A4669460448C7
:10FD80000068FFF74BFB8146484604B0BDE8F087AA
:10FD9000540A002000C1814001C0804101C080415F
:10FDA00000C1814001C0804100C1814000C181404B
:10FDB00001C0804101C0804100C1814000C181403B
:10FDC00001C0804100C1814001C0804101C080412B
:10FDD00000C1814001C0804100C1814000C181401B
:10FDE00001C0804100C1814001C0804101C080410B
:10FDF00000C1814000C1814001C0804101C08041FB
:10FE000000C1814001C0804100C1814000C18140EA
:10FE100001C0804101C0804100C1814000C18140DA
:10FE200001C0804100C1814001C0804101C08041CA
:10FE300000C1814000C1814001C0804101C08041BA
:10FE400000C1814001C0804100C1814000C18140AA
:10FE500001C0804100C1814001C0804101C080419A
:10FE600000C1814001C0804100C1814000C181408A
:10FE700001C0804101C0804100C1814000C181407A
:10FE800001C0804100C1814001C0804101C080416A
:10FE900000C1814000C0C101C30302C2C60607C73A
:10FEA00005C5C404CC0C0DCD0FCFCE0E0ACACB0BAA
:10FEB000C90908C8D81819D91BDBDA1A1EDEDF1FDA
:10FEC000DD1D1CDC14D4D515D71716D6D21213D3CA
:10FED00011D1D010F03031F133F3F23236F6F7377A
:10FEE000F53534F43CFCFD3DFF3F3EFEFA3A3BFB6A
:10FEF00039F9F83828E8E929EB2B2AEAEE2E2FEF1A
:10FF00002DEDEC2CE42425E527E7E62622E2E32389
:10FF1000E12120E0A06061A163A3A26266A6A767B9
:10FF2000A56564A46CACAD6DAF6F6EAEAA6A6BAB29
:10FF300069A9A86878B8B979BB7B7ABABE7E7FBF59
:10FF40007DBDBC7CB47475B577B7B67672B2B37349
:10FF5000B17170B0509091519353529296565797F9
:10FF6000559594549C5C5D9D5F9F9E5E5A9A9B5BE9
:10FF700099595898884849894B8B8A4A4E8E8F4F99
:10FF80008D4D4C8C44848545874746868242438309
:10FF900041818040E00D01080000000000000000E9
:10FFA0000000000000000000000200001800000037
:10FFB0000000000000000000600B010800000000CD
:10FFC000000000000000000000000000000400002D
:10FFD000080000000000000000000000DC0B010829
:10FFE0000000000000000000000000000000000011
:10FFF00000040000080000000000000000000000F5
:020000040801F1
:100000004C0C01080000000000000000000000008F
:1000100000000000000400000800000000000000D4
:1000200000000000BC0C01080000000000000000FF
:1000300000000000000000000002000008000000B6
:100040000000000000000000080D01080000000092
:10005000000000000000000000000000000200009E
:10006000080000000000000000000000480D01082A
:100070000000000000000000000000000000000080
:100080000002000008000000000000000000000066
:10009000880D0108000000000000000000000000C2
:1000A0000000000000020000080000000000000046
:1000B00000000000C80D0108000000000000000062
:1000C0000000000000000000000200000800000026
:1000D0000000000000000000CC0A01080000000041
:1000E000000000000000000000000000000200000E
:1000F000080000000000000000000000480B01089C
:1001000000000000000000000000000000000000EF
:1001100000020000080000000000000000000000D5
:10012000C40B0108000000000000000000000000F7
:1001300000000000000200000200000000000000BB
:1001400000000000E40A01080000000000000000B8
:10015000000000000000000000000000540B010837
:10016000000000000000000000000000000000008F
:1001700000000000D00B010800000000000000009B
:10018000000000000000000000000000400C01081A
:10019000000000000000000000000000000000005F
:1001A00000000000B00C010800000000000000008A
:1001B000000000000000000000000000FC0C01082E
:1001C000000000000000000000000000000000002F
:1001D00000000000100B01080000000000000000FB
:1001E000000000008C0B010800000000000000006F
:1001F00000000000080C01080000000000000000E2
:1002000000000000780C0108000000000000000061
:1002100000000000D80C01080000000000000000F1
:1002200000000000240D0108000000000000000094
:1002300000000000640D0108000000000000000044
:1002400000000000A40D01080000000000000000F4
:1002500000000000D40D01080000000000000000B4
:1002600000000000D80A01080000000000000000A3
:10027000000000003C0B010800000000000000002E
:1002800000000000B80B01080000000000000000A2
:1002900000000000340C0108000000000000000015
:1002A00000000000A40C0108000000000000000095
:1002B00000000000F00C0108000000000000000039
:1002C000000000003C0D01080000000000000000DC
:1002D000000000007C0D010800000000000000008C
:1002E00000000000BC0D010800000000000000003C
:1002F00000000000280B01080100000000000000C1
:1003000000000000A40B0108010000000000000034
:1003100000000000200C01080100000000000000A7
:1003200000000000900C0108010000000000000027
:1003300000000000000B01080000000000000000A9
:10034000000000007C0B010800000000000000001D
:1003500000000000F80B0108000000000000000091
:1003600000000000680C0108000000000000000010
:1003700000000000C80C01080000000000000000A0
:1003800000000000140D0108000000000000000043
:1003900000000000540D01080000000000000000F3
:1003A00000000000940D01080000000000000000A3
:1003B00000000000F00A010800000000000000003A
:1003C000000000006C0B01080000000000000000AD
:1003D00000000000E80B0108000000000000000021
:1003E00000000000580C01080000000000000000A0
:1003F000000000001C0B01080000000000000000CD
:1004000000000000980B0108000000000000000040
:1004100000000000140C01080000000000000000B3
:1004200000000000840C0108000000000000000033
:1004300000000000E40C01080000000000000000C3
:1004400000000000300D0108000000000000000066
:1004500000000000700D0108000000000000000016
:1004600000000000B00D01080000000000000000C6
:100470000000000000000D05100513051605190504
:100480001C051F052205250528052B052E05310510
:100490003305360539053C053F0542054505480548
:1004A0004B054E055105540557055A055D05600578
:1004B0006305660569056C056F05720575057805A8
:1004C0007B057E058105840587058A058D059005D8
:1004D000930596059A059D05A005A305A605A90502
:1004E000AC05AF05B205B605B905BC05BF05C2052B
:1004F000C505C805CC05CF05D205D505D805DB0552
:10050000DF05E205E505E805EB05EF05F205F50574
:10051000F805FB05FF050206050608060C060F0692
:100520001206150618061C061F06220625062906B1
:100530002C062F063306360639063C0640064306CF
:1005400046064A064D065006530657065A065E06EC
:100550006106640668066B066F0672067606790603
:100560007D068106840688068B068F06930696060E
:100570009A069E06A106A506A906AD06B006B40613
:10058000B806BC06C006C306C706CB06CF06D30610
:10059000D706DB06DF06E306E806EC06F006F406FF
:1005A000F906FD06010706070A070F0714071907D2
:1005B0001D07230728072D07330739073F0745077E
:1005C000000000000000000000000000000000002B
:1005D000000000000000000000000000000000001B
:1005E000000000000000000000000000000000000B
:1005F00000000000000000000000000000000000FB
:100600000000000000002205250528052B052E0509
:100610003105340537053A053D05400543054605D6
:1006200049054C054F055205550558055B055E0506
:100630006105640567056A056D0570057305760536
:1006400079057C057F058205850588058B058E0566
:100650009205950598059B059E05A105A405A7058E
:10066000AA05AD05B005B405B705BA05BD05C005B9
:10067000C305C605CA05CD05D005D305D605D905E0
:10068000DD05E005E305E605E905ED05F005F30503
:10069000F605FA05FD050006030606060A060D0620
:1006A0001006130617061A061D062106240627063D
:1006B0002A062E063106340638063B063E0642065A
:1006C000450648064C064F065206560659065C0675
:1006D0006006630667066A066D067106740678068C
:1006E0007B067F06830686068A068D06910695069A
:1006F00098069C06A006A406A706AB06AF06B3069E
:10070000B706BB06BF06C206C606CA06CE06D30695
:10071000D706DB06DF06E306E706EB06F006F4067F
:10072000F906FD06010706070B070F07140719074F
:100730001D07220727072B07300736073B0741070E
:1007400048074E07550700000000000000000000A9
:100750000000000000000000000000000000000099
:100760000000000000000000000000000000000089
:100770000000000000000000000000000000000079
:100780000000000000000000000000000000000069
:100790000000000000000C050F05120515051805E6
:1007A0001B051E0521052405270529052C052F05F8
:1007B0003205350538053B053E054105440547052D
:1007C0004A054D0550055305560559055C055F055D
:1007D0006205650568056B056E057105740577058D
:1007E0007A057D0580058305860589058C059005BC
:1007F0009305960599059C059F05A205A505A805E5
:10080000AB05AE05B105B405B805BB05BE05C10510
:10081000C405C705CA05CD05D005D405D705DA0539
:10082000DD05E005E305E605EA05ED05F005F30560
:10083000F605FA05FD050006030606060A060D067E
:100840001006130617061A061D062006240627069C
:100850002A062E063106340637063B063E064106BA
:10086000450648064B064F065206560659065D06D3
:100870006006640667066B066E06720675067906E4
:100880007C068006840687068B068F0693069606EE
:100890009A069E06A206A606A906AD06B106B506EC
:1008A000B906BD06C106C406C806CC06D006D406E5
:1008B000D806DD06E106E506E906ED06F206F606CF
:1008C000FB06FF06040708070D07120717071C079A
:1008D000210726072B07310736073C074107470743
:1008E0000000000000000000000000000000000008
:1008F00000000000000000000000000000000000F8
:1009000000000000000000000000000000000000E7
:1009100000000000000000000000000000000000D7
:1009200000000000000018051B051E052105240518
:10093000260529052C052F053205350538053B050B
:100940003E0541054405460549054C054F05520540
:10095000550558055B055E056105640567056A0573
:100960006D0570057305760579057C057F058205A3
:10097000850588058B058E059105940597059A05D3
:100980009D05A005A405A705AA05AD05B005B305FD
:10099000B605B905BC05BF05C305C605C905CC0527
:1009A000CF05D205D605D905DC05DF05E205E5054D
:1009B000E905EC05EF05F205F605F905FC05FF056F
:1009C0000306060609060C061006130616061A0686
:1009D0001D062006240627062A062E0631063406A2
:1009E00038063B063F064206450649064C065006B9
:1009F000530657065A065E066106650668066C06CB
:100A00006F06730677067A067E06820685068906D5
:100A10008D069006940698069C06A006A306A706D7
:100A2000AB06AF06B306B706BB06BF06C306C706CE
:100A3000CB06CF06D306D706DC06E006E406E906B9
:100A4000ED06F206F606FB06FF06040709070D078A
:100A5000120717071C07210726072B073007360741
:100A60003B074107470700000000000000000000AE
:100A70000000000000000000000000000000000076
:100A80000000000000000000000000000000000066
:100A90000000000000000000000000000000000056
:100AA0000000000000000000000000000000000046
:100AB000000000000000000000000000010203042C
:100AC0000607080900000000010203046D79546163
:100AD000736B3130000000006D7954696D657231BF
:100AE000300000006D79517565756530310000008A
:100AF0006D79436F756E74696E6753656D30310043
:100B00006D7942696E61727953656D303100000014
:100B10006D7954696D657230310000006D794576EC
:100B2000656E7430310000006D79526563757273C3
:100B30006976654D75746578303100006D794D7555
:100B400074657830310000006D795461736B313118
:100B5000000000006D795175657565303200000048
:100B60006D795461736B3032000000006D79436F12
:100B7000756E74696E6753656D3032006D794269C8
:100B80006E61727953656D30320000006D79546981
:100B90006D657230320000006D794576656E743097
:100BA000320000006D795265637572736976654D28
:100BB00075746578303200006D794D7574657830E4
:100BC000320000006D795461736B31320000000017
:100BD0006D79517565756530330000006D7954612C
:100BE000736B3033000000006D79436F756E74696C
:100BF0006E6753656D3033006D7942696E6172794D
:100C000053656D30330000006D7954696D65723045
:100C1000330000006D794576656E74303300000056
:100C20006D795265637572736976654D7574657813
:100C3000303300006D794D757465783033000000F5
:100C40006D79517565756530340000006D795461BA
:100C5000736B3034000000006D79436F756E7469FA
:100C60006E6753656D3034006D7942696E617279DB
:100C700053656D30340000006D7954696D657230D4
:100C8000340000006D794576656E743034000000E4
:100C90006D795265637572736976654D75746578A3
:100CA000303400006D794D75746578303400000083
:100CB0006D79517565756530350000006D79546149
:100CC000736B3035000000006D7942696E61727996
:100CD00053656D30350000006D7954696D65723073
:100CE000350000006D794576656E74303500000082
:100CF0006D794D7574657830350000006D795175EA
:100D000065756530360000006D795461736B30365F
:100D1000000000006D7942696E61727953656D3033
:100D2000360000006D7954696D6572303600000040
:100D30006D794576656E7430360000006D794D75BD
:100D400074657830360000006D795461736B30370C
:100D5000000000006D7942696E61727953656D30F3
:100D6000370000006D7954696D65723037000000FE
:100D70006D794576656E7430370000006D794D757C
:100D800074657830370000006D795461736B3038CA
:100D9000000000006D7942696E61727953656D30B3
:100DA000380000006D7954696D65723038000000BC
:100DB0006D794576656E7430380000006D794D753B
:100DC00074657830380000006D795461736B303988
:100DD000000000006D7954696D65723039000000C3
:100DE00064656661756C745461736B000C0E010868
:100DF00000000020880A000054050008581001086F
:100E0000880A002048BB00007ECD00085200011374
:100E100001390510091055090300D005010B0032F6
:100E20003DAA55AA550102030405060708090A0B45
:100E30000C0D0E0F101112131415161718191A1B7A
:100E40001C1D1E1F202122232425262728292A2B6A
:100E50002C000120118877AA9908000020390195FB
:100E60005000010003140006ED9505AAAA00012216
:100E700011FA158134060D0A21032A1A100DAABB96
:100E8000CCDDEEDDCCBB3103000202111A810A5227
:100E90004114212852E43A24057103003D40328177
:100EA0001020079BCA51040A0F2E275104E2200785
:100EB00003AE610300046201FF01055FCC4602CB73
:100EC00039CD52090C65795004FE89340B00FF00BE
:100ED000401F541F681F7C1F901FA41FB81FCC1FEA
:100EE000E01FF41F08201C203020442058206C20D4
:100EF00080209420A820BC20D020E420F8200C21C1
:100F00002021342148215C21702184219821AC21A9
:100F1000C021D421E821FC211022242238224C2295
:100F20006022742288229C22B022C422D822EC2281
:100F30000023142328233C235023642378238C2369
:100F4000A023B423C823DC23F023042418242C2456
:100F50004024542468247C249024A424B824CC2441
:100F6000E024F42408251C253025442558256C252B
:100F700080259425A825BC25D025E425F8250C2618
:100F80002026342648265C26702684269826AC2601
:100F9000C026D426E826FC261027242738274C27ED
:100FA0006027742788279C27B027C427D827EC27D9
:100FB0000028142828283C285028642878288C28C1
:100FC000A028B428C828DC28F028042918290C4DAA
:100FD000442C294029542968297C299029A429B81E
:100FE00029CC29E029F429082A1C2A302A442A5825
:100FF0002A6C2A802A942AA82ABC2AD02AE42AF811
:101000002A0C2B202B342B482B5C2B702B842B98F9
:101010002BAC2BC02BD42BE82BFC2B102C820305E4
:10102000FF90053D900D4E120505FF900DFF20032A
:101030000DFF20030D193008231004023006980319
:1010400049075802052FCF4324F4489D9C060D669E
:08105000EC088FAAAAE00900D8
:0400000508000131BD
:00000001FF
